:100000000C9432140C945C140C945C140C945C14DA
:100010000C945C140C945C140C945C140C945C14A0
:100020000C945C140C945C140C945C140C945C1490
:100030000C945C140C94F2750C945C140C945C1489
:100040000C945C140C94AC730C94FBC30C945C1473
:100050000C945F3A0C94553A0C945C140C945C1418
:100060000C945C140C945C140C945C140C945C1450
:100070000C945C140C945C140C945C140C945C1440
:100080000C945C140C945C140C945C144E414E491A
:100090004E495459494E46CDCCCC3D0AD7233C1746
:1000A000B7D13877CC2B329595E6241FB14F0A0093
:1000B0000020410000C84200401C4620BCBE4CCA83
:1000C0001B0E5AAEC59D7400407A10F35A00A07200
:1000D0004E18090010A5D4E80000E8764817000083
:1000E000E40B54020000CA9A3B000000E1F5050051
:1000F0000080969800000040420F000000A086019A
:10010000000000102700000000E803000000006469
:1001100000000000000A00000000000100000000D4
:10012000002C76D888DC674F0823DFC1DFAE59E1A9
:10013000B1B796E5E3E453C63AE651997696E8E618
:10014000C28426EB898C9B62ED407C6FFCEFBC9CEB
:100150009F40F2BAA56FA5F490055A2AF75C936BFD
:100160006CF9676DC11BFCE0E40D47FEF520E6B5B8
:1001700000D0ED902E0300943577050080841E0892
:100180000000204E0A000000C80C333333330F98B0
:100190006E12831141EF8D2114893BE65516CFFE77
:1001A000E6DB18D1844B381BF77C1D901DA4BBE403
:1001B00024203284725E228100C9F124ECA1E53D45
:1001C00027434F4D4D554E49434154494F4E0044EE
:1001D000525952554E004552524F525300494E46C5
:1001E0004F004543484F00486F74656E6420496472
:1001F0006C652054696D656F757400486F74656E29
:10020000642049646C652054696D656F75740A00DB
:100210002121204B494C4C20636175736564206239
:100220007920746F6F206D75636820696E616374E7
:100230006976652074696D65202D2063757272651D
:100240006E7420636F6D6D616E643A200053544F7D
:10025000505045442E20005072696E7465722073B0
:10026000746F707065642064756520746F206572AA
:10027000726F72732E2046697820746865206572EB
:10028000726F7220616E6420757365204D39393943
:1002900020746F20726573746172742E2028546507
:1002A0006D70657261747572652069732072657313
:1002B00065742E20536574206974206166746572BC
:1002C0002072657374617274696E67290A004E6FDB
:1002D00020436865636B73756D2077697468206C63
:1002E000696E65206E756D6265722C204C61737449
:1002F000204C696E653A20004E6F20436865636B41
:1003000073756D2077697468206C696E65206E75F1
:100310006D6265722C204C617374204C696E653A75
:100320002000636865636B73756D206D69736D6123
:100330007463682C204C617374204C696E653A209C
:10034000004C696E65204E756D6265722069732080
:100350006E6F74204C617374204C696E65204E750D
:100360006D6265722B312C204C617374204C696E68
:10037000653A20004D3131300053657269616C205F
:10038000737461747573206D69736D617463680A49
:100390000053442072656164206572726F720A00B6
:1003A0004D6564696120496E7365727465640050BF
:1003B0006C65617365205265736574005052494ED7
:1003C0005445522048414C5445440025533A202579
:1003D0005300706F7765726F6666004B494C4C45F1
:1003E000442E20005072696E7465722068616C74CE
:1003F00065642E206B696C6C28292063616C6C65C8
:1004000064210A006563686F3A004572726F723A40
:10041000000A4D6561737572656420706F696E7452
:10042000733A0A00357835206D6573682E205A209E
:100430006F66667365743A2000206E6F7420656E77
:1004400074657265642E0A0050726F62696E67206F
:10045000506F696E740025532025692F256900208F
:100460006F6620004D424C2047323920706F696E14
:10047000742000290A004A206F7574206F6620726C
:10048000616E67652028302D00290A0049206F75AC
:1004900074206F662072616E67652028302D0047DA
:1004A00032384C30004D6573682070726F62696E2F
:1004B0006720646F6E65004D6573682070726F62AF
:1004C000696E6720646F6E652E0A005374617274E2
:1004D000206D6573682070726F62696E672077693E
:1004E00074682022473239205331222066697273A2
:1004F000742E0A004732395332004732384C300AE2
:10050000473239533200686173206E6F2064617422
:10051000612E0A004D65736820426564204C657643
:10052000656C696E67200053206F7574206F6620BC
:1005300072616E67652028302D35292E0A0020490A
:100540006E76616C6964206578747275646572207A
:1005500000536C6565702E2E2E004D6573682070FB
:100560006F696E74206F7574206F662072616E679C
:10057000650A00436C69636B20746F205265737564
:100580006D652E2E2E004E6F204D6F76652E004528
:100590006E642066696C65206C6973740A0042653C
:1005A00067696E2066696C65206C6973740A004E19
:1005B0006F206D656469610A00706175736500285C
:1005C0006E6F2066696C65290043757272656E7482
:1005D0002066696C653A20005344207072696E741D
:1005E000696E67206279746520004E6F74205344F1
:1005F000207072696E74696E670A002E0A00446585
:100600006C6574696F6E206661696C65642C204648
:10061000696C653A200046696C652064656C657498
:1006200065643A002569730025696D2025697300AA
:100630002569682025696D20256973002569642076
:100640002569682025696D20256973002569792051
:10065000256964202569682025696D202569730056
:100660005072696E742074696D653A20006F6B007A
:100670006F666600E201DD01D601CF01C10144458C
:100680004255473A0020573A0042656420436F6F55
:100690006C696E672E2E2E00426564204865617479
:1006A000696E672E2E2E00544D334420456E6465CE
:1006B0007232204F46462E004649524D5741524510
:1006C0005F4E414D453A4D61726C696E20322E305D
:1006D0002E375F4457372E3320544D334420453254
:1006E000454D444E4E202841707220323420323025
:1006F00032312032313A35373A34372920534F5589
:100700005243455F434F44455F55524C3A687474B9
:1007100070733A2F2F6769746875622E636F6D2F3F
:10072000496E73616E6974794175746F6D61746936
:100730006F6E2F4D61726C696E2F747265652F43F9
:100740007265616C6974794477696E5F322E30200E
:1007500050524F544F434F4C5F56455253494F4EA2
:100760003A312E30204D414348494E455F5459504F
:10077000453A544D334420456E64657232204558E5
:100780005452554445525F434F554E543A312055CB
:100790005549443A63656465326132662D3431618E
:1007A000322D343734382D396231322D633535638B
:1007B00036326633363766660A002F2F004D3134E5
:1007C0003520533C696E6465783E206F7574206FE8
:1007D000662072616E67652028302D31290A00205D
:1007E0005200416363656C65726174696F6E3A2093
:1007F00050005741524E494E4721204C6F77205AA6
:10080000204A65726B206D6179206C65616420748B
:100810006F20756E77616E746564207061757365A5
:10082000732E0A004D32303620580020204D61785A
:100830003A2000200020204D696E3A2000536F6658
:100840007420656E6473746F70733A200046523A78
:100850000020466C6F773A20004D424C2041646A7C
:10086000757374205A0020643A0020693A002070A1
:100870003A00496E76616C696420657874727564BB
:1008800065720A004C434420436F6E747261737446
:100890003A200064697300656E0043290A006162B2
:1008A0006C656420286D696E2074656D702000434E
:1008B0006F6C64206578747275646573206172650D
:1008C00020004F4646004F4E00426564204C65763E
:1008D000656C696E6720004661696C656420746FA1
:1008E00020656E61626C6520426564204C657665AA
:1008F0006C696E670A004D65736820426564204C20
:100900006576656C20646174613A0A00496E7661AF
:100910006C6964206D6573682E0A004D65736820EC
:10092000706F696E74206F7574206F662072616ECF
:1009300067650A004D34323120696E636F727265EB
:10094000637420706172616D657465722075736186
:1009500067650A004F666673657473204170706C3A
:10096000696564004572723A20546F6F2066617247
:100970002100546F6F206661722066726F6D207265
:1009800065666572656E636520706F696E740A00D6
:10099000454550524F4D204F4B0A004D38340044CE
:1009A0006F6E65207072696E74696E672066696C1F
:1009B000650A004D3737004D333100496E76616C62
:1009C00069642065787472756465720A0020573A0C
:1009D00000436F6F6C696E672E2E2E004865617440
:1009E000696E672E2E2E0045202553002364656610
:1009F000696E652044454641554C545F004B642068
:100A0000004B6920004B7020005049442041757410
:100A10006F74756E652066696E6973686564212000
:100A200050757420746865206C617374204B702C51
:100A3000204B6920616E64204B6420636F6E737479
:100A4000616E74732066726F6D2062656C6F7720C3
:100A5000696E746F20436F6E666967757261746941
:100A60006F6E2E680A00504944204175746F74758A
:100A70006E65206661696C6564212074696D656FBF
:100A800075740A00504944204175746F74756E6521
:100A9000206661696C6564212054656D70657261C2
:100AA0007475726520746F6F20686967680A00202A
:100AB0004B643A2000204B693A2000204B703A20CA
:100AC0000020436C617373696320504944200A001D
:100AD0002054753A2000204B753A2000206D617833
:100AE0003A2000206D696E3A200020643A200020F0
:100AF000626961733A2000504944204175746F74F3
:100B0000756E652073746172740A00504944204107
:100B100075746F74756E65206661696C65642120FB
:100B200054656D706572617475726520746F6F20A5
:100B3000686967680A00504944204175746F74758C
:100B40006E65206661696C6564212042616420687D
:100B500065617465722069640A00504944204175DA
:100B6000746F74756E65004572723A2075746638DC
:100B700020666F6E74206E6F7420696E697469618F
:100B80006C697A65642E004572723A207574663815
:100B900020666F6E74206E6F7420696E697469616F
:100BA0006C697A65642E004572723A2075746638F5
:100BB00020666F6E74206E6F7420696E697469614F
:100BC0006C697A65642E00FFE0FFD140A0C8A6A240
:100BD0002FF80023AC00AF10FFFEFF05FFD0FFE0B1
:100BE000FFC1FFD1E240A0C8A6A22FF800238127B1
:100BF000AC00AFFFD0FF64FFD1A5FFD0FF64FF645E
:100C0000FFD1A4FFD0FF16FFFE42656400456E636E
:100C10006C6F73757265002568753A25303268759A
:100C20000025303268753A25303268750020202062
:100C3000202020200020202020003FFFF0380070DE
:100C400030FC3020FC102078102030102C00D02EEA
:100C500031D02F7BD02F7BD02E31D02C00D0203024
:100C60001020781020FC1030FC303800703FFFF06E
:100C70003FFFF03800703186302387102787902F90
:100C800087D02F03D020301020781020781020300B
:100C9000102F03D02F87D0278790238710318630DD
:100CA0003800703FFFF004104002082002082004C2
:100CB00010400820801041001041000820800410DE
:100CC000400000001FFFF81FFFF863616E63656C52
:100CD000005072696E742041626F72746564004DD9
:100CE00032350050617573696E672E2E2E00726565
:100CF00073756D65004D32340046696C2E20446971
:100D0000612E004F6666004F6E004520696E206DB3
:100D10006D5E33005654726176204D696E00566DDB
:100D2000696E00566D6178204500566D6178205AD5
:100D300000566D6178205900566D61782058004149
:100D40006D6178204500416D6178205A00416D61E8
:100D500078205900416D6178205800412D5472610E
:100D600076656C00412D5265747261637400416355
:100D700063656C0056652D4A65726B00565A2D4AA4
:100D800065726B0056592D4A65726B0056582D4A94
:100D900065726B00452073746570732F6D6D005A1A
:100DA0002053746570732F6D6D00592053746570F6
:100DB000732F6D6D00582053746570732F6D6D0027
:100DC000416476616E6365642053657474696E670F
:100DD00073003F0043616E63656C00496E69740087
:100DE0004D34323800496E697469616C697A6520E6
:100DF000454550524F4D0046696C616D656E7400FB
:100E000053746570732F6D6D004A65726B0041639A
:100E100063656C65726174696F6E0056656C6F63B3
:100E20006974790053657420486F6D65204F66665C
:100E30007365747300436F6E666967757261746978
:100E40006F6E004C6576656C696E6720446F6E65E9
:100E500021004D6F7665205A004732395332000029
:100E60000C0F00FE07022503BB017FFE08FE08FEF3
:100E700005080806000040F0C88888987810050822
:100E800008060000C0F88888888888F805050506E7
:100E900000012030F830200508080600002070F816
:100EA00020202020E00509090600FF2070A8A8B82E
:100EB00088887020070505070001D86C366CD805B6
:100EC00009090600FFF8A88888888888A8F8050A14
:100ED0000A0600FE205050505088A8A888700303CE
:100EE0000306000340A040FFFFFFFFFFFFFFFFFFDF
:100EF000FFFFFFFFFFFFFFFFFFFFFFFFFF000000FF
:100F00000605FF01070706020080808080800080C0
:100F1000030303060105A0A0A00506060600005075
:100F2000F85050F8500509090600FF2070A8A0707D
:100F300028A87020050707060000C8C810204098A0
:100F40009805070706000040A0A040A8906801038C
:100F5000030602058080800309090601FF20404046
:100F60008080804040200309090601FF8040402026
:100F7000202040408005070706000020A870207050
:100F8000A8200505050600012020F8202002030303
:100F90000601FFC04080050101060003F8020202BD
:100FA000060100C0C0050707060000081010204019
:100FB0004080050707060000708898A8C88870035D
:100FC000070706010040C040404040E00507070613
:100FD0000000708808102040F8050707060000F898
:100FE0000810300888700507070600001030509080
:100FF000F81010050707060000F880F00808887050
:10100000050707060000304080F088887005070754
:10101000060000F808101020202005070706000031
:1010200070888870888870050707060000708888B7
:1010300078081060020505060100C0C000C0C002AB
:1010400006060601FFC0C000C0408003050506017A
:10105000012040804020050303060002F800F80349
:1010600005050601018040204080050707060000B5
:10107000708810202000200507070600007088B83F
:10108000A8B88070050707060000708888F888886F
:1010900088050707060000F04848704848F0050733
:1010A00007060000708880808088700507070600AA
:1010B00000F04848484848F0050707060000F88057
:1010C00080F08080F8050707060000F88080F08037
:1010D000808005070706000070888080988870056A
:1010E0000707060000888888F888888803070706AD
:1010F0000100E04040404040E0050707060000389E
:101100001010101090600507070600008890A0C01E
:10111000A09088050707060000808080808080F806
:1011200005070706000088D8A8888888880507076B
:101130000600008888C8A898888805070706000068
:1011400070888888888870050707060000F08888FE
:10115000F080808005070706000070888888A890C6
:1011600068050707060000F08888F0A0908805074A
:101170000706000070888070088870050707060061
:1011800000F820202020202005070706000088887E
:101190008888888870050707060000888888885036
:1011A000502005070706000088888888A8A85005F1
:1011B0000707060000888850205088880507070622
:1011C000000088885020202020050707060000F82E
:1011D0000810204080F80309090601FFE0808080A4
:1011E00080808080E00507070600008040402010D6
:1011F00010080309090601FFE020202020202020FC
:10120000E00503030600052050880501010600FEE5
:10121000F8030303060105804020050505060000CC
:1012200070087888780507070600008080F08888B5
:1012300088F00505050600007080808870050707A6
:1012400006000008087888888878050505060000EB
:101250007088F08070050707060000304840E040C5
:1012600040400507070600FE7088888878087005EA
:1012700007070600008080F0888888880307070633
:1012800001004000C0404040E00409090601FE1092
:1012900000301010101090600507070600008080D5
:1012A0008890E09088030707060100C04040404056
:1012B00040E0050505060000D0A8A8A8A80505057A
:1012C000060000B0C88888880505050600007088FB
:1012D0008888700507070600FEF0888888F08080FF
:1012E0000507070600FE7888888878080805050540
:1012F000060000B0C88080800505050600007880E3
:101300007008F00507070600002020F820202018AC
:10131000050505060000888888986805050506000B
:101320000088888850200505050600008888A8A840
:10133000500505050600008850205088050707065F
:1013400000FE88888850204080050505060000F8CA
:10135000102040F80309090601FF2040404080406A
:101360004040200109090602FF8080808080808043
:1013700080800309090601FF804040402040404032
:101380008005030306000248A890FF414253005025
:101390004C41004E65787420506F696E7400256969
:1013A000202F2025750047323953310047323953F9
:1013B0003200436C69636B20746F20426567696E0D
:1013C00000486F6D696E672058595A0053746F72E8
:1013D000652053657474696E6773004C6F61642097
:1013E00053657474696E677300426564205A004FD8
:1013F0006666004F6E00426564204C6576656C69D8
:101400006E67004C6576656C20426564004D6F74B4
:10141000696F6E00426564004E6F7A7A6C650046B3
:10142000616E20537065656400436F6E6669677511
:10143000726174696F6E00526573746F72652044D7
:10144000656661756C7473004C6F616420536574DC
:1014500074696E67730053746F726520536574749A
:10146000696E67730050726568656174202420435B
:101470006F6E66004C434420436F6E7472617374E8
:1014800000416476616E6365642053657474696EAF
:101490006773004D61696E003F004261636B0053EA
:1014A000746F70004D3231005072696E7420667234
:1014B0006F6D204D656469610052656C656173658F
:1014C000204D65646961004D323200436F6E66697C
:1014D0006775726174696F6E0054656D70657261D5
:1014E00074757265004D6F74696F6E005265737527
:1014F0006D65205072696E74004174746163682078
:101500004D656469610054756E650053746F702099
:101510005072696E74005061757365205072696E07
:101520007400496E666F2053637265656E00436197
:101530006E6E6F7420656E74657220737562646977
:10154000723A2000022E2E000152656672657368A1
:10155000004D61696E002100486F74656E642074EF
:101560006F6F20636F6C64004261636B0050726F39
:1015700063656564004D6F74696F6E0044697361E3
:10158000626C65205374657070657273004D3834F9
:1015900000426564204C6576656C696E6700417534
:1015A000746F20486F6D6500473238004D61696E79
:1015B0000050726568656174202420456E64005097
:1015C0007265686561742024204265640054656D0D
:1015D0007065726174757265008F138B13436F6F42
:1015E0006C646F776E0050726568656174202400CA
:1015F00046616E20537065656400426564004E6FFD
:101600007A7A6C65004D61696E004261627973742B
:101610006570205A00466C6F770046616E205370EB
:1016200065656400426564004E6F7A7A6C650042BD
:101630006564205A005370656564004D61696E00F1
:10164000486F6D696E67204661696C6564006F70F4
:10165000656E00545249474745524544003A2000C0
:101660007A5F6D696E00795F6D696E00785F6D6994
:101670006E005265706F7274696E6720656E647378
:10168000746F70207374617475730A0020746F6FC7
:10169000206C6F6E6720657874727573696F6E2049
:1016A00070726576656E7465640A0020636F6C64A1
:1016B00020657874727573696F6E207072657665D7
:1016C0006E7465640A000000000000000000000065
:1016D00000005761726E696E673A20486F6D696EDF
:1016E000672042756D702044697669736F72203C83
:1016F00020310A00020204000016430000164300D5
:10170000004843000000410000004100000040008C
:10171000001643000016430000484300000000008C
:101720000000000000000053657474696E67732048
:1017300053746F72656400454550524F4D20496E99
:10174000697469616C697A65640A003B2000202035
:101750004D3235302043004C434420436F6E747249
:101760006173743A0020440020490020204D33303A
:10177000312050005049442073657474696E67735A
:101780003A0020460020420020480020204D3134FD
:10179000352053004D6174657269616C2068656124
:1017A00074757020706172616D65746572733A0052
:1017B0002020473239205334205A00204A0020206C
:1017C00047323920533320490020204D3432302015
:1017D00053004D65736820426564204C6576656CE6
:1017E000696E673A0020204D323036205800486F2D
:1017F0006D65206F66667365743A0020580020534B
:101800000020204D323035204200416476616E6305
:1018100065643A20423C6D696E5F7365676D656E05
:10182000745F74696D655F75733E20533C6D696EBE
:101830005F66656564726174653E20543C6D696ED7
:101840005F74726176656C5F66656564726174650C
:101850003E20583C6D61785F785F6A65726B3E2010
:10186000593C6D61785F795F6A65726B3E205A3CC6
:101870006D61785F7A5F6A65726B3E20453C6D6191
:10188000785F655F6A65726B3E00205400205200ED
:1018900020204D323034205000416363656C657206
:1018A0006174696F6E2028756E6974732F733229A5
:1018B0003A20503C7072696E745F616363656C3E80
:1018C00020523C726574726163745F616363656C1E
:1018D0003E20543C74726176656C5F616363656C35
:1018E0003E0020204D3230312058004D6178696D26
:1018F000756D20416363656C65726174696F6E20FC
:1019000028756E6974732F7332293A0020204D3286
:1019100030332058004D6178696D756D20666565BE
:101920006472617465732028756E6974732F7329EE
:101930003A0053746570732070657220756E697417
:101940003A0020440020204D323030205300204403
:10195000697361626C65640A0046696C616D656EED
:10196000742073657474696E67733A0020204D317A
:1019700034392043203B20556E69747320696E20F2
:1019800043656C736975730A0020286D6D2900200A
:1019900020473231202020203B20556E697473206F
:1019A000696E206D6D0000803B4400803B44000068
:1019B0002041000096420000A0420000A04200002A
:1019C000C8430000BE42D0070000D00700006400FA
:1019D00000004B00000024F4D43050C38E20C2A27B
:1019E0004017828B7011127A910D816CD90AA8610F
:1019F000E108C7586607615143061E4B5D05C145A6
:101A0000A7041A411104093D980371393103403686
:101A1000DB0265339102D4305402802E1D02632C08
:101A2000EE01752AC501B028A001102781018F257C
:101A300064012B244B01E0223401AC211F018D20D5
:101A40000D01801FFC00841EED00971DDF00B81CF7
:101A5000D200E61BC600201BBC00641AB200B219FB
:101A6000A8000A19A0006A189900D1179100401720
:101A70008B00B516840031167E00B31579003A1537
:101A80007300C7146F0058146A00EE1366008813C1
:101A9000630025135E00C7125B006C12570015121D
:101AA0005400C111510070114F0021114B00D6108C
:101AB00049008D1047004610440002104200C00F3C
:101AC0004000800F3E00420F3C00060F3B00CB0E53
:101AD0003800930E37005C0E3500270E3400F30DEE
:101AE0003200C10D3100900D3000600D2E00320D1E
:101AF0002D00050D2C00D90C2B00AE0C2900850CF7
:101B000029005C0C2700350C27000E0C2600E80B82
:101B10002400C40B2400A00B23007D0B23005A0BD0
:101B20002100390B2100180B2000F80A1F00D90AE8
:101B30001E00BB0A1E009D0A1D00800A1D00630ACC
:101B40001C00470A1B002C0A1B00110A1A00F70987
:101B50001A00DD091900C4091900AB09190092091E
:101B600017007B091800630917004C091600360995
:101B70001600200916000A091500F5081500E008EE
:101B80001400CC081400B8081400A408140090082D
:101B900013007D0812006B08130058081200460855
:101BA0001200340811002308110012081100010866
:101BB0001100F0071000E0071000D0071000C00768
:101BC0001000B0070F00A107100091070E00830757
:101BD0000F0074070F0065070E0057070E00490736
:101BE0000E003B070D002E070E0020070D00130707
:101BF0000D0006070D00F9060C00ED060D00E006CD
:101C00000C00D4060C00C8060C00BC060C00B00684
:101C10000C00A4060B0099060C008D060B00820632
:101C20000B0077060B006C060B0061060A005706D6
:101C30000B004C060A0042060A0038060A002E066F
:101C40000A0024060A001A060A0010060900070600
:101C50000A00FD050900F4050900EB050900E2058D
:101C60000900D9050900D0050900C7050900BE050E
:101C70000900B5050800AD050800A50509009C058B
:101C80000800940508008C050800840508007C0500
:101C90000800740508006C050700650508005D056F
:101CA0000700560508004E050700470507004005D8
:101CB000080038050700310507002A05070023053D
:101CC00007001C050600160507000F05070008059C
:101CD000060002050700FB040600F5040700EE04F9
:101CE0000600E8040600E2040700DB040600D50451
:101CF0000600CF040600C9040600C3040600BD04A4
:101D00000600B7040600B1040500AC040600A604F2
:101D10000600A00405009B0406009504050090043D
:101D200006008A04050085040500800406007A0484
:101D3000050075040500700405006B0405006604C9
:101D40000500610405005C04050057040500520409
:101D500005004D04050048040500430405003E0449
:101D600004003A04050035040500300404002C0486
:101D7000050027040400230405001E0404001A04BF
:101D8000040016040500110404000D0404000904F5
:101D900005000404040000040400FC030400F8032C
:101DA0000400F4030400F0030400EC030400E8035F
:101DB0000400E4030400E0030400DC030400D8038F
:101DC0000400D4030400D0030400CC030400C803BF
:101DD0000300C503030024F404D9201BC40C5C0ECB
:101DE0009804C4095F0265077101F405F900FB045A
:101DF000B30048048700C10369005803550003037A
:101E00004500BE023A008402310053022A00290232
:101E1000250004022000E4011C00C8011900AF01E4
:101E20001700980114008401130071011000610172
:101E3000100051010E0043010D0036010B002B0173
:101E40000B0020010B00150109000C010900030122
:101E50000800FB000800F3000800EB000700E400A6
:101E60000600DE000600D8000600D2000600CC0006
:101E70000500C7000500C2000500BD000400B90050
:101E80000400B5000400B1000400AD000400A90086
:101E90000400A5000300A20003009F0004009B00B3
:101EA00003009800030095000200930003009000D7
:101EB00003008D0002008B000300880002008600F2
:101EC000020084000300810002007F0002007D0008
:101ED00002007B000200790002007700010076001A
:101EE00002007400020072000100710002006F0025
:101EF00002006D0001006C0002006A000100690030
:101F00000200670001006600010065000100640036
:101F100002006200010061000100600001005F003A
:101F200002005D0001005C0001005B0001005A003E
:101F3000010059000100580001005700010056003F
:101F4000010055000100540001005300000053003F
:101F500001005200010051000100500001004F003B
:101F600001004E0000004E0001004D0001004C0039
:101F700001004B0000004B0001004A000100490035
:101F80000100480000004800010047000100460031
:101F9000000046000100450000004500010044002B
:101FA0000100430000004300010042000000420025
:101FB00001004100000041000100400001003F001D
:101FC00000003F0001003E0000003E0001003D0017
:101FD00000003D0001003C0000003C0000003C000F
:101FE00001003B0000003B0001003A0000003A0005
:101FF00001003900000039000100380000003800FD
:1020000000003800010037000000370001003600F2
:1020100000003600000036000100350000003500E9
:1020200000003500010034000000340000003400DE
:1020300001003300000033000000330001003200D3
:1020400000003200000032000100310000003100C9
:1020500000003100010030000000300000003000BE
:1020600001002F0000002F0000002F0000002F00B3
:1020700001002E0000002E0000002E0001002D00A7
:1020800000002D0000002D0000002D0001002C009C
:1020900000002C0000002C0000002C0001002B0090
:1020A00000002B0000002B0000002B0001002A0084
:1020B00000002A0000002A0000002A000100290078
:1020C000000029000000290000002900000029006C
:1020D000010028000000280000002800000028005F
:1020E0000000280001002700000027000000270052
:1020F0000000270000002700010026000000260045
:102100000000260000002600000026000100250037
:10211000000025000000250000002500000025002B
:10212000000025000100240000002400000024001D
:102130000000240000002400010023000000230010
:102140000000230000002300000023000000230003
:1021500000002300010022000000220000002200F5
:1021600000002200000022000000220001002100E7
:1021700000002100000021000000210000002100DB
:1021800000002100000021000100200000002000CC
:1021900000002000000020000000200000002000BF
:1021A000000020000000200001001F0000001F00B0
:1021B00000001F0000001F0000001F0000001F00A3
:1021C00000001F0001001E0000001E0000001E0095
:1021D00000001E000000043700001E290000511BF3
:1021E00000005810000010090000CC040000780224
:1021F00000004101000020436F756E7420583A00C2
:1022000042656400453100626564002C2073797377
:1022100074656D2073746F7070656421204865610A
:102220007465725F49443A200048656174696E675D
:10223000204661696C65640048656174696E672059
:102240006661696C6564004D313132205368757484
:10225000646F776E001000C90210012C014001224A
:102260000170011801B0010E01F00104015002FAE1
:1022700000B002F0003003E600D003DC009004D28E
:10228000007005C800A006BE000008B400B009AA8E
:1022900000D00BA000600E960060118C000015822B
:1022A0000020197800C01D6E00A0226400B0275ADB
:1022B00000902C500000314600E0343C00103832D1
:1022C00000903A2800603C1E00A03D1400803E0AA9
:1022D00000203F0000544845524D414C2052554E7D
:1022E0004157415900546865726D616C2052756E9A
:1022F00061776179004572723A204D415854454DDD
:1023000050004D415854454D5020747269676765BF
:10231000726564004572723A204D494E54454D50E5
:10232000004D494E54454D5020747269676765727F
:10233000656400202F002042403A0020403A007C93
:102340003C3E5E2B3D3F2F5B5D3B2C2A225C0043D5
:10235000616E6E6F74206F70656E20737562646954
:1023600072200053442063617264206F6B0A006F17
:1023700070656E526F6F74206661696C65640A00E7
:10238000766F6C756D652E696E6974206661696C17
:1023900065640A004E6F20534420636172640A0032
:1023A0000A4D3234004D3233202573002E0A006F5F
:1023B00070656E206661696C65642C2046696C6589
:1023C0003A200046696C652073656C6563746564CA
:1023D0000A002053697A653A200046696C65206FCF
:1023E00070656E65643A2000454E44205355425254
:1023F0004F5554494E450A002220706F7300222029
:10240000706172656E743A2200535542524F5554B2
:10241000494E452043414C4C207461726765743AC3
:10242000220053756263616C6C204F766572666C36
:102430006F77004578636565646564206D61782019
:10244000535542524F5554494E4520646570746847
:102450003A0057726974696E6720746F2066696C00
:10246000653A2000667265736800646F696E670084
:102470002066696C653A20004E6F7720002F6175E9
:10248000746F25632E67006001F4017001EA01900A
:1024900001E001B001D601D001CC010002C201303F
:1024A00002B8016002AE019002A401D0029A01209C
:1024B00003900170038601C0037C0130047201A007
:1024C00004680120055E01B005540160064A012040
:1024D000074001F0073601F0082C01100A220150D4
:1024E0000B1801C00C0E01500E04013010FA002030
:1024F00012F0005014E600C016DC007019D2005033
:102500001CC800501FBE007022B400B025AA00F005
:1025100028A000202C9600302F8C0010328200A0C2
:10252000347800F0366E00E0386400803A5A00409B
:102530003B5500E03B5000F03C4600C03D3C006095
:102540003E3200E03E2800303F1E00503F19007030
:102550003F1400A03F0A00C03F0000D03FF6FFE05C
:102560003FECFF2020506C616E6E657242756666AE
:10257000657242797465733A200020467265652061
:102580004D656D6F72793A2000436F6D70696C65AF
:10259000643A2041707220323420323032310A00E5
:1025A000204C61737420557064617465643A203204
:1025B0003032312D30342D3138207C204175746813
:1025C0006F723A2054696E794D616368696E657304
:1025D00033440A00322E302E375F4457372E330AE9
:1025E000004D61726C696E0020536F667477617282
:1025F000652052657365740A0020576174636864CE
:102600006F672052657365740A002042726F776E9F
:10261000206F75742052657365740A0020457874C4
:1026200065726E616C2052657365740A00506F7735
:10263000657255700A0073746172740A004732380B
:102640005859004D31303031006F6B006572726F38
:10265000722077726974696E6720746F2066696C86
:10266000650A00446F6E6520736176696E67206647
:10267000696C652E0A004D323900456E6473746FC3
:1026800070730025532025632025632025632025B2
:102690006300205A3A0020593A0020583A00656EEB
:1026A0006473746F7073206869743A2000000000CE
:1026B000010200090A0000000004030807000000EE
:1026C00000000000000000000000000000004D6F4E
:1026D00076652025736D6D004D6F766520302E3147
:1026E0006D6D004D6F766520316D6D004D6F7665B7
:1026F0002031306D6D004D6F766520417869730033
:102700004578747275646572004D6F7665205A0065
:102710004D6F76652059004D6F76652058005072D8
:10272000696E742066726F6D204D6564696100FF8B
:10273000FFFF486F6D65202573257325732046695B
:1027400072737400220A00556E6B6E6F776E206391
:102750006F6D6D616E643A202200544D3344204504
:102760006E646572322052656164792E0050726920
:102770006E74696E672E2E2E005072696E74205032
:10278000617573656400204500205A0020590020BF
:102790004D393220580020453A00205A3A0020593D
:1027A0003A00583A004572726F7220777269746904
:1027B0006E6720746F20454550524F4D210A00200E
:1027C000746F6F206C6F6E672065787472757369B3
:1027D0006F6E2070726576656E7465640A002063A2
:1027E0006F6C6420657874727573696F6E20707297
:1027F0006576656E7465640A00526573656E643A49
:10280000200000002200250028002B0000002100ED
:10281000240027002A00020202020202020204042B
:102820000404040404040303030303030303010176
:102830000101010101010102040810204080010290
:1028400004081020408001020408102040808040CD
:102850002010080402012F2F616374696F6E3A0023
:1028600012D7E5DD11241FBECFEFD0E4DEBFCDBF10
:1028700012E0A0E0B1E0ECE1F8ED01E00BBF02C036
:1028800007900D92A631B107D9F727E1A6E1B2E092
:1028900001C01D92A13BB207E1F714E1C1E3D4E10D
:1028A00004C02197FE010E946CE9C033D107C9F72B
:1028B0000E9436D80C9401EC0C9400008F929F92E9
:1028C000AF92BF92CF92DF92EF92FF92CF936B01C4
:1028D0007C0120E030E0A9010E9487E287FD9FC0D3
:1028E0006DEB77E386E095E3A70196010E947EE910
:1028F0006B017C0120E030E040E251E40E94EDE217
:1029000020E030E048EC52E40E94EDE24B015C0133
:1029100020E030E0A901C701B6010E9487E220E073
:1029200030E040EA50E487FF04C020E030E040EAB5
:1029300050ECC501B4010E947EE920E030E040E2A5
:1029400051E40E9401EA0E9473EA6B017C018BE270
:10295000F7FE09C0F094E094D094C094C11CD11C3F
:10296000E11CF11C8DE28093DC03C701B60120E17C
:1029700037E240E050E00E944DE98AE0882E912C39
:10298000A12CB12CCA01B901A50194010E944DE905
:10299000605D6093DD03C701B60128EE33E040E0DF
:1029A00050E00E944DE9CA01B901A50194010E94BD
:1029B0004DE9605D6093DE03C701B60124E630E0B7
:1029C00040E050E00E944DE9CA01B901A50194011F
:1029D0000E944DE9605D6093DF038EE28093E00327
:1029E000C701B601A50194010E944DE9C62FCA0195
:1029F000B901A50194010E944DE9605D6093E10376
:102A0000C05DC093E2038CED93E0CF91FF90EF9017
:102A1000DF90CF90BF90AF909F908F9008956DEB17
:102A200077E386E095EB60CF8F929F92AF92BF9253
:102A3000CF92DF92EF92FF92CF936B017C0120E067
:102A400030E0A9010E9487E287FDAAC06DEB77E321
:102A500086E095E3A70196010E947EE96B017C0167
:102A600020E030E0A9010E9487E287FF9EC0C701F5
:102A7000B601905820E030E040E251E40E94EDE2DF
:102A800020E030E040E251E40E94EDE220E030E05E
:102A900040EA50E40E947EE920E030E040E251E468
:102AA0000E9401EA0E9473EA6B017C0180E280933C
:102AB000DC0360E280E1C81687E2D806E104F10495
:102AC0008CF0C701B60120E137E240E050E00E94FF
:102AD0004DE9CA01B9012AE030E040E050E00E942F
:102AE0004DE9605D6093DD0360E288EEC81683E027
:102AF000D806E104F1048CF0C701B60128EE33E0FA
:102B000040E050E00E944DE9CA01B9012AE030E0FE
:102B100040E050E00E944DE9605D6093DE0360E2BA
:102B200084E6C816D104E104F1048CF0C701B601B3
:102B300024E630E040E050E00E944DE9CA01B901CE
:102B40002AE030E040E050E00E944DE9605D609393
:102B5000DF038AE0882E912CA12CB12CC701B6018D
:102B6000A50194010E944DE9C62FCA01B901A50132
:102B700094010E944DE9605D6093E0038EE28093D2
:102B8000E103C05DC093E2038CED93E0CF91FF9031
:102B9000EF90DF90CF90BF90AF909F908F9008956F
:102BA0006DEB77E386E095EB55CF20E030E040E237
:102BB00051E4C701B60162CFCF93DF93EC01CB01A3
:102BC000BA010E948EE220E030E040E251E40E942F
:102BD00001EA20E030E0A9010E947EE96883798360
:102BE0008A839B83DF91CF9108950E948EE220E03B
:102BF00030E040E251E40E9401EA20E030E0A90127
:102C00000E947EE90C941415CF93DF93EC01CB0165
:102C1000BA010E948EE220E030E048EC52E40E94CB
:102C200001EA20E030E0A9010E947EE9688379830F
:102C30008A839B83DF91CF9108950E948EE220E0EA
:102C400030E048EC52E40E9401EA20E030E0A901C3
:102C50000E947EE90C945E14CF93DF93EC01CB01CC
:102C6000BA010E948EE220E030E0A9010E947EE9D4
:102C7000688379838A839B83DF91CF910895CF9373
:102C8000DF93EC01CB01BA010E948EE220E030E03C
:102C9000A9010E947EE9688379838A839B83DF91FF
:102CA000CF910895CF93DF93EC01CB01BA010E943D
:102CB0008EE22AE037ED43E25DE30E9401EA20E084
:102CC00030E0A9010E947EE90E947AEA6883798354
:102CD0008A839B83DF91CF910895CF93DF93EC019B
:102CE000CB01BA010E948EE22AE037ED43E25DE3B8
:102CF0000E9401EA20E030E0A9010E947EE9688399
:102D000079838A839B83DF91CF910895CF93DF935B
:102D1000EC01CB01BA010E948EE220E030E04AE7EC
:102D200054E40E9401EA20E030E0A9010E947EE91B
:102D3000688379838A839B83DF91CF910895FC0117
:102D400084910895FC0180810895FC0180E09191B7
:102D5000992329F0907C9038D1F38F5FF8CF0895B4
:102D600090E080E00895CF93DF93DB01F9019C911F
:102D70009130C1F0943080F094509C938830D1F41D
:102D800080819181009771F0019791838083480F32
:102D9000591FEA01188206C08C3539F49C5F9C9358
:102DA000943041F4DF91CF9108958B3339F781E06E
:102DB0008C93F8CF20813181B9016F5F7F4F718390
:102DC0006083420F531FEA018883808191818F3590
:102DD00091056CF7E7CF0F931F9381E00091C11627
:102DE0001091C2162091C3163091C4164091BD16A1
:102DF0005091BE166091BF167091C016041715074A
:102E00002607370708F480E01F910F910895282FB7
:102E100090913803833021F495FD0FC094FD0FC0CD
:102E2000892F90E0B0E0A0E004C0B695A7959795F3
:102E300087952A95D2F78170089581E0089580E002
:102E4000089580915501882341F06091D7037091D6
:102E5000D80341E081E00C9472BE089563E972E00A
:102E600084E690E00E94A6966AEB72E084E690E029
:102E70000C94A69681110C942E1768EB71E084E1F6
:102E800090E00C94A696CF93DF9300D000D0CDB7FE
:102E9000DEB70E947AEA0E948CE269837A838B8390
:102EA0009C83CE0101960E94CA920F900F900F90C2
:102EB0000F90DF91CF9108950E948EE22AE037EDC6
:102EC00043E25DE30E9401EA20E030E0A9010E94B4
:102ED0007EE90C944317CF92DF92EF92FF92CF934B
:102EE000DF9300D000D0CDB7DEB76B017C0120E0CE
:102EF00030E0A9010E9487E287FD1BC06DEB77E3FC
:102F000086E095E3A70196010E947EE969837A83B2
:102F10008B839C83CE0101960E94CA920F900F90E2
:102F20000F900F90DF91CF91FF90EF90DF90CF90B7
:102F300008956DEB77E386E095EBE4CF0E948EE297
:102F40002AE037ED43E25DE30E9401EA20E030E051
:102F5000A9010E947EE90C946B170E948EE220E08A
:102F600030E0A9010E947EE90C946B17CF92DF92AA
:102F7000EF92FF926B017C0120E030E0A9010E94FA
:102F800087E287FD26C06DEB77E386E095E3A70136
:102F900096010E947EE96B017C0120E030E0A901EE
:102FA0000E9487E220E030E040E05FE387FF04C05A
:102FB00020E030E040E05FEBC701B6010E947EE90F
:102FC0000E9473EACB01FF90EF90DF90CF900C94BA
:102FD00068946DEB77E386E095EBD9CF0E948EE2A3
:102FE00020E030E0A9010E947EE90C94B6170E940F
:102FF0008EE220E030E04AE754E40E9401EA20E05B
:1030000030E0A9010E947EE90C94D396EF92FF92E2
:103010000F931F9382EDE82E8DE0F82E05EE1DE054
:1030200030E020E041E85CE164ED7DE08BED9DE087
:103030000E9478C61F910F91FF90EF9008950E9413
:103040006D760C943A170E9422910C942E170C94D2
:1030500080790C9480790C9480790C9480790C940C
:1030600032790C9432790C9432790C9432790E9432
:10307000C0A80C943A1720914003022E000C330B89
:103080008217130641F0809340036FE57EE089E4E8
:1030900095E10C941AC80895EF92FF920F931F9335
:1030A000CF93DF93EC018B017A018A859B8586178C
:1030B000970731F0888199810E941AC81B870A8777
:1030C000B701888199810E9448BF2E813F81820F7C
:1030D000932F911D9F838E8390E080E0DF91CF91AD
:1030E0001F910F91FF90EF9008959F92AF92BF9222
:1030F000CF92DF92EF92FF920F931F93CF93DF93C4
:10310000EC018B01942EA52E8A859B858617970747
:1031100031F0888199810E941AC81B870A878885A7
:103120009985019649F5BC800A818E81080FC88077
:10313000D980D6015596ED91FC91C6010995B80E3E
:10314000E92CFA2C10E0F70121917F01211127C011
:103150008E819F81810F911D9F838E8390E080E0FF
:10316000DF91CF911F910F91FF90EF90DF90CF9063
:10317000BF90AF909F9008950E811F81692D7A2D89
:10318000888199810E9448BF800F912F911D2885C9
:1031900039852817390738F681E090E0E1CF4B2DCB
:1031A000602FC6010E9472C8080F180FCCCFDF92A3
:1031B000EF92FF920F931F93CF93DF93EC01D62EE4
:1031C0001CAD0BAD7C0184E0E80EF11CE98DFA8D9D
:1031D000C7010995412F480F2D2D602FC7010E946F
:1031E00072C89BAD890F8BAF81E090E0DF91CF91EA
:1031F0001F910F91FF90EF90DF900895AF92BF92D3
:10320000DF92EF92FF920F931F93CF93DF938C0186
:10321000EB01D42E79018FE0481709F486C0A5E1AF
:103220004A17B1F1BAE04B130EC0EC81FD8130E0DA
:1032300020E042E061E0C80109954CED5BE0BE0191
:10324000C8010E941DC90A80DB81C02DF2E3DF1690
:1032500009F4E2C0FD1508F491C085E1D81609F41F
:10326000E0C0A7E1DA1609F4EFC0B4E1DB127BC0DD
:10327000EE81FF818D8190E0880F991F8E0F9F1F37
:1032800011928E179F07E1F7CE010E945BC46BC0BD
:10329000AA80BB8047EC5BE0C8010E941DC9F50114
:1032A0004481440F406BBE01C8010E9405C941E042
:1032B000BE01C8010E940DC9D50116962D913C9101
:1032C0001797EC81FD8115964C9166E0C801099530
:1032D00040E0BE01C8010E9415C947EC5BE0BE0199
:1032E000C8010E941DC9F5014481440F4F5F406B26
:1032F000BE01C8010E9405C941E0BE01C8010E948B
:103300000DC9D50115964C91159716962D913C91A6
:10331000240F311DEC81FD8166E0C801099540E074
:10332000BE01C8010E9415C98ECF41E0C8010E94AC
:1033300015C940E0BE01C8010E940DC941E8BE01A7
:10334000C8010E9405C9F701408150E05595479595
:1033500055954795BE01C8010E9405C940E0BE01D0
:10336000C8010E9415C981E0DF91CF911F910F9193
:10337000FF90EF90DF90BF90AF900895E6E4DE16E7
:1033800009F471C0F7E4DF1609F471C08BE3D812B9
:10339000EACFD70111969C91119713968C9138E042
:1033A000390F813031F0833011F0392F02C0392FBD
:1033B000985021E04B81491708F420E041E039178B
:1033C00008F040E091E05A81351708F490E0322F80
:1033D000342B932311F4242331F2F701128100E0FE
:1033E000D12C843048F490E0FC01E859FE4FD080A5
:1033F0008C599E4FDC010C9117FF04C0B701CE0120
:103400000E9462C4F70180818D0D80838181800FCD
:103410008183110F89F7A7CFB701CE010E9462C443
:10342000A2CFCE010E9445C4882309F49DCFEE812E
:10343000FF818D8190E0880F991F8E0F9F1F119241
:103440008E179F07E1F78FCFD7011C928A811196C3
:103450008C9311978D81815012968C9312978B814A
:1034600013968C9380CF8D81F70180837CCF8981E7
:10347000D7018C9378CFCF92DF92EF92FF920F9388
:103480001F93CF93DF93CDB7DEB72C970FB6F89489
:10349000DEBF0FBECDBFF0908015E090811520916A
:1034A000420321111DC047E85BE06E2D8F2D0E9465
:1034B000DEC890E080E0F80EF0928015E092811571
:1034C00099272C960FB6F894DEBF0FBECDBFDF91C3
:1034D000CF911F910F91FF90EF90DF90CF900895C3
:1034E000C0904D15D0904E1529E435E13A832983DB
:1034F0002F2D30E03C832B832E2D30E03E832D8317
:1035000018861F827A8769871C861B8605E718E163
:103510009E012F5F3F4F4FE956E1BC01C6010E945B
:10352000B9B8B60189E495E10E941AC88F819885DF
:10353000C2CFEF92FF920F931F93CF937C01009124
:103540003B0310913C03C0E0F701EC0FF11D6081DB
:10355000662351F0062E000C770BC8010E94C7EBC2
:10356000892B49F4CF5FF0CF80E0CF911F910F916D
:10357000FF90EF90089581E0F8CF682F880F770BC8
:1035800080913B0390913C030E94C7EBFC0181E0DA
:10359000309709F480E0309781F0918120ED290F78
:1035A0002A3030F09E3251F4928190539A3098F440
:1035B0003196F0932D03E0932C0308959D3211F082
:1035C0009B3249F4928120ED290F2A3088F39E32F4
:1035D00011F49381EACFF0E0E0E0EBCF80912C038F
:1035E00090912D03009731F04AE050E070E060E0E8
:1035F0000C94A9E060E070E0CB01089580912C0369
:1036000090912D03009731F04AE050E070E060E0C7
:103610000C947BDF60E070E0CB0108950E94FE1AFD
:10362000CB0108950F931F93CF9380912C0390911A
:103630002D030097E9F0FC018F01C1912C2F2F7D04
:1036400081F0C53411F0C536B9F7F801108270E089
:1036500060E00E941DDEF801C083CF911F910F91A1
:10366000089570E060E0CF911F910F910C941DDEE2
:1036700060E070E0CB01F1CFCF93DF93CDB7DEB741
:1036800020E24F8158856E818D810E94CFBEDF91EF
:10369000CF9108958F929F92AF92BF92EF92FF9237
:1036A0000F931F93CF93DF93EC018B01E42EF22E47
:1036B00080914315909144158C179D0709F43EC0E5
:1036C0002091D10327FD1092D1032CE9C63AD207ED
:1036D00009F03FC08155934371F40E945AC36E5163
:1036E0007B4F8F4F9F4F6093D3037093D40380938E
:1036F000D5039093D603D0934415C093431530E07F
:1037000020E00093D3051093D4052093D505309382
:10371000D605E092CE05F092CF05C155D34321F4F2
:103720001092CD051092D20382E08093550181E082
:103730008093D0051092DB031092CC05DF91CF91DE
:103740001F910F91FF90EF90BF90AF909F908F903F
:10375000089523E3C135D20771F6865A9C4919F0C2
:10376000C1E5D3E3C8CF0E945AC38090D3039090A1
:10377000D403A090D503B090D603681979098A09BB
:103780009B0997FFEDCF80919B058770873041F7AC
:10379000C5EFD5E6B0CF80911D1590911E15891B00
:1037A0008F7051F48091F805813031F08091C51609
:1037B00082FB882780F9089581E00895E091D20383
:1037C000E63010F581E08E0F8093D2034091D3054F
:1037D0005091D4056091D5057091D6059091CE0594
:1037E0008091CF0528E0E29FF0011124EE56FC4FB6
:1037F00020914315309144153183208342835383B4
:10380000648375839683878308952F923F924F92A6
:103810005F926F927F928F929F92AF92BF92CF9260
:10382000DF92EF92FF920F931F93CF93DF9300D01D
:1038300000D000D0CDB7DEB71C017A8369832B831B
:103840003C834D835E832701380181E08093D0055E
:103850000E94DE1B83E0809355013092D0032092BA
:10386000CF0389819A819093CE038093CD038B817E
:103870009C81AD81BE818093C9039093CA03A093BC
:10388000CB03B093CC034092C5035092C603609221
:10389000C7037092C803F12CE12CC092D305D092DB
:1038A000D405E092D505F092D605B0924415A092C9
:1038B00043159092C4038092C3038B8D8093C203FF
:1038C00026960FB6F894DEBF0FBECDBFDF91CF9125
:1038D0001F910F91FF90EF90DF90CF90BF90AF902E
:1038E0009F908F907F906F905F904F903F902F9020
:1038F000089520E040E070E060E081E593E30C94FF
:103900004A1BCF930E9422910E946D76C82F882374
:1039100019F080E00E94CEA28C2F0E943A17CF911E
:103920000C94791CE091D203EE2389F0E150E093EE
:10393000D20388E0E89FF0011124EE56FC4F62812B
:10394000738127814681808191810C944A1B0C945C
:10395000791C8091D903811106C01092CD050E9477
:10396000921C0E942E1780915501882331F041E06E
:1039700063E47EE081E00E9472BE82E080935501A4
:1039800008954F925F926F927F928F929F92AF9223
:10399000BF92CF92DF92EF92FF920F931F93CF933C
:1039A000DF930E94CB1B782E0E9488BFC091CE056A
:1039B00015E0711001C016E06C2E85E0582E5C0EEB
:1039C00005E00C1B84E0F82EFC1A83E0E82EEC1ACC
:1039D00082E0982E9C1A90EEA92E9DE0B92E24E24A
:1039E000C22E2EE0D22E81E0882E8C1A4C2E4194CD
:1039F000C11132C08091D105882389F08091550191
:103A0000882309F447C081E09091D105911180E0AD
:103A100024E045E35EE0642D0E94CFBE3BC0809170
:103A2000CB051092CB05882349F30E94921C80910C
:103A3000D005882319F3DF91CF911F910F91FF904B
:103A4000EF90DF90CF90BF90AF909F908F907F903E
:103A50006F905F904F900895C13009F05BC08091E6
:103A6000D105813009F443C080915501882391F03C
:103A70001F92DF92CF928F9281E09091D105913089
:103A800009F080E08F930E943C1B0F900F900F90E5
:103A90000F900F90711079C0C53009F076C08091F9
:103AA000D105853009F49EC0809155018111ABC0CC
:103AB000D6E081E08D0F8C1313C09091D1059C1737
:103AC00009F4CCC080915501882351F06C2F661900
:103AD00081E09C1380E023E045EE5DE00E94CFBED4
:103AE000CF5FC51185CFDE5FD093CF05A4CF809186
:103AF000CB051092CB05882309F4B6CFB092A90567
:103B0000A092A8050E94791C8091D005882309F411
:103B1000ABCF91CFC23009F0C2C08091D1058230C5
:103B200081F080915501882309F4B4CF81E0909110
:103B3000D105923009F080E023E04BE15EE0692D91
:103B40006BCF8091CB051092CB05882351F38BE886
:103B500095E20E9407978091D005882311F36BCFDF
:103B60008091D1058330F1F080915501882309F4CB
:103B700091CF81E09091D105933009F080E023E06E
:103B80004EE05EE06E2D0E94CFBE1C1309C08091F6
:103B9000D105811709F444C080915501811151C0AC
:103BA000D12F87CF8091CB051092CB058823E1F2EE
:103BB0008BE597E20E9407978091D0058823A1F2B8
:103BC0003ACF8091CB051092CB05882309F472C0BF
:103BD00088E59AE20E9407978091D005882309F42E
:103BE00069C029CF8091CB051092CB05882309F4B9
:103BF0005BCF8EE39CE20E9407978091D0058823DB
:103C000009F452CF18CF81E09091D105953009F099
:103C100080E023E040E05EE0602F0E94CFBE48CF0E
:103C20008091CB051092CB05882309F4B5CF8DE6A2
:103C30009DE20E9407978091D005882309F4ACCFBC
:103C4000FACE6C2F661981E09091D1059C1380E02B
:103C500023E047EF5DE00E94CFBEA2CF8091CB056D
:103C60001092CB05882309F42DCF0E94DE1B20E0A3
:103C700040E070E060E086E098E1DF91CF911F9135
:103C80000F91FF90EF90DF90CF90BF90AF909F90FB
:103C90008F907F906F905F904F900C944A1BC33031
:103CA00009F45ECFC43009F0F5CE8091D10584309F
:103CB00009F487CF80915501882309F4EBCE81E088
:103CC0009091D105943009F080E023E049E05EE076
:103CD0006F2D59CFCF93DF93CDB7DEB78D81909104
:103CE0008E12891768F080938E129E01285F3F4FD5
:103CF0004E815F816AE270E083E692E10E944EE2CB
:103D0000DF91CF9108950F931F93CF93DF938C0191
:103D10006F3F19F410928E1260E020918E12862F60
:103D2000062E000C990B2817190609F0F4F460937D
:103D30008E12C8010E94D4E1800F911FEC01C01BBC
:103D4000D10BCB32D1053CF00197FC012491207CB2
:103D50002038D1F3F3CFDD27AE01B80183E692E13D
:103D60000E94F5E1CD59DD4E1882DF91CF911F9170
:103D70000F910895CF9380918A03811109C083EE3A
:103D80009CE09093D8038093D70381E080938A03CB
:103D90000E94DE1B20E040E070E060E081E297E1FD
:103DA0000E944A1BC1E0C093CD050E94A4791092E5
:103DB000CD050E94921CC093CD0560E089E797E293
:103DC0000E94831E8FED9CE09093A9058093A80527
:103DD000CF91089510928903109254018091C516D5
:103DE00080648093C5168AEC9CE00E94E6B760E090
:103DF00081ED9CE00E94831E0C94791C0F931F930D
:103E00000E945AC300918503109186032091870375
:103E100030918803601B710B820B930B97FD0CC0D4
:103E200089B183FB882780F991E089274A9B8260CA
:103E3000309B84608093840380918403817090918F
:103E4000840391FD826090918303981749F081303B
:103E500009F148F0823079F0833091F08093830348
:103E60001F910F910895913079F09230B9F79091A8
:103E7000820391500CC0992339F09330C1F3EECFF7
:103E80009130A9F3923051F7909182039F5F909304
:103E90008203E4CF992359F3933001F7F5CFCF9202
:103EA000DF92EF92FF92CF93C82F0E945AC36B010B
:103EB0007C0124EA30E74DE75FE360911B017091DC
:103EC0001C0180911D0190911E010E9487E287FDD7
:103ED00018C08AEF90E0A0E0B0E08C0D9D1DAE1DF3
:103EE000BF1D8093720390937303A0937403B093E8
:103EF0007503C0931901CF91FF90EF90DF90CF90A1
:103F0000089580E090E0DC01E8CFFC01A081B18160
:103F10001C92A281B3818C918F5F8C930280F3817C
:103F2000E02D90818CE0989F800D1124E5E4F5E16F
:103F300013AE84AF0895FC0180E09491992331F091
:103F4000907C903809F08F5F3196F7CF0895AF924B
:103F5000BF92CF92DF92EF92FF920F931F93CF9376
:103F6000DF93EC015B018A01FB01099587FD16C017
:103F7000C82ED12CF12CE12C2196F801C082D182DF
:103F8000E282F382CE01DF91CF911F910F91FF90DA
:103F9000EF90DF90CF90BF90AF900895982F907ED4
:103FA000903CA9F48F7190E0B0E0A0E06C017D013D
:103FB00056E0CC0CDD1CEE1CFF1C5A95D1F7CE014F
:103FC0000196F50109958F73C82A2296D6CF982FAE
:103FD000907F903E11F58F7090E0B0E0A0E06C0112
:103FE0007D0136E0CC0CDD1CEE1CFF1C3A95D1F7B0
:103FF000CE010196F50109958F73C82A46E0CC0CD5
:10400000DD1CEE1CFF1C4A95D1F7CE010296F5018E
:1040100009958F73C82A2396B0CF982F987F903F29
:1040200079F5877090E0B0E0A0E06C017D0186E05A
:10403000CC0CDD1CEE1CFF1C8A95D1F7CE0101963D
:10404000F50109958F73C82A96E0CC0CDD1CEE1C97
:10405000FF1C9A95D1F7CE010296F50109958F7351
:10406000C82A26E0CC0CDD1CEE1CFF1C2A95D1F7DB
:10407000CE010396F50109958F73C82A24967DCF4A
:10408000982F907C903841F4807C803869F4219698
:10409000CE01F5010995F8CF8E7F8D3F28F021964E
:1040A000CE01F5010995F8CFC12CD12C760165CF51
:1040B0009CE0899F802D112491E0980F90934103FB
:1040C0002CE0280F2093DC0530E02E5F3F4F40911D
:1040D0007D154217130619F014F080E00895209121
:1040E0007F159217D0F7662341F08E5F0E94C4C5FA
:1040F0008091DC058E5F0E94C4C58091DC059091A3
:104100007D15891750F320917F1590914103291750
:1041100020F3109280158093811581E008951F93FC
:10412000CF93DF931F92CDB7DEB78F3F910519F084
:1041300014F08FEF90E08837910514F488E790E051
:104140009093420180934101182F80918215811133
:1041500005C081E0809382150E94A3C460914B1535
:1041600070914C1519839E012F5F3F4F4FE089E4FA
:1041700095E10E9478C40F90DF91CF911F9108952F
:10418000CF938091430381114EC0109280151092FD
:1041900081151092821510924E1510924D151092A5
:1041A000501510924F151092521581E080935115C1
:1041B00082E2809353151092581510925715ECE631
:1041C000F5E18FEF819395E1EA37F907D9F7C1E07F
:1041D000C093691526E639EA30935F1520935E1582
:1041E000C0936015109261151092621590E490933F
:1041F00063151092641524E439EA30937B152093FB
:104200007A1521E131E030934C1520934B159CE158
:1042100090936E159EE190936D1580936C150E949E
:10422000A3C4C093430380914101909142010E9435
:104230008F2081E08093420387E19CE09093971464
:1042400080939614109299141092981453985B9A34
:1042500052985A9A3898409A0E94FE1E10928203F1
:10426000CF910895CF92DF92EF92FF920F931F9319
:10427000CF93DF93CDB7DEB72C970FB6F894DEBFA0
:104280000FBECDBF6F3F71058105910509F0D0F4D8
:1042900085E495E10E94D718E0914D15F0914E15F7
:1042A0003196849190E02C960FB6F894DEBF0FBE45
:1042B000CDBFDF91CF911F910F91FF90EF90DF90D5
:1042C000CF900895F0908015E090811520914203E1
:1042D00021110FC047EA5BE06E2D8F2D0E94DEC8D2
:1042E00090E080E0F80EF0928015E0928115992719
:1042F000DACFC0904D15D0904E1529E435E13A83C0
:1043000029832F2D30E03C832B832E2D30E03E83FC
:104310002D8318861F822FEF3FEF3A8729871C864F
:104320001B8605E718E19E012F5F3F4FAB01BC01E3
:10433000C6010E94F5B7B60189E495E10E941AC84A
:104340008F819885CFCFAF92BF92CF92DF92EF92BD
:10435000FF920F931F93CF93DF9300D000D0CDB780
:10436000DEB77C01062F6A01122F86E0A82EB12C41
:1043700011160CF040C0AE014F5F5F4F6FE976E160
:10438000C7010E94A71F7C0169817A818B819C8172
:10439000611571058105910571F16D337105810517
:1043A000910509F450C06E3771058105910509F436
:1043B0004AC06A3271058105910569F507FF12C08F
:1043C0008DE09CE00E3F11F089E09CE026E01202B7
:1043D000B00111240E943B1A66E070E00E9439E9A6
:1043E000161B61C065E470E080E090E00E9432211D
:1043F000115059F510E0812F0F900F900F900F90F2
:10440000DF91CF911F910F91FF90EF90DF90CF90B0
:10441000BF90AF900895643271058105910579F4DC
:10442000C114D10461F026E01202B0011124C601CA
:104430000E943B1AB5010E9439E9161B99CF0E94D0
:104440003221115095CF07FDBBCF61E089819A8160
:10445000AB81BC81CD97A105B10509F460E0600F87
:104460006A30ACF01150862F6AE00E9417E9092FDC
:10447000682F880F770B605D7F4F072E000C880B2D
:10448000990B0E943221112309F4B4CF602F062E1C
:10449000000C770B605D7F4F072E000C880B990B8B
:1044A0000E9432211150112309F4A4CF86E0180292
:1044B000B0011124C7010E943B1A66E070E00E941F
:1044C00039E9161B98CF6FEF7FEF0C943B1ACF9210
:1044D000DF92EF92FF920F931F93CF93DF93CDB7AD
:1044E000DEB72C970FB6F894DEBF0FBECDBFF090AD
:1044F0008015E09081152091420321111DC047E6EF
:104500005BE06E2D8F2D0E94DEC890E080E0F80EFB
:10451000F0928015E092811599272C960FB6F894A9
:10452000DEBF0FBECDBFDF91CF911F910F91FF90E6
:10453000EF90DF90CF900895C0904D15D0904E151C
:1045400029E435E13A8329832F2D30E03C832B8306
:104550002E2D30E03E832D8318861F827A8769874F
:104560001C861B8605E718E19E012F5F3F4F42EA3C
:1045700056E1BC01C6010E94B9B8B60189E495E1D3
:104580000E941AC88F819885C2CF6FEF7FEF0C947D
:104590006722AF92BF92CF92DF92EF92FF920F937A
:1045A0001F93CF93DF935C016B010E949B1FE82E4A
:1045B000C6010E94A516F12C03E110E0081B1109A9
:1045C000C5E20E151F050CF4CFE18C2F90E09C0185
:1045D0002E5F3F4F40917D154217130609F0CCF531
:1045E000099720917F15281719069CF14091DE0547
:1045F0005091DF056091DD0510928015C093811503
:1046000025E1C5010E94A321D1E0C114D104B1F07C
:104610006AE370E080E090E00E9432210E151F05F1
:10462000D4F4C45F80917D15C81740F020917F15A8
:104630004C2F4950550B241715067CF4DF91CF9170
:104640001F910F91FF90EF90DF90CF90BF90AF90B0
:104650000895D0E0DACFDD2389F3802F880F080F8B
:10466000000F00938015C093811560E270E080E038
:1046700090E00E943221C601DF91CF911F910F91EE
:10468000FF90EF90DF90CF90BF90AF900C94C52239
:10469000CF92DF92EF92FF92CF93DF9300D000D0C2
:1046A000CDB7DEB78091CB051092CB05882331F1D1
:1046B0008091DA038F5F8093DA038931E0F081E043
:1046C0008093D90320E040E070E060E089EA9CE15B
:1046D0000E944A1B89E59EE09093A9058093A80556
:1046E0000F900F900F900F90DF91CF91FF90EF9070
:1046F000DF90CF9008950E94A0A2F2CF6091D305E1
:104700007091D4058091D5059091D60561157105FC
:104710008105910509F43EC00E948EE22DEC3CEC2F
:104720004CEC5CE30E94EDE22091440B3091450B90
:104730004091460B5091470B0E947EE96B017C0132
:1047400020E030E040E850EC0E9487E287FD53C053
:1047500020E030E040E850E4C701B6010E9401EBE0
:1047600018160CF44FC0C092440BD092450BE09247
:10477000460BF092470B84E891E00E94678782E045
:10478000809355011092D3051092D4051092D5054F
:104790001092D60580915501882309F4A1CFC090CD
:1047A000440BD090450BE090460BF090470B20E077
:1047B00030E0A901C701B6010E9487E227E137EB8B
:1047C00041ED58E387FF04C027E137EB41ED58EB9B
:1047D000C701B6010E947EE969837A838B839C833B
:1047E0006BE2CE0101960E944D93BC0182E59EE0F2
:1047F0000E94C92275CFC12CD12C90E8E92E90ECF3
:10480000F92EB1CFC12CD12C80E8E82E80E4F82E0F
:10481000AACF0F931F93CF93DF93FC01EB018091FD
:10482000D3059091D405A091D505B091D605B7FFD9
:1048300008C01092D3051092D4051092D50510929D
:10484000D6058091C5039091C603A091C703B0918E
:10485000C8034091D3055091D4056091D50570915E
:10486000D60584179507A607B70744F48093D305A8
:104870009093D405A093D505B093D60580915501AA
:104880008823E1F06091D3057091D4058091D5051E
:104890009091D6050091C9031091CA032091CB03D2
:1048A0003091CC03600F711F821F931F0995BC01CB
:1048B0008091CF039091D0030E94C9228091CB05B3
:1048C000811108C08091C2038823D1F180915501E4
:1048D0008823B1F18091CD039091CE030097B1F080
:1048E0004091D3055091D4056091D5057091D605BE
:1048F0000091C9031091CA032091CB033091CC03DE
:10490000400F511F621F731FFE010995E091C30301
:10491000F091C403309741F08091C203811103C02C
:104920008091CB05811109958091CB051092CB0523
:10493000882331F0DF91CF911F910F910C94921C3D
:10494000DF91CF911F910F9108956CED75E185EF87
:1049500095E10C94092464E076E18DE196E10C94F4
:1049600009246FE376E18EEE97E10C94092462E569
:1049700076E18CE597E10C9409246DE676E18EE909
:1049800097E10C9409246CE276E18DEA97E10C94AE
:10499000092466E876E187EF97E10C9409248F9269
:1049A0009F92AF92BF92CF92DF92EF92FF920F93BE
:1049B0001F93CF93DF93CDB7DEB72C970FB6F89444
:1049C000DEBF0FBECDBF982F862F5A017901D02EA2
:1049D000692F0E945820882309F487C01091420350
:1049E000C701002381F10E949B1FC82E80904D15A6
:1049F00090904E15111143C01FEF23E12C194091E7
:104A0000DE055091DF056091DD05C5010E94A321FF
:104A1000CC2009F46AC0B6E08B9F500111246AE3F0
:104A200070E080E090E00E94322157E0A516B104CA
:104A300008F442C060E270E080E090E00E94322121
:104A4000A81AB90AF2CF0E94A516C82E80904D155B
:104A500090904E15112381F2FE0133968AE0DF011A
:104A60001D928A95E9F789E495E19A8389830CE49C
:104A700018E19E012F5F3F4F42EA56E112C0FE014E
:104A800033968AE0DF011D928A95E9F789E495E182
:104A90009A8389830CE418E19E012F5F3F4F4FE911
:104AA00056E1B701C4010E94B9B8B40189E495E1A7
:104AB0000E941AC81F81A1CF4091DC05212F30E050
:104AC000A6E0CA9EC00111242E5F3F4F2817390768
:104AD0000CF49C0180E8821B809380154093811523
:104AE000C701DD20A9F00E9463222C960FB6F8942E
:104AF000DEBF0FBECDBFDF91CF911F910F91FF9011
:104B0000EF90DF90CF90BF90AF909F908F900895DF
:104B10000E94C522EACF7F928F929F92AF92BF925E
:104B2000CF92DF92EF92FF920F931F93CF93DF9379
:104B30000E9488BFC091CE0565E0862E8C0ED6E01F
:104B4000DC1B85E0D82EDC1A84E0C82ECC1A83E06A
:104B5000B82EBC1A82E0A82EAC1A81E0982E9C1ABE
:104B60007C2E7194C11134C08091D1058823B1F09D
:104B700080915501882359F081E09091D1059111E0
:104B800080E024E040EC5DE0672D0E94CFBECF5F67
:104B9000C811E8CF87E08093CF050CC08091CB058A
:104BA0001092CB05882321F30E94921C8091D0059E
:104BB0008823F1F2DF91CF911F910F91FF90EF9039
:104BC000DF90CF90BF90AF909F908F907F9008958F
:104BD000C130E9F58091D1058130E9F0809155012E
:104BE0008823A9F211E08091D105813009F010E00D
:104BF0006091180B7091190B80911A0B90911B0BFF
:104C00000E946B1700E09C0148E35DE0692D812F55
:104C10000E94CF24BCCF8091CB051092CB05882376
:104C2000E9F20E947CBFE12C1CE3F12E0CE116E4BA
:104C300020E030E040E85FE368E17BE088E39DE06E
:104C40000E94DEBF8091D005882341F2B3CFC230ED
:104C500009F006C18091D1058230D9F080915501CB
:104C6000882309F494CF11E08091D105823009F0B6
:104C700010E060911C0B70911D0B80911E0B9091A8
:104C80001F0B0E946B1700E09C0141E35DE06A2D61
:104C9000BECF8091CB051092CB058823F9F20E94FC
:104CA0007CBFE12C1CE3F12E0CE116E420E030E0A7
:104CB00040E85FE36CE17BE081E39DE00E94DEBFC2
:104CC0008091D005882351F275CF8091D105833032
:104CD000D9F080915501882309F459CF11E08091D2
:104CE000D105833009F010E06091200B7091210B09
:104CF0008091220B9091230B0E946B1700E09C0186
:104D00004AE25DE06B2D83CF8091CB051092CB05FD
:104D10008823F9F20E947CBFE12C1CE3F12E0CE108
:104D200016E420E030E040E85FE360E27BE08AE206
:104D30009DE00E94DEBF8091D005882351F23ACFDA
:104D40008091D1058430D9F080915501882309F4F0
:104D50001ECF11E08091D105843009F010E0609100
:104D6000240B7091250B8091260B9091270B0E94AC
:104D70006B1700E09C0143E25DE06C2D48CF809111
:104D8000CB051092CB058823F9F20E947CBFE12C61
:104D90001CE3F12E0CE116E420E030E040E85FE394
:104DA00064E27BE083E29DE00E94DEBF8091D0055B
:104DB000882351F2FFCE8091D1058530D9F08091C2
:104DC0005501882309F4E3CE11E08091D1058530A7
:104DD00009F010E06091340B7091350B8091360B27
:104DE0009091370B0E946B1700E09C014EE15DE053
:104DF0006D2D0DCF8091CB051092CB058823F9F254
:104E00000E947CBFE12C1CE3F12E0CE116E420E0B3
:104E100030E0A90164E37BE08EE19DE00E94DEBF0B
:104E20008091D005882359F2C5CE8091CB05109290
:104E3000CB05882329F10E947CBFE12C1CE3F12ED5
:104E40000CE116E420E030E0A90168E37BE084E1B6
:104E50009DE00E94DEBF8091D005882389F0AACE14
:104E6000C33009F432CFC43009F46ACFC53009F435
:104E7000A2CFC63009F08BCE8091D1058630A9F241
:104E800080915501882309F482CE11E08091D105EB
:104E9000863009F010E06091380B7091390B8091E9
:104EA0003A0B90913B0B0E946B1700E09C0144E190
:104EB0005DE06D2FACCE2F923F924F925F926F923A
:104EC0007F928F929F92AF92BF92CF92DF92EF929A
:104ED000FF920F931F93CF93DF93CDB7DEB72C973D
:104EE0000FB6F894DEBF0FBECDBFC090F80AD090C9
:104EF000F90AE090FA0AF090FB0A8091FC0A90917E
:104F0000FD0AA091FE0AB091FF0A8C159D05AE0521
:104F1000BF0510F4D701C601C090F40AD090F50A7D
:104F2000E090F60AF090F70ABC01CD016C157D0502
:104F30008E059F0510F4C701B6010E948CE22B017B
:104F40003C010E9488BF2091CE052B872E83822FA3
:104F50008B5F8D8387E0922F821B8F8386E0821B7D
:104F6000888785E0821B898784E0821B8A8783E0AB
:104F7000282E221A82E0382E321A91959C872B8592
:104F8000211142C08091D1058823C9F0809155013B
:104F9000882359F081E09091D105911180E024E0BF
:104FA00040EC5DE06C850E94CFBE8B858F5F8B8768
:104FB0009D819813E4CF88E08093CF050CC0809149
:104FC000CB051092CB05882309F30E94921C809197
:104FD000D0058823D9F22C960FB6F894DEBF0FBE09
:104FE000CDBFDF91CF911F910F91FF90EF90DF9098
:104FF000CF90BF90AF909F908F907F906F905F9079
:105000004F903F902F9008958B85813009F08BC091
:105010008091D1058130F9F080915501882329F2E2
:1050200011E08091D105813009F010E06091280BEA
:105030007091290B80912A0B90912B0B0E946B177A
:1050400061E02E81621B00E09C014EE65DE0812F55
:105050000E94CF24AACF8091CB051092CB05882344
:10506000D9F20E947CBF2AE037ED43E25DE3C30141
:10507000B2010E94EDE220E030E0A9010E947EE949
:105080004B015C0120E030E040E05FE40E9487E2F9
:1050900087FD05C0812C912CA12C3FE4B32E2AE082
:1050A00037ED43E25DE36091280B7091290B80910D
:1050B0002A0B90912B0B0E94EDE220E030E0A90139
:1050C0000E947EE920E030E040E85FE30E947DE955
:1050D0000E947AEA69837A838B839C83C501B40139
:1050E0000E9473EA7B018C0121E0E21AF1080109B8
:1050F00011091F92912C812C2DEBA22E24E2B22EAD
:10510000C980DA8021E030E040E050E068E27BE0F6
:105110008EE69DE00E94051C0F908091D0058823AB
:1051200009F47ACF58CF8B85823009F090C18091F5
:10513000D1058230D9F080915501882309F435CF0B
:1051400011E08091D105823009F010E060912C0BC4
:1051500070912D0B80912E0B90912F0B0E946B174D
:1051600000E09C0144E65DE0632D71CF8091CB05AA
:105170001092CB058823F9F20E947CBF6091000B4E
:105180007091010B8091020B9091030B0E948CE2B5
:105190007B018C0120E030E048EC52E46CE27BE0E3
:1051A00084E69DE00E94DEBF8091D005882319F23D
:1051B00012CF8091D1058330D9F080915501882399
:1051C00009F4F3CE11E08091D105833009F010E0AD
:1051D0006091300B7091310B8091320B9091330BB9
:1051E0000E946B1700E09C014BE55DE0622D2FCF24
:1051F0008091CB051092CB058823F9F20E947CBFE9
:105200002AE037ED43E25DE3C301B2010E94EDE223
:1052100020E030E0A9010E947EE94B015C0120E022
:1052200030E040E05FE40E9487E287FD05C0812C0A
:10523000912CA12C9FE4B92E2AE037ED43E25DE3E7
:105240006091300B7091310B8091320B9091330B48
:105250000E94EDE220E030E0A9010E947EE920E01A
:1052600030E040E85FE30E947DE90E947AEA6983CA
:105270007A838B839C83C501B4010E9473EA7B010E
:105280008C0121E0E21AF108010911091F92912C09
:10529000812C8DEBA82E84E2B82EC980DA8021E023
:1052A00030E040E050E060E37BE08BE59DE00E9471
:1052B000051C0F908091D005882309F47ECF8BCEFA
:1052C0008091D1058430E9F080915501882309F45B
:1052D0006CCE11E08091D105843009F010E060912E
:1052E000F40A7091F50A8091F60A9091F70A0E94EB
:1052F0008CE20E94431700E09C0144E55DE06A8572
:10530000A6CE8091CB051092CB058823E9F20E94AE
:105310007CBF05E318E124E630E040E050E064EFB4
:105320007AE084E59DE00E947DC08091D0058823CD
:1053300059F251CE8091D1058530E9F08091550127
:10534000882309F432CE11E08091D105853009F02F
:1053500010E06091F80A7091F90A8091FA0A909130
:10536000FB0A0E948CE20E94431700E09C014DE47E
:105370005DE069856CCE8091CB051092CB058823CA
:10538000E9F20E947CBF03E318E124E630E040E04C
:1053900050E068EF7AE08DE49DE00E947DC080914E
:1053A000D005882359F217CE8091D1058630E9F0D7
:1053B00080915501882309F4F8CD11E08091D10541
:1053C000863009F010E06091FC0A7091FD0A80912E
:1053D000FE0A9091FF0A0E948CE20E94431700E0AF
:1053E0009C0146E45DE0688532CE8091CB05109249
:1053F000CB058823E9F20E947CBF01E318E12AE093
:1054000030E040E050E06CEF7AE086E49DE00E94FE
:105410007DC08091D005882359F2DDCD8091CB05E8
:105420001092CB05882339F10E947CBF0FE218E16E
:1054300024E630E040E050E060E07BE08FE39DE078
:105440000E947DC08091D0058823A9F0C4CD2B8512
:10545000233009F4AECE243009F432CF253009F4DC
:1054600069CF263009F4A0CF273009F09ECD809176
:10547000D105873099F280915501882309F495CDA3
:1054800011E08091D105873009F010E06091000BA8
:105490007091010B8091020B9091030B0E948CE2A2
:1054A0000E94431700E09C014FE35DE06F81CFCD88
:1054B0003F924F925F926F927F928F929F92AF92A4
:1054C000BF92CF92DF92EF92FF920F931F93CF93F1
:1054D000DF930E9488BFC091CE05A5E04A2E4C0EF6
:1054E000D4E0DC1B83E0782E7C1A82E0682E6C1AF4
:1054F00081E0582E5C1A3C2E3194C11138C0809145
:10550000D1058823B1F080915501882359F081E0BD
:105510009091D105911180E024E040EC5DE0632D95
:105520000E94CFBECF5FC411E8CF85E08093CF0546
:105530000CC08091CB051092CB05882321F30E94EB
:10554000921C8091D0058823F1F2DF91CF911F91B9
:105550000F91FF90EF90DF90CF90BF90AF909F9012
:105560008F907F906F905F904F903F900895C130E3
:1055700009F05DC08091D1058130E9F0809155013D
:10558000882381F211E08091D105813009F010E08B
:1055900060910706709108068091090690910A06AD
:1055A0000E94B61700E09C014CE85DE0652D812F5C
:1055B0000E94CF24B7CF8091CB051092CB058823D2
:1055C000E9F20E947CBF20E030E0A901609107066B
:1055D000709108068091090690910A060E947EE962
:1055E00020E030E040E85FE30E947DE90E947AEA33
:1055F0001F92912C812CE1EBAE2EE4E2BE2E6B01CA
:105600001DEDE12E13E0F12E00E010E021E030E08E
:1056100040E050E067E076E08CE89DE00E94051CE9
:105620000F908091D005882309F4A8CF8ECFC23087
:1056300009F0FEC08091D1058230D9F080915501EA
:10564000882309F46FCF11E08091D105823009F0F1
:1056500010E060910B0670910C0680910D06909100
:105660000E060E94B61700E09C0144E85DE0662D3E
:105670009ECF8091CB051092CB058823F9F20E9432
:105680007CBF20E030E0A90160910B0670910C0610
:1056900080910D0690910E060E947EE920E030E098
:1056A00040E85FE30E947DE90E947AEA1F92912C14
:1056B000812C41EBA42E44E2B42E6B011DEDE12EB2
:1056C00013E0F12E00E010E021E030E040E050E097
:1056D0006BE076E084E89DE00E94051C0F908091CD
:1056E000D005882309F4AACF30CF8091D10583302B
:1056F000D9F080915501882309F414CF11E08091ED
:10570000D105833009F010E060910F06709110060A
:1057100080911106909112060E945E1400E09C0197
:105720004CE75DE0672D43CF8091CB051092CB0510
:105730008823F9F20E947CBF20E030E048EC52E47C
:1057400060910F06709110068091110690911206DB
:105750000E94EDE220E030E0A9010E947EE920E015
:1057600030E040E251E40E947DE90E947AEA1F9213
:10577000912C812C2BEAA22E24E2B22E6B011EEA80
:10578000E12E12E8F12E01E010E02AE030E040E0E6
:1057900050E06FE076E08CE79DE00E94051C0F90E2
:1057A0008091D005882309F4A4CFCFCE8091CB057A
:1057B0001092CB05882309F446C00E947CBF20E0EC
:1057C00030E048EC52E46091130670911406809129
:1057D0001506909116060E94EDE220E030E0A90146
:1057E0000E947EE920E030E040E251E40E947DE941
:1057F0000E947AEA1F92912C812C8BEAA82E84E2D7
:10580000B82E6B011EEAE12E12E8F12E01E010E045
:105810002AE030E040E050E063E176E084E79DE09C
:105820000E94051C0F908091D005882361F08DCED9
:10583000C33009F45ACFC43009F074CE8091D10539
:10584000843009F4B3CF80915501882309F46ACEDE
:1058500011E08091D105843009F010E060911306C9
:105860007091140680911506909116060E945E14A0
:1058700000E09C0144E75DE06D2F99CEBF92CF928E
:10588000DF92EF92FF920F931F93CF93DF930E94CB
:1058900088BFC091CE0585E0C82ECC0ED4E0DC1BBD
:1058A00013E01C1B82E0F82EFC1A81E0E82EEC1AB3
:1058B000BC2EB194C11130C08091D1058823B1F0C4
:1058C00080915501882359F081E09091D105911183
:1058D00080E024E040EC5DE06B2D0E94CFBECF5F06
:1058E000CC11E8CF85E08093CF050CC08091CB052B
:1058F0001092CB05882321F30E94921C8091D00541
:105900008823F1F2DF91CF911F910F91FF90EF90DB
:10591000DF90CF90BF900895C130B9F58091D10547
:105920008130F1F0809155018823C9F2DD24D394B0
:105930008091D105813009F0D12C6091080B7091D4
:10594000090B80910A0B90910B0B0E94141500E03B
:105950009C0145EB5DE06E2D8D2D0E94CF24BFCFC5
:105960008091CB051092CB058823E1F20E947CBF89
:105970004DE258E168E07BE085EB9DE00E94FFC0CE
:105980008091D005882371F2BDCFC23009F07FC06D
:105990008091D1058230E1F080915501882309F48E
:1059A0009ECFDD24D3948091D105823009F0D12C93
:1059B00060910C0B70910D0B80910E0B90910F0B61
:1059C0000E94141500E09C014AEA5DE06F2DC4CFEF
:1059D0008091CB051092CB058823F1F20E947CBF09
:1059E0004BE258E16CE07BE08AEA9DE00E94FFC058
:1059F0008091D005882381F285CF8091D1058330B5
:105A0000E1F080915501882309F469CFDD24D39416
:105A10008091D105833009F0D12C6091100B7091E9
:105A2000110B8091120B9091130B0E94141500E042
:105A30009C014FE95DE0612F8FCF8091CB051092E3
:105A4000CB058823F1F20E947CBF49E258E160E176
:105A50007BE08FE99DE00E94FFC08091D005882304
:105A600081F250CF8091CB051092CB058823C9F0ED
:105A70000E947CBF47E258E164E17BE084E99DE05D
:105A80000E94FFC08091D005882359F03BCFC330DE
:105A900009F4B3CFC43009F022CF8091D10584300E
:105AA00009F380915501882309F419CFDD24D3949B
:105AB0008091D105843009F0D12C6091140B709144
:105AC000150B8091160B9091170B0E94141500E096
:105AD0009C0144E95DE06D2F3FCF2F923F924F92A2
:105AE0005F926F927F928F929F92AF92BF92CF926E
:105AF000DF92EF92FF920F931F93CF93DF930E9459
:105B000088BFC091CE0535E0432E4C0E43E0342EC5
:105B100056EB652E5EE5752ED1E0DC1B2C2E219414
:105B200082E0582E5C1AC11141C08091D1058823B2
:105B3000F1F080915501882359F081E09091D105D1
:105B4000911180E024E040EC5DE0622D0E94CFBE28
:105B500080910D04882309F4C5C0C23009F45CC0EB
:105B600083E0CF5FC411DFCF8093CF050CC080915D
:105B7000CB051092CB058823E1F20E94921C809104
:105B8000D0058823B1F2DF91CF911F910F91FF9043
:105B9000EF90DF90CF90BF90AF909F908F907F90CD
:105BA0006F905F904F903F902F900895C13081F695
:105BB0008091D1058130C9F080915501882341F24F
:105BC00081E09091D105913009F080E090910D0431
:105BD00027E03DE0911102C023E03DE001E04AE012
:105BE0005DE06D2F0E94CF24B3CF80910D04909182
:105BF000CB051092CB059923F9F28C2780930D04E5
:105C0000309255016114710411F00E94B65E8091CA
:105C1000D005882389F2B7CF8091D1058230F1F089
:105C200080915501882309F49BCF11E08091D10523
:105C3000823009F010E06091090470910A048091AB
:105C40000B0490910C040E94D39600E09C0149EF54
:105C50005CE0652D812F0E94CF2482CF8091CB05FF
:105C60001092CB058823E1F20E947CBF20E030E057
:105C70004AE754E46091090470910A0480910B048E
:105C800090910C040E94EDE220E030E0A9010E9416
:105C90007EE920E030E84BEB54E40E947DE90E946D
:105CA0007AEA1F9286EB882E8EE5982E99ECA92E23
:105CB00094E2B92E6B0116EDE12E16E0F12E00E014
:105CC00010E02CED35E040E050E069E074E089EF51
:105CD0009CE00E94051C0F908091D005882309F458
:105CE0009FCF51CF82E03DCFE5E4F5E183AF64AFD4
:105CF000CA010C94C5220F931F93CF9310923A03BD
:105D0000109239032FE320933F0310923E03109229
:105D10003D039C01F90190812F5F3F4F9032D1F3F9
:105D20009E34C9F4818190ED980F9A3020F08D3225
:105D300011F08B3281F432969F012F5F3F4F8081AB
:105D400080538A3008F468C09F012F5F3F4F8081E5
:105D5000803209F463C0F093EA05E093E9058F010E
:105D60000F5F1F4FC0816AE270E0C8010E94C7EB5D
:105D7000009731F0FC01319780818032E1F311828C
:105D8000CD3429F0C43519F0C73409F041C0F80109
:105D900080810F5F1F4F8032D1F380538A30C0F56E
:105DA000C0933F0330E020E06AE0AF014F5F5F4FF8
:105DB000629FC001639F900D11249C012053310903
:105DC0008081280F311D87FD3A95FA01808180532B
:105DD0008A3058F330933E0320933D03CA01FC01FF
:105DE000019640814032D9F3F0933C03E0933B03AA
:105DF000CD3401F52E31310539F090F427313105DC
:105E000019F02C313105B1F4F0933A03E0933903E2
:105E1000CF911F910F910895F9018ECFF90194CF81
:105E20002537310538F02737310570F3203A83E004
:105E3000380751F350E040E0CF01019660816623BE
:105E400009F45AC0613291F4CD3481F42032310525
:105E500069F490933A038093390363E270E00E94FF
:105E6000C7EB0097A9F2FC011082D2CFFC01DF0141
:105E70008D91803271F090ED980F9A3008F18E324A
:105E800051F4918190539A30D8F041155105E1F4C5
:105E900014C0FD01ECCF8D3211F08B3259F4918199
:105EA00060ED690F6A3060F09E3221F49281905368
:105EB0009A3030F04115510519F4AF0141505109A4
:105EC00081548A3108F4B8CFDF01FD018D91882318
:105ED00009F4B2CF90ED980F9A30B8F393ED980F84
:105EE000923098F38B3289F3CF0101966081603252
:105EF00009F0A2CFFC01F8CF50933A034093390345
:105F000087CF0E94FE1A97FD0CC00E94FE1A6F3FB9
:105F100071058105910509F034F40E94FE1A862F5F
:105F2000089580E008958FEF089580912C0390915B
:105F30002D03892B41F00E94812F91E0811101C036
:105F400090E0892F089591E0FCCF0E94BD1A88232C
:105F500041F081E020912C0330912D03232B09F493
:105F600080E00895CF93DF93EB010E94A52F882353
:105F700019F00E94FE1AEB01CE01DF91CF91089536
:105F8000CF93DF93C82FD62F0E94A52F882321F00F
:105F9000DF91CF910C94952F8C2F0E94BD1A811107
:105FA00001C08D2FDF91CF9108951092720410924D
:105FB00073041092740410927504EEE0F4E084E629
:105FC000DF011D928A95E9F70895909108049817CA
:105FD000B1F00E94A47980910804882341F08CE3F9
:105FE0009BE00E94DD79109208040C94598881E0AE
:105FF000809308048CE39BE00E94C579F6CF089556
:106000009091080481E089270C94E52FEF92FF928C
:106010000F931F93CF93DF930EE014E0C5E0780158
:10602000D5E0F70161917191819191917F0120E01B
:1060300030E0A9010E9487E281110EC0D15089F79A
:10604000C1500C5E1F4FC111EACFDF91CF911F915C
:106050000F91FF90EF90089581E0F7CFEFE6F0E029
:1060600080818260808308954F925F926F927F92C9
:106070008F929F92AF92BF92CF92DF92EF92FF9258
:106080000F931F93CF93DF9300D000D0CDB7DEB72F
:106090000E945AC34B015C01809119018F3F09F4A2
:1060A00041C00E945AC3C0907203D0907303E09025
:1060B0007403F09075036C197D098E099F0997FD93
:1060C00031C080911D1590911E158F5F8F708917BB
:1060D00049F1E091190180E090E0A8E4B3E4E430F4
:1060E00050F424E0E29FF0011124E459FE4F808136
:1060F0009181A281B38189839A83AB83BC83C12CB4
:10610000D12C76018E010F5F1F4F28E43BE044E461
:106110005BE060E47BE08CE39BE00E949FBB8FEF41
:10612000809319010E94FE1E8091840382FF33C078
:1061300080918103811131C091E09093810380911E
:10614000890389278093CB051092890383E080938C
:106150005501109284030E945AC36C507E4F8F4F9A
:106160009F4F60938503709386038093870390937A
:10617000880368E873E182E090E00E94A69616E04A
:10618000115059F00E944A9662E070E080E090E081
:106190000E94BFC2F5CF1092810380917D03909140
:1061A0007E03A0917F03B0918003A5019401281B79
:1061B000390B4A0B5B0BDA01C901B7FF05C08091AF
:1061C000DB03882309F4C8C1D501C4018C599F4F52
:1061D000AF4FBF4F80937D0390937E03A0937F03C7
:1061E000B093800360918203062E000C770B77FF3B
:1061F00003C07195619571099091820380917C0330
:10620000981365C0633008F062C0109282038091D9
:10621000820380937C03653008F06BC08091CB05CE
:106220008111E9C0809143159091441581559343A4
:1062300041F480911A01882309F4EFC081508093C2
:106240001A010E94CB7BC0902B06D0902C06E090C8
:106250002D06F0902E0681110E942E30D701C60126
:106260003AE0B695A795979587953A95D1F7009717
:1062700041E0A407B10520F08FEF9FEFA0E0B0E070
:1062800096958795209155012111D9C03091DB0356
:10629000311190C1809143159091441581559343DC
:1062A00009F46FC18091CD0581116BC18091780394
:1062B00090917903A0917A03B0917B03881A990A8F
:1062C000AA0ABB0AB7FC6BC10E94791C68C18DEF9A
:1062D000860F823008F09BCF8091820391E087FD8A
:1062E0009FEF892F880F880F890F8093820365E0C5
:1062F0008ECF8091DB0521E030E040E050E0882344
:1063000009F456C0C090D705D090D805E090D905C3
:10631000F090DA05C114D104E104F104E9F170E070
:1063200090E080E00E948CE220E030E040EA50E41F
:106330000E9401EA2B013C01C501B4016C197D09E1
:106340008E099F090E948CE29B01AC01C301B2013E
:106350000E9401EA20E030E04AE754E40E94EDE2C6
:106360006B017C0120E030E042E053E40E9401EB4D
:1063700024E630E040E050E087FF12C020E030E04B
:1063800040EA52E4C701B6010E9401EB2AE030E086
:1063900040E050E087FF04C021E030E040E050E002
:1063A0008092D7059092D805A092D905B092DA05CF
:1063B000A09182030A2E000CBB0B0E9475E925E018
:1063C00030E040E050E00E944DE98091D30590918B
:1063D000D405A091D505B091D605820F931FA41FB7
:1063E000B51F8093D3059093D405A093D505B093A2
:1063F000D60510928203D501C4018856954CAF4F43
:10640000BF4F8093780390937903A0937A03B0935E
:106410007B0381E08093550105CF8CE080931A01C6
:106420008091760390917703009729F001979093DC
:1064300077038093760381E08093550102CF009724
:1064400041F040917603509177034817590708F0BF
:1064500021CF8091DB0381111DC0223038F0243020
:1064600008F44CC0243011F410925501809182152B
:10647000811105C081E0809382150E94A3C48091A0
:106480004B1590914C150E947CC481E08093D205FD
:106490008093DB0383E00E943B1881E080936915C1
:1064A000E0914315F091441509951092D205809121
:1064B000DB03811127C01092CB0580914315909189
:1064C00044158155934309F0EDCE0E945AC3DC0177
:1064D000CB0188199909AA09BB09C0907603D0900D
:1064E0007703F12CE12CC816D906EA06FB0608F062
:1064F000D1CE9093770380937603CCCE81E08093C6
:106500005501B4CF89E495E10E94E8C791E081117B
:1065100001C090E09093DB03882369F280914315DA
:106520009091441581559343B9F40E945AC3DC01FC
:10653000CB0188199909AA09BB09C0907603D090AC
:106540007703F12CE12CC816D906EA06FB0620F4E5
:1065500090937703809376030F900F900F900F9096
:10656000DF91CF911F910F91FF90EF90DF90CF902F
:10657000BF90AF909F908F907F906F905F904F9063
:10658000089548E9840E4AE3941EA11CB11C809230
:10659000780390927903A0927A03B0927B03809162
:1065A000DB038111D9CF809155018130A9F610927A
:1065B0005501D2CF009709F46DCF43CF8091E40508
:1065C0009091E505892B79F48091E4059091E5059A
:1065D000892B49F42091E4053091E50581E0232BD6
:1065E00019F480E0089581E00895CF92DF92EF9250
:1065F000FF926B017C0183E3C816D104E104F1042E
:1066000070F082E3C81AD108E108F10862E370E093
:1066100080E090E00E94BFC20E945B88ECCFC7017F
:10662000B6010E94BFC2FF90EF90DF90CF900C9414
:106630005B885E9A80919B058E7F80939B055E9A16
:1066400080919B058D7F80939B05159A80919B057A
:106650008B7F80939B055E9A08959091C51693FB5E
:10666000882780F993FF06C081E09091BA149111B8
:1066700001C080E008950E941DBD0E942D33882333
:1066800051F08091C51682FD06C085EF9CE0909385
:10669000A9058093A8058EEE9CE00E94E6B70C94B5
:1066A00091924F925F926F927F928F929F92AF9250
:1066B000BF92CF92DF92EF92FF920F931F93CF93EF
:1066C000DF9300D000D01F92CDB7DEB71092DB056C
:1066D0008091CB051092CB058823E9F020E040E0C3
:1066E00070E060E086EA9CE90F900F900F900F90A9
:1066F0000F90DF91CF911F910F91FF90EF90DF905E
:10670000CF90BF90AF909F908F907F906F905F9051
:106710004F900C944A1B20911F0130912001409111
:10672000D3055091D405CA01820F931F2436310539
:1067300009F015C44730510544F006978A30910599
:106740000CF01CC48AE090E023C406964A3F5F4FD9
:10675000ACF38091D205882309F4C0C12091F905DA
:106760003091FA054091FB055091FC0560913C0B7E
:1067700070913D0B80913E0B90913F0B0E947EE902
:106780004B015C012091FD053091FE054091FF0514
:10679000509100066091400B7091410B8091420B2B
:1067A0009091430B0E947EE969837A838B839C835B
:1067B0002091010630910206409103065091040693
:1067C0006091440B7091450B8091460B9091470B63
:1067D0000E947EE92B013C0120E030E040E251E4E0
:1067E0000E94EDE220E030E048EC52E40E94EDE24D
:1067F0006B017C0120E030E0A901C301B2010E94DD
:1068000087E220E030E040EA50EC87FD04C020E061
:1068100030E040EA50E4C701B6010E947EE920E082
:1068200030E040E251E40E9401EA0E9473EA2B0149
:106830003C0180E277FE09C07094609450944094CB
:10684000411C511C611C711C8DE28093DC0360E2D1
:10685000F0E14F16F7E25F06610471048CF0C301AA
:10686000B20120E137E240E050E00E944DE9CA0168
:10687000B9012AE030E040E050E00E944DE9605D5F
:106880006093DD0360E228EE421623E052066104C5
:1068900071048CF0C301B20128EE33E040E050E017
:1068A0000E944DE9CA01B9012AE030E040E050E021
:1068B0000E944DE9605D6093DE03C301B20124E6EE
:1068C00030E040E050E00E944DE96AE0C62ED12C55
:1068D000E12CF12CCA01B901A70196010E944DE9F2
:1068E000605D6093DF03C301B201A70196010E94BE
:1068F0004DE96D83CA01B901A70196010E944DE9D6
:10690000CD80CC2009F454C38EE28093E003605D17
:106910006093E1032C2D205D2093E2036CED73E086
:106920008AE693E00E94D2EB20E030E0A901C501A5
:10693000B4010E9487E220E030E040E05FEB87FD99
:1069400004C020E030E040E05FE3C501B4010E94F4
:106950007EE90E9473EACB010E94E993BC0185E6BF
:1069600093E00E94D2EB20E030E0A90169817A81B6
:106970008B819C810E9487E220E030E040E05FEB69
:1069800087FD04C020E030E040E05FE369817A8168
:106990008B819C810E947EE90E9473EACB010E9458
:1069A000E993BC0180E693E00E94D2EB4091D103D1
:1069B0004F774983411127C00E942D33882319F155
:1069C0008091BD169091BE16A091BF16B091C016D1
:1069D0000097A105B105B9F0BC01CD016D597F4FFC
:1069E0008F4F9F4F24E630E040E050E00E94CFE818
:1069F0006091C1167091C2168091C3169091C41611
:106A00000E94CFE829830E944492B62E872E982EAA
:106A1000A92E6D8380911801C9808C15C1F0C09298
:106A2000180128E4C29EB001112490E080E00E9489
:106A30008CE22AE037ED43E25CE30E94EDE20E9443
:106A40007AEA60935F03C110C5C210925A03809125
:106A50001701CD80C81609F441C0B09217016B2D03
:106A6000782D892D9A2D20E13EE040E050E00E94F3
:106A7000CFE869012CE3422E512C612C712C6B2D37
:106A8000782D892D9A2DA30192010E94CFE8CA0189
:106A9000B901A30192010E94CFE824E6C216D104F5
:106AA00008F0BFC27F936F93DF92CF9281E29CE0A8
:106AB0009F938F938AE493E09F938F930E941EE2AB
:106AC0000FB6F894DEBF0FBECDBF85E0982F990FAB
:106AD000990F891B880F8058809349030E945AC3DD
:106AE00000914503109146032091470330914803DC
:106AF0006B017C01C01AD10AE20AF30A97018601F0
:106B000037FD11C0209144032095209344036A541B
:106B10007C4F8F4F9F4F6093450370934603809344
:106B2000470390934803D0904403D98281E00E94A8
:106B30003B1880917D15843158F480917F15883001
:106B400038F026EA3CE04CE068E080E50E941BC596
:106B500080917D158431A0F480917F15823080F082
:106B6000E980EE2031F080912F0620E73CE0811192
:106B700002C02AE33CE042E162E088E60E941BC5D5
:106B800080917D158C3108F0D0C0E090A414F09075
:106B9000A514883028F58091A6149091A7140E941E
:106BA0006894FC01808193E0803229F4818192E035
:106BB000803209F491E043E050E0491B51094E0F47
:106BC0005F1F892F880F880F981B892F67E0815FCF
:106BD0000E94742E69E070E080E090E00E94322113
:106BE00080917D158C3130F580917F15843110F1C5
:106BF000C7010E946894FC01808193E0803229F4EF
:106C0000818192E0803209F491E043E050E0491B39
:106C100051094E0F5F1F892F880F880F981B892FEE
:106C20006CE1815F0E94742E69E070E080E090E08A
:106C30000E943221E090B005F090B10580917D1561
:106C4000883028F58091B2059091B3050E94689430
:106C5000FC01808193E0803229F4818192E08032CE
:106C600009F491E043E050E0491B51094E0F5F1FCA
:106C7000892F880F880F981B892F67E0865A0E94FA
:106C8000742E69E070E080E090E00E9432218091F3
:106C90007D158C3130F580917F15843110F1C7015D
:106CA0000E946894FC01808193E0803229F4818104
:106CB00092E0803209F491E043E050E0491B510931
:106CC0004E0F5F1F892F880F880F981B892F6CE14B
:106CD000865A0E94742E69E070E080E090E00E9485
:106CE000322180917D158C3100F580917F158431A2
:106CF000E0F080912F068823C1F024E6829FC00136
:106D0000112481589F4F6FEF70E00E9439E9CB0149
:106D10000E946894AC016CE187E60E94742E65E2E3
:106D200070E080E090E00E9432210E942D338823A1
:106D300069F180917D15843348F580917F158A3201
:106D400028F107E028E04AE26AE289E495E10E943E
:106D500024C605E022E04CE262E389E495E10E946A
:106D600024C66AE08AE20E94DDC560914B157091ED
:106D70004C1582E3809365158BE28093661525E6BA
:106D800035E142E389E495E10E9478C480917D1564
:106D9000853340F480917F15813320F06AE486E3E7
:106DA0000E94DDC580917D15843368F480917F1544
:106DB000823348F002E020915F0342E367E389E415
:106DC00095E10E9424C680917D158033D8F480918E
:106DD0007F158832B8F080915A03882361F04AE524
:106DE00053E060E387E30E94742E65E270E080E088
:106DF00090E00E9432214AE453E060E3809149032D
:106E00000E94742E80917D15873208F055C08091C4
:106E10007F158F3108F450C083E08093801546E2DF
:106E20004093811568E570E080E090E00E94322197
:106E30008BE08093801566E260938115C980CC2039
:106E400009F404C185E693E00E94C52288E280939C
:106E50008015F6E2F093811569E570E080E090E03E
:106E60000E94322180E38093801596E2C92EC09261
:106E70008115D980DD2009F40AC180E693E00E94E3
:106E8000C5228DE480938015F6E2F09381156AE5C2
:106E900070E080E090E00E94322185E580938015CB
:106EA00086E2C82EC0928115D980DD2009F412C176
:106EB0008AE693E00E94C52280917D15833338F5E0
:106EC00080917F158B3218F183E00E943B1883E09C
:106ED0008093801583E38093811566E070E080E005
:106EE00090E00E94322181E00E943B1880911F01B6
:106EF000909120010E946894AC0163E38CE00E94B1
:106F0000742E65E270E080E090E00E943221809172
:106F10007D15813408F007C180917F15863308F410
:106F200002C1109280158EE38093811583E692E171
:106F30000E94A516898360E870E083E692E10E94D2
:106F40006722F981F53108F0EEC060E270E080E080
:106F500090E00E94322129812F5F2983F2CF2436CD
:106F600031054CF48536910504F58A30910534F4E9
:106F70008AE090E009C084369105BCF0883EE3E0E9
:106F80009E0714F087EE93E02817390709F4E1CB48
:106F90009093200180931F011092D3051092D40585
:106FA0001092D5051092D605D4CB84E690E0F0CFB0
:106FB000662351F08EE28093E003605D6093E1030D
:106FC00080E28093E203AACC80E28093E103809385
:106FD000E003F6CF498180E2443628F0842F64E64E
:106FE0000E940BE9805D8093E003698190E26A3042
:106FF00040F02AE0862F622F0E940BE90E940BE9E5
:10700000905D9093E10389816AE00E940BE9905DB5
:107010009093E20360EE73E08AE593E00E94D2EB86
:1070200016CD7F936F93DF92CF9287E19CE09F9381
:107030008F938AE493E09F938F930E941EE20FB692
:10704000F894DEBF0FBECDBF86E040CD87E00E9442
:10705000518780FF13C005E613E0F80161918F01AD
:10706000662309F4F3CE6F320CF06FE3062E000CAA
:10707000770B880B990B0E943221EFCF80919B05F3
:1070800080FDE0CE85E39CE00E946322DFCE87E0B6
:107090000E945187869580FF13C000E613E0F80137
:1070A00061918F01662309F4ECCE6F320CF06FE32F
:1070B000062E000C770B880B990B0E943221EFCF24
:1070C00080919B05869580FDD8CE85E39CE00E944B
:1070D0006322D7CE87E00E9451878695869580FFF0
:1070E00017C08AE693E09A838983E981FA816191E6
:1070F000FA83E983662309F4DFCE6F320CF06FE385
:10710000062E000C770B880B990B0E943221EDCFD5
:1071100080919B058695869580FDCACE8DE29CE088
:107120000E946322C9CE0F900F900F900F900F9086
:10713000DF91CF911F910F91FF90EF90DF90CF9053
:10714000BF90AF909F908F907F906F905F904F9087
:1071500008950E942D33882339F08091C51682FB53
:10716000882780F991E08927089581E0089590911A
:10717000C00095FFFCCF8093C6000895CF93DF93A6
:10718000EC018991882319F00E94B738FACF8DE07D
:107190000E94B7388AE0DF91CF910C94B738CF9333
:1071A000DF93EC01FE0184912196882319F00E945F
:1071B000B738F8CFDF91CF910895E091360C81E692
:1071C000E89FF0011124E856F34F8081811107C038
:1071D00089E496E20E94CF388AE00C94B73808958B
:1071E0000E94B73889E394E00C94CF38AF92BF92F5
:1071F000CF92DF92EF92FF920F931F93CF93DF9383
:1072000084E294E00E94CF3860917204709173041C
:10721000809174049091750445E00E94937281E11D
:1072200094E00E94CF38C0E0D9E0D15021F080E254
:107230000E94B738FACF8C2F0E94EDC9CF5FC530BE
:1072400099F78AE00E94B7380EE014E0C0E080E2CF
:107250000E94B7388C2F0E94EDC95801D5E080E21A
:107260000E94B738F501C080D180E280F380A70189
:107270009601C701B6010E947FEB81112CC020E06E
:1072800030E0A901C701B6010E9401EB87FD03C0F0
:107290008BE20E94B73845E0C701B6010E949372A5
:1072A000D15084E1A80EB11CD111D9CF8AE00E943F
:1072B000B738CF5F0C5F1F4FC53049F68AE0DF91CA
:1072C000CF911F910F91FF90EF90DF90CF90BF90E3
:1072D000AF900C94B738F12C80E20E94B738F39449
:1072E0008DE3F8E0FF12F9CFDBCFCF92DF92EF9280
:1072F000FF926A017B010E94CF3842E0C701B601CC
:10730000FF90EF90DF90CF900C949372CF93DF9328
:10731000EB010E94CF38CE01DF91CF910C9496B94A
:107320008AE094E00C94CF3884E094E00C94CF3859
:10733000CF9384E50E94A52FC0E08823D9F00E9456
:10734000812FC82F1816B4F40E9494398DE40E943E
:10735000B73880913D0390913E030E94F4C96C2F91
:10736000CC0F770B8EE395E00E9486398AE00E946D
:10737000B738CFEF8C2FCF910895EC018B01F42E0D
:107380000E94E4730E94903984EE93E00E94CF380B
:107390000115110511F40DEC16E2209711F4CBED57
:1073A000D3E00E94C0201F930F93DF93CF938BEC09
:1073B00093E09F938F93D1E0DF930E946A1E0E9417
:1073C000791CC0914A15C695C6958DB79EB707968C
:1073D0000FB6F8949EBF0FBE8DBF809182158111AC
:1073E00004C0D09382150E94A3C480914B15909144
:1073F0004C150E947CC4DC2FDD0F1D2F1C0F83E079
:107400000E943B1843E652E16C2F80E00E94742EEC
:1074100010928015D09381158CEB93E00E9463222B
:1074200010928015109381158FEA93E00E946322D9
:1074300089E495E10E94E8C78111E1CF82ED93E0F4
:107440000E94E6B789EE93E030E6019729F0232FFA
:107450002A950000E9F7F9CFF89489EE93E038EE29
:10746000019729F0232F2A950000E9F7F9CF0E9410
:10747000E473FF2021F00E941933A895FECF5E9A95
:10748000FCCF80914C0B90914D0B2FEF3FEF981755
:1074900051F0E92FF0E0E45BF44F228130E09F5F90
:1074A0009F7790934D0BC90108951F920F920FB6CD
:1074B0000F9211240F900FBE0F901F9018951F92DE
:1074C0000F920FB60F9211240BB60F922F933F938A
:1074D0004F935F938F939F93EF93FF938091C60099
:1074E00040914D0B90914C0B31E0390F3F7720913B
:1074F00019032C3008F072C0E22FF0E0EE57F54C83
:107500000C946CE98E3AB53AC43ACF3AD63AEE3A90
:10751000DA3AEE3ADE3AE23AEE3AE63A803229F0E8
:10752000E8F48A3011F08D30F1F4431731F0E92F8F
:10753000F0E0E45BF44F8283932F90934C0BFF9128
:10754000EF919F918F915F914F913F912F910F906C
:107550000BBE0F900FBE0F901F9018958D3481F0C9
:1075600021E08E3471F02BE00CC08A3338F4803384
:10757000E0F68032D1F28D32B1F7D7CF8D3499F762
:1075800022E020931903D1CF813329F0843329F0ED
:10759000803249F7CACF23E0F4CF28E0F2CF24E0CD
:1075A000803379F326E0813361F3DDCF25E0883342
:1075B000D1F6E7CF27E08233B1F6E3CF29E081337C
:1075C00091F6DFCF2AE0803371F6DBCF8A3019F0F5
:1075D0008D3009F0AACF10921903A7CF8A3019F085
:1075E0008D3009F0A2CF509183155523A1F3273098
:1075F00049F02A3059F0253071F710925401109259
:107600008903E9CF21E020937804E5CF21E020939E
:107610007704E1CF8EBD0DB407FEFDCF08958FEF47
:107620008EBD0DB407FEFDCF8EB508959091640018
:107630009B7F90936400982F906A96959CBD80FDE7
:1076400003C091E0863009F490E09DBD0895CF928B
:10765000DF92EF92FF92CF936B017C01C42F4A30EF
:1076600069F4F7FE0BC0F094E094D094C094C11C70
:10767000D11CE11CF11C8DE20E94B7384C2FC701D0
:10768000B601CF91FF90EF90DF90CF900C9486C918
:10769000CF92DF92EF92FF926A017B010E94CF3876
:1076A0004AE0C701B601FF90EF90DF90CF900C94B5
:1076B000273B2F923F924F925F926F927F928F92D1
:1076C0009F92AF92BF92CF92DF92EF92FF920F9371
:1076D0001F93CF93DF93CDB7DEB7EB970FB6F89438
:1076E000DEBF0FBECDBF85E40E94A52F882321F009
:1076F0000E940E1B811183C283E50E94A52F88235F
:1077000009F45EC00E940E1B9A83898383E40E9461
:10771000A52FA5E07A2E882319F00E940E1B782E43
:1077200060E085E50E94C02F8FAB60E08AE59BE0BA
:107730000E94831E49815A81BA01550F880B990B0B
:107740000E948EE2162F7D838E83292E0E945AC3BB
:107750006B877C878D879E87609152017091530162
:107760006F507109072E000C880B990B0E948EE256
:107770009B01AC01612F7D818E81922D0E9401EBD6
:1077800018161CF58BE09BE00E94CF38EB960FB6E5
:10779000F894DEBF0FBECDBFDF91CF911F910F9147
:1077A000FF90EF90DF90CF90BF90AF909F908F9021
:1077B0007F906F905F904F903F902F900C941DBDE5
:1077C00024EB30E03A832983A1CF8B859C85AD855E
:1077D000BE85805B9C43AF4FBF4F8BAB9CABADABCB
:1077E000BEAB87EF9AE00E94CF380E94E4738FE728
:1077F0008093A81481E0809354018B849C84AD8491
:10780000BE848AA69BA6ACA6BDA61C8E1D8E1E8E0F
:107810001F8E18A219A21AA21BA219821A821B82F9
:107820001C822FE730E040E050E02F87388B498BF7
:107830005A8B1F8230E43D8B4CE14E8B56E45F8BBC
:10784000188E198E1A8E1B8EFFE7CF2ED12CE12CAD
:10785000F12C1EA61FA618AA19AA1AAA1DA21EA2BA
:107860001FA218A68CA31C8A1B8A312C00E01AAE1A
:107870001BAEA72D770CBB0BB9AFA8AF80915401FD
:10788000882309F48BC00E945AC32B013C01B0919C
:107890007904B9A7BB2309F46BC00E949774609167
:1078A000A4147091A514072E000C880B990B0E944C
:1078B0008EE2362E072F8AAF9BAF288D398D4A8DE9
:1078C0005B8D0E9401EB181634F4388E098F2AADB7
:1078D0002A8F3BAD3B8F2F813D894E895F89632D78
:1078E000702F8AAD9BAD0E9487E287FF06C03F8262
:1078F0000D8B4AAD4E8B5BAD5F8B8CA1232D302F52
:107900004AAD5BAD612F7D81882309F494C18E81DE
:10791000922D0E9487E287FF2BC0B301A201481974
:1079200059096A097B09DB01CA0188589341A109F9
:10793000B109B7FD1DC08F859889A989BA898C19AD
:107940009D09AE09BF09B595A79597958795809331
:10795000A8144DA35EA36FA378A7188F9D81998F5C
:10796000AE81AA8F2B8E4B865C866D867E861CA28E
:1079700020E030E040EF51E4612F7D818E81922D37
:107980000E947EE9232D302F4AAD5BAD0E9487E235
:1079900087FF22C084E89AE00E94CF3810925401F9
:1079A0000E94E473F3CE4BEEC42ED12CE12CF12CCB
:1079B00095C184E190E0A0E0B0E08F87988BA98B1F
:1079C000BA8B34E1C32ED12CE12CF12C95C1CF869A
:1079D000D88AE98AFA8A90C1D301C2012AA53BA5B7
:1079E0004CA55DA5821B930BA40BB50BB7FD4CC03A
:1079F00080E00E9437738AE00E94B738D301C20149
:107A00008053984FAF4FBF4F8AA79BA7ACA7BDA786
:107A10009EA5911167C02FA538A949A95AA9632D20
:107A2000702F8AAD9BAD0E9401EB18160CF046C07A
:107A300020E030E040E050E4632D702F8AAD9BAD34
:107A40000E947EE96FA778AB89AB9AABA301920144
:107A5000205B3C434F4F5F4F2BAB3CAB4DAB5EAB22
:107A600020E030E040EC50E4612F7D818E81922D4A
:107A70000E947DE9232D302F4AAD5BAD0E9487E245
:107A8000881F8827881F8EA78B859C85AD85BE851E
:107A900088169906AA06BB0610F4D501C401481A37
:107AA000590A6A0A7B0A31E843163FE4530632E179
:107AB0006306710480F186E69AE06ECFD301C201BD
:107AC0002BA93CA94DA95EA9821B930BA40BB50B56
:107AD00049E252E268E372E2B7FDD6CF80E00E944D
:107AE000AF74D2CF20E030E040EF51E4612F7D81D0
:107AF0008E81922D0E947DE99B01AC01632D702F38
:107B00008AAD9BAD0E9487E287FFBECF45ED52E272
:107B100065EE72E2E3CF48AD59AD8B899C89481779
:107B200059070CF069C003970CF466C089E09AE02D
:107B30000E94CF388CEE99E00E94CF3849815A815B
:107B40006B817C8185E09AE00E9475398AE00E9411
:107B5000B7388CEE99E00E94CF3848A159A16AA1AC
:107B60007BA181E09AE00E9475398AE00E94B738D3
:107B70008CEE99E00E94CF384C8D5D8D6E8D7F8D9F
:107B80008DEF99E00E9475398AE00E94B7389FA96D
:107B9000992309F4FBCD29813A814B815C812093A3
:107BA000A9143093AA144093AB145093AC142CEA4C
:107BB00035EC47E25EE368A179A18AA19BA10E940E
:107BC000EDE26093AD147093AE148093AF14909374
:107BD000B0142CEA35EC47E25EE36C8D7D8D8E8D22
:107BE0009F8D0E9401EA6093B1147093B214809348
:107BF000B3149093B414CACD0E9434303FCE86E3C0
:107C00009BE0EB960FB6F894DEBF0FBECDBFDF91C1
:107C1000CF911F910F91FF90EF90DF90CF90BF9089
:107C2000AF909F908F907F906F905F904F903F901C
:107C30002F900C94CF388E81922D0E9401EB181654
:107C40000CF096CED301C2012B853C854D855E8517
:107C5000821B930BA40BB50BAC01BD0148585341DB
:107C60006109710977FD84CE4B895C89452B09F444
:107C7000FEC08DA09EA0AFA0B8A4880E991EAA1E1B
:107C8000BB1E2DA13EA14FA158A5281B390B4A0BA5
:107C90005B0BC701B6010E94BFE8A50194010E94D9
:107CA0004DE9CF84D888E988FA88C20ED31EE41E35
:107CB000F51E54E1C516D104E104F1040CF479CEAB
:107CC0008CEEC816D104E104F1040CF06CCE90E8FF
:107CD000C916D104E104F1040CF479CECF86D88A18
:107CE000E98AFA8A2EEF30E040E050E02C193D0995
:107CF0004E095F0969017A014F85588969897A8936
:107D00008FEE9AE00E94483BB701A6018AEE9AE006
:107D10000E94483B4F815D896E897F8983EE9AE09E
:107D20000E947539488D598D6A8D7B8D8CED9AE056
:107D30000E947539AB89BC8913970CF498C0C701B0
:107D4000B6010E948EE220E030E040E850E40E945C
:107D5000EDE269837A838B839C832F813D894E89F1
:107D60005F89688D798D8A8D9B8D0E947DE92BEDD1
:107D70003FE049E450E40E94EDE220E030E040E0E2
:107D80005FE30E94EDE29B01AC0169817A818B8106
:107D90009C810E9401EA6F83788789879A87C50151
:107DA000B4010E948EE22FE632E143E85AE30E94DA
:107DB000EDE24B015C012AE939E949E15FE36F81BA
:107DC000788589859A850E94EDE269837A838B8321
:107DD0009C839B01AC010E947EE9A50194010E9455
:107DE00001EA68A379A38AA39BA329813A814B81E5
:107DF0005C81C501B4010E94EDE220E030E040E08A
:107E00005EE30E94EDE26C8F7D8F8E8F9F8F4F819E
:107E1000588569857A8586ED9AE00E947539B501A5
:107E2000A40180ED9AE00E9475398AE00E94B7387B
:107E300081EC9AE00E94CF3849815A816B817C8124
:107E40008BEB9AE00E94753948A159A16AA17BA1E8
:107E500085EB9AE00E9475394C8D5D8D6E8D7F8D1E
:107E60008FEA9AE00E9475398AE00E94B7388F85C0
:107E70009889A989BA898C0D9D1DAE1DBF1DB59528
:107E8000A795979587958093A8142B893C892F5F98
:107E90003F4F3C8B2B8B1F833D813D8B4E814E8B07
:107EA0002F8A5301420159A55CA362CDCF93DF9382
:107EB000EB010E94CF38CE01DF91CF910C9410CE10
:107EC0004F925F926F927F928F929F92AF92BF92EA
:107ED000CF92DF92EF92FF920F931F93CF93DF9396
:107EE00000D01F92CDB7DEB78091350C803108F0FD
:107EF000C7C131E6E32E8091350C803108F0F8C01F
:107F000080914C0B90914D0B891B8F7709F4F0C039
:107F10000E94413A97FF0BC00E94903989E793E095
:107F20000E94CF3880914C0B80934D0BE4CF8A3068
:107F300019F08D3009F0D3C01092340C8091D20B1F
:107F40009091D30BFC01E253F44F1682892B19F464
:107F50000E945B88D0CF1092D30B1092D20B04ED0D
:107F60001BE0F8018191803209F446C08E3409F09B
:107F7000A1C064E773E0C8010E9404E26C01892B90
:107F800041F06EE470E0C80104960E94C7EB0097D0
:107F900009F4C8014AE050E070E060E001960E94F8
:107FA0007BDF4B015C018091CE0B9091CF0BA091B8
:107FB000D00BB091D10B0196A11DB11D8816990669
:107FC000AA06BB0629F060E081E493E0CD2851F1D8
:107FD0006AE270E0C8010E94F6EB9C01009729F16B
:107FE000982F901BF12C992349F09150F801E90F3B
:107FF000F11D8081F826F7CF8F01B3CF4AE050E022
:1080000070E060E0C90101960E947BDF4F2C512C8B
:10801000712C612C641575058605970551F060E09B
:1080200082E293E00E9416BB66CF60E088EF92E0A8
:10803000F9CF8092CE0B9092CF0BA092D00BB09242
:10804000D10B8091AB058130E1F067E470E0C801AD
:108050000E94C7EB0097A9F04AE050E070E060E0B2
:1080600001960E947BDF623071058105910548F41D
:1080700087E592E00E94CF3860E08DE492E00E94B4
:10808000831E8091D40B8B3309F435CF8091350C4E
:10809000803108F030CF8091370C8E9DC0011124C3
:1080A00064ED7BE0885C934F0E94D2EB80E00E94FD
:1080B000E2BA21CF8091C51680FFC3CF66E776E292
:1080C000C8010E9404E2009731F0FC0183818053D3
:1080D0008A3008F0B6CF60E08EEC92E0A3CF22EDBC
:1080E0003BE044ED5BE064E37CE00E94B31603CF29
:1080F0008091C51682FFC4C01A82198281E6F82ECB
:1081000090E1B92E29E6A22E8091350C803108F03D
:10811000B7C00E94EB168111B3C041E050E0BE0130
:108120006D5F7F4F87EB94E10E9493CF0B8110E04E
:10813000019711F00FEF1FEF8091BF149091C014C1
:10814000A091C114B091C2148093C1169093C2162D
:10815000A093C316B093C4160E94EB160F3F1007EE
:1081600049F4811107C00E94903981E993E00E948F
:10817000CF38CACF4091370C242F30E00A3061F05D
:108180000D3051F0882309F46DC089819A810097E0
:1081900019F001969A8389831092260389819A8126
:1081A000F29EF001F39EF00D1124EB5CF34FDF0122
:1081B000A80FB91F13961C92892BB9F50E945B88F2
:1081C0000E94EB16882309F49FCF0E94A47987EBC5
:1081D00094E10E947F6C8091BC168823F1F181505C
:1081E0008093BC168A9DC001112462E08C5D9A4F79
:1081F0000E94CAD1E091BC1624E0E29FF001112454
:10820000E05EFA4F40815181628173814093C116D3
:108210005093C2166093C3167093C41687EB94E113
:108220000E946BCE0E9409CA6FCF1A821982838185
:108230008D3479F48481823361F48581853349F406
:10824000868180538A3028F08091C5168B7F809379
:10825000C51681E00E94E2BAB3CF0E94FAC9B0927B
:10826000AB0552CF4F9DA0011124485C534F9E0196
:108270002F5F3F4F66E273E0802F0E94B31644CF1A
:108280000E945AC34B015C018091340390913503E5
:10829000A0913603B09137030097A105B10551F1C4
:1082A0004091E0055091E1056091E2057091E30590
:1082B000840F951FA61FB71FA5019401281B390B1A
:1082C0004A0B5B0BDA01C901B7FD14C00E9490395B
:1082D0006091E9057091EA0580E192E00E94563FC5
:1082E0008AE00E94B73840E070E060E090E080E013
:1082F0000E94BD3980910B0190910C01A0910D015C
:10830000B0910E01892B8A2B8B2B79F090911D1542
:1083100080911E15981709F4FCC08092E005909298
:10832000E105A092E205B092E3050E945AC36B01F9
:108330007C0180918903811108C020911D159091C5
:108340001E1581E0291301C080E02091A414309112
:10835000A51491E089272A3A31050CF480E091E0D8
:1083600040912203509123036091240370912503CF
:10837000452B462B472B09F490E0981789F088236A
:1083800009F401C1D701C60180569444A24FBF4FE2
:108390008093220390932303A0932403B093250397
:1083A0004090480B5090490B60904A0B70904B0BDB
:1083B00020911E0330911F0340912003509121030F
:1083C000C301B2010E9487E2882319F18091220340
:1083D00090912303A0912403B091250340921E03A2
:1083E00050921F036092200370922103892B8A2BE5
:1083F0008B2B09F449C0D701C60180569444A24F83
:10840000BF4F8093220390932303A0932403B09340
:1084100025038091220390912303A0912403B0911E
:1084200025030097A105B10579F1C81AD90AEA0A0E
:10843000FB0AF7FC29C0109222031092230310922A
:108440002403109225038BEF91E00E94CF3860E067
:1084500087EE91E00E94831E8091A6149091A7144C
:108460001816190624F490E080E00E9494A28091EE
:10847000B2059091B3051816190634F41092B3059D
:108480001092B2050E94EF6180912703909128031A
:10849000A0912903B0912A03A5019401281B390B4F
:1084A0004A0B5B0BDA01C901B7FD8FC090911D1516
:1084B00080911E15F0902F06981749F0E0911E1537
:1084C0003BE4E39FF0011124E757F94FF0800E944D
:1084D0005AC3FF2009F4D1C000911A0310911B0365
:1084E00020911C0330911D03011511052105310553
:1084F00009F04DC06C597F4F8F4F9F4F60931A0307
:1085000070931B0380931C0390931D03FF24FA9424
:1085100044C00E945AC30091E0051091E1052091EA
:10852000E2053091E305C0900B01D0900C01E09082
:108530000D01F0900E010C0D1D1D2E1D3F1D601B29
:10854000710B820B930B97FF03C010922B03EDCEA0
:1085500080912B038111E9CE81E080932B035E9AF9
:1085600080919B058E7F80939B055E9A80919B05F1
:108570008D7F80939B05159A80919B058B7F8093BF
:108580009B055E9AD2CE80E090E0DC0101CF601BBB
:10859000710B820B930B97FDB9CF0F2D10E084E088
:1085A0000E94A0BAF11072C060E084E00E94D9C1BC
:1085B00044E6840E911CA11CB11C8092270390926A
:1085C0002803A0922903B0922A030E945B8880911D
:1085D000AB058823F1F1109108011130B1F18091C0
:1085E000C51680628093C51681E08093080164EF10
:1085F00071E080E090E00E94F5320E942BD48091DF
:10860000C51683FFA5C0123028F460E080EA93E02D
:108610000E94831E01E083E0809355010E945AC3AB
:108620006C597F4F8F4F9F4F60937D0370937E03F4
:1086300080937F0390938003002339F0123029F454
:1086400081E08093BB160E9486D40E944A960E94C5
:1086500034300F900F900F90DF91CF911F910F91B9
:10866000FF90EF90DF90CF90BF90AF909F908F9052
:108670007F906F905F904F90089510921A03109220
:108680001B0310921C0310921D0387CF0F3F11058F
:1086900011F461E08ACFE1EBF6E2E491E150EA30D7
:1086A00008F051C0F0E0E95AFC4B0C946CE96143CE
:1086B00066436B437543A343A3437F4387438F4381
:1086C000994384B5806884BDF7BC72CF84B580625D
:1086D00084BDF8BC6DCF809180008068809380005D
:1086E000109389000093880063CF8091800080629E
:1086F0008093800010938B0000938A0059CF809163
:10870000B00080688093B000F092B30051CF8091A8
:10871000B00080628093B000F092B40049CF8091A5
:1087200090008068809390001093990000939800C7
:108730003FCF8091900080628093900010939B00C7
:1087400000939A0035CF003811050CF0A2CF2CCF42
:1087500000E0112309F479CF5ECF2F923F924F9220
:108760005F926F927F928F929F92AF92BF92CF92C1
:10877000DF92EF92FF920F931F93CF93DF93CDB7CA
:10878000DEB764970FB6F894DEBF0FBECDBF809101
:10879000F30A83FDB0C10E949839898787FDABC178
:1087A00089E40E94A52F882309F497C10E94812F94
:1087B00090E01816190614F481E090E026E0289F56
:1087C000F001299FF00D1124EB54FA4F8081918123
:1087D0001B8A0E9494A22091A6143091A714809124
:1087E000A4149091A514821793078CF48CED99E052
:1087F0009F938F9387EE99E09F938F931F920E9490
:108800006A1E0F900F900F900F900F9005C02B894C
:1088100081ED99E0222361F381E0809354011C8271
:108820001D821E821F821A861B861C861D861F863D
:108830002CE3288B3CE1398B46E44A8B212C312CEC
:1088400050E85A838FEB8B83198291E09E87812CAD
:10885000912C540101C01E860091A6141091A714FA
:10886000B801012E000C880B990B0E948EE2D62EC7
:10887000E72EF82E988791014A815B810E9487E25A
:10888000882391F08091A4149091A5143B89311113
:10889000E7C041E04983081719070CF019822D2C15
:1088A0003E2CFA8258855B830E945AC36B017C017F
:1088B000DC01CB012A853B854C855D85821B930BB2
:1088C000A40BB50BB7FD2FC0D701C60188519C4F33
:1088D000AF4FBF4F8A879B87AC87BD8789850E9432
:1088E00037738DEC99E00E94CF3881149104A10474
:1088F000B10409F4E0C0C501B4016053784F8F4F53
:108900009F4F6C197D098E099F0928EE33E040E0E6
:1089100050E00E94CFE8CA01B9014AE00E94273B1B
:108920008AE00E94B7380E94603F0E945AC3609359
:10893000E0057093E1058093E2059093E305609173
:10894000A4147091A514072E000C880B990B0E949B
:108950008EE26887072F182F9C8B262F372F482FE2
:10896000592FB1018A819B810E947DE92B013C0135
:1089700020E030E0A9010E9401EB87FF04C077FAF4
:10898000709477F8709481149104A104B10409F0F3
:1089900096C020E030E040E85FE3C301B2010E94EE
:1089A00087E287FF10C09E85812C912C540199236A
:1089B00031F08AE9882E82E0982EA12CB12C8C0C03
:1089C0009D1CAE1CBF1CA981AA2399F12C813D815D
:1089D0004E815F81211531054105510541F0D701D7
:1089E000C601821B930BA40BB50BB7FD22C02885D3
:1089F000302F412F5C896F85788989899A890E94F7
:108A00007DE920E030E040EC5FE30E9487E287FDF3
:108A10002AC0D701C601805A9541AF4FBF4F8C8302
:108A20009D83AE83BF8398859F87088B198BAC8904
:108A3000AA8B809154018823B1F081149104A10480
:108A4000B10409F408CFB0EDCB1AB7E0DB0AE108B6
:108A5000F108C818D908EA08FB08F7FCFCCE03C0E7
:108A6000081719070CF580915401882309F443C0B5
:108A70001092540164960FB6F894DEBF0FBECDBFBE
:108A8000DF91CF911F910F91FF90EF90DF90CF90EA
:108A9000BF90AF909F908F907F906F905F904F901E
:108AA0003F902F900C941DBD2D2C3E2CFA82888572
:108AB0008B831982F9CE8FE30E94B73831CF20E043
:108AC00030E040E450E4C301B2010E9401EB18160B
:108AD0000CF079CF4601570176CF83E50E94A52F90
:108AE0008B8B811105C082E50E94A52F882319F088
:108AF0000E940E1B6ECE64960FB6F894DEBF0FBEBA
:108B0000CDBFDF91CF911F910F91FF90EF90DF903C
:108B1000CF90BF90AF909F908F907F906F905F901D
:108B20004F903F902F9008952F923F924F925F92D7
:108B30006F927F928F929F92AF92BF92CF92DF926D
:108B4000EF92FF920F931F93CF93DF93CDB7DEB7D2
:108B5000CB54D1090FB6F894DEBF0FBECDBF2C9613
:108B60008FAF2C9780913F038D3409F488C48435EE
:108B700011F40C944A5B873491F480913D039091F9
:108B80003E038C31910509F43BC208F071C084307A
:108B9000910509F4B5C130F4029708F4FEC00E94B3
:108BA00043BD7EC18531910509F47AC14B97B9F770
:108BB0000E9451BD811174C119821A821B821C82CC
:108BC0001D821E821F82188680E090E0A0E2B1E440
:108BD00089879A87AB87BC8770E060E080E50E9458
:108BE000B22F40E050E068E472E44CA35DA36EA3B2
:108BF0007FA340E050E060EA70E448A359A36AA371
:108C00007BA3813009F4B5C1823009F4D1C120E0E1
:108C100030E040E050E46091440B7091450B80914E
:108C2000460B9091470B0E947EE97B018C0120E06E
:108C300030E048E453E40E9401EB181624F4E12CE0
:108C4000F12C08E413E4A984BA84CB84DC84970172
:108C5000A801B501C6010E9401EB181614F47501B4
:108C60008601C701D8018C8F9D8FAE8FBF8FC2C187
:108C70008A35910509F4E6C360F58D31910509F453
:108C80003DC38A9709F08BCF8091AB05813009F005
:108C900007C189E40E94A52F082F10E0882319F04E
:108CA0000E940E1B182F8AE40E94A52FF82E8823FD
:108CB00011F40C94AB5B0E940E1B002309F421C33A
:108CC000153010F40C949D5B8AE595E00E94CF3836
:108CD000E7C08B35910509F4B8C38C35910509F0CF
:108CE0005ECF90E6C92E91E0D92EF12CE12C00E068
:108CF00010E0D6018D916D010E94A52F382E88239A
:108D0000E1F10E94121B4B015C01133059F0F70195
:108D1000E750FA4F20813181428153810E947DE9E1
:108D20004B015C01F701E45CF44F20813181428109
:108D30005381C501B4010E947DE92B013C012DEB5B
:108D400037E346E855EB0E9401EB87FD0AC02DEBA7
:108D500037E346E855E3C301B2010E9487E21816E3
:108D600064F4133009F075C38092480B9092490B5C
:108D7000A0924A0BB0924B0B032D1F5FB4E0EB0E99
:108D8000F11C143009F0B5CF002321F088E49BE0FA
:108D90000E9489850E941A9083C08091AB05813022
:108DA00009F07EC064EFC62E63E0D62E7CE3E72E8A
:108DB0007BE0F72EE9EFAE2EE5E0BE2E10E088E571
:108DC000810F0E94A52F882309F47EC00E94121BE8
:108DD0002B013C01812F0E940717882309F46AC0E8
:108DE000D7012D913D914D915C91C301B2010E943B
:108DF0007EE9D6016D937D938D939C9313971F5FAE
:108E0000F4E0CF0ED11C24E0E20EF11C34E0A30EFE
:108E1000B11C1330A1F685E40E94A52F882309F424
:108E20005EC00E94121B6B017C0183E00E94071749
:108E3000882371F02091480B3091490B40914A0BE7
:108E400050914B0BC701B6010E947EE96B017C017A
:108E5000C0920004D0920104E0920204F092030454
:108E600086E40E94A52F8823C9F00E94121B20E0EF
:108E700030E0A9010E9401EB181684F40E94121B35
:108E800020E030E040E752E40E9401EA60932101D3
:108E90007093220180932301909324010E94648B9C
:108EA0002C96FFAD2C97F1110C9426530E94DD38BF
:108EB0000C942653F5012081318142815381C301F5
:108EC000B2010E947DE995CFF70180819181A28155
:108ED000B381F60180839183A283B38390CF809185
:108EE000480B9091490BA0914A0BB0914B0B80938A
:108EF000000490930104A0930204B0930304B0CF44
:108F000080E50E94A52FC12CD12C7601882321F069
:108F10000E94EE1A6B017C0183E50E94A52F882335
:108F200061F00E94121B20E030E04AE754E40E9406
:108F3000EDE20E947AEA6B017C010E94A4798091A3
:108F40006312811105C060E081E595E00E94831EF7
:108F50000E945AC3C60ED71EE81EF91E0E945AC3AD
:108F60006C197D098E099F0997FF9ACF0E94603F77
:108F7000F5CFBE01605E7F4FCE0109960E943A8810
:108F8000E090440BF090450B0091460B1091470B7D
:108F90002D813E814F81588569817A818B819C81A9
:108FA000DE0194966D010E9482870E941A9078CF0C
:108FB00029853A854B855C856091440B7091450B02
:108FC0008091460B9091470B0E947EE96B017C01DA
:108FD00020E030E048E453E40E9487E287FD06C0C9
:108FE000C12CD12C58E4E52E53E4F52ECC8EDD8E29
:108FF000EE8EFF8EBE01605E7F4FCE014C96BECFDF
:1090000087E00E945187882309F464C10E94A479F3
:1090100010922801609108048CE40E94C02F982EC1
:1090200080E00E94E52F0E945AC36093E005709390
:10903000E1058093E2059093E305809121019091F1
:109040002201A0912301B0912401809330039093D9
:109050003103A0933203B093330380911F019091A9
:10906000200190932F0380932E0384E690E0909349
:10907000200180931F0181E0809399050E94179140
:109080008AE50E94BD1AA82E88E50E94BD1A182FF5
:1090900089E50E94BD1AB82E181308C0B12EA1127E
:1090A00005C011E0BB24B394AA24A39482E50E94D6
:1090B000A52F882309F416C10E94121B3B01882E9C
:1090C000C92E20E030E0A9010E9487E2882309F43C
:1090D00044C0111103C0BB2009F4D0C0D090440B90
:1090E000E090450BF090460B0091470B9301482D03
:1090F0005C2D6D2D7E2D8F2D902F0E9401EB18166B
:1091000024F0D62CE72CF82C0C2D80E090E0A0E881
:10911000B0E48C8F9D8FAE8FBF8F20E030E048E4AD
:1091200053E46D2D7E2D8F2D902F0E9487E287FDB9
:1091300005C0D12CE12C28E4F22E03E48D2D9E2DC8
:10914000AF2DB02F89839A83AB83BC83BE01645E4D
:109150007F4FCE0101960E943A88112309F489C0FD
:10916000BB2009F483C010923C0B10923D0B10926F
:109170003E0B10923F0B1092400B1092410B10923D
:10918000420B1092430B0E945988E7EFF6E1C5901D
:10919000D590E590F490EBEFF6E145905590659011
:1091A0007490A7019601C301B2010E9487E287FF74
:1091B000A0C0A7019601C301B2010E9401EA9B0170
:1091C000AC010E94EDE220E030E040E85FE30E9465
:1091D0007EE90E943FEB20E030E048E452E40E9448
:1091E000EDE269837A838B839C832091440B3091D9
:1091F000450B4091460B5091470B28A739A74AA72A
:109200005BA720E030E040EC5FE3C301B2010E94C5
:10921000EDE22B013C0177FA709477F8709420E02E
:1092200030E040EC5FE3C701B6010E94EDE29058E8
:10923000AE014F5F5F4F6A01E8A4F9A40AA51BA520
:10924000A30192010E9482870E94369210923C0BE9
:1092500010923D0B10923E0B10923F0B1092400B60
:109260001092410B1092420B1092430B80E00E942F
:10927000C98EBB2019F081E00E94C98EAA2019F086
:1092800082E00E94C98E0E9459888091980580933F
:109290009905892D0E94E52F80913003909131032B
:1092A000A0913203B0913303809321019093220166
:1092B000A0932301B093240180912E0390912F035A
:1092C0009093200180931F0183E0809355010E94B9
:1092D0001A90E6CD60E08FE40E94C02F882309F445
:1092E00095CEDECD612C712C30E8832E40E4C42E67
:1092F000F0CEA3019201C701B6015FCF0E942C5CA2
:10930000CFCD853008F0E0CC90E1ECE3FBE0A4EFBA
:10931000B3E001900D929A95E1F70023A1F054E09B
:109320001502F0011124E856FA4E40815181628104
:1093300073814093F4035093F5036093F6037093A5
:10934000F703FF2091F094E08902F0011124EC571B
:10935000FA4E80819181A281B3818093F80390932A
:10936000F903A093FA03B093FB0386E40E94A52FB0
:10937000811151C0C12CD12C760180902101909097
:109380002201A0902301B090240120E030E0A90147
:10939000C701B6010E9487E2882341F0C0922101F3
:1093A000D0922201E0922301F092240100911F014A
:1093B0001091200184E690E09093200180931F019A
:1093C000C0905A01D0905B01E0905C01F0905D018B
:1093D00080E090E0A0E8BFE380935A0190935B01A6
:1093E000A0935C01B0935D010E94648B8092210187
:1093F00090922201A0922301B092240110932001A7
:1094000000931F01C0925A01D0925B01E0925C016F
:10941000F0925D0145CD0E94121B6B017C0120E0A2
:1094200030E0A9010E9401EB18160CF0A3CF20E058
:1094300030E040E752E4C701B6010E9401EA6B0147
:109440007C019BCF109238032BCD8FE080933803A3
:1094500027CDF701E851FC4F5F01A3019201608124
:109460007181828193810E947EE9D5016D937D9304
:109470008D939C931397812F0E9431877ECC80918E
:109480003D0390913E038337910511F40C94C05431
:1094900008F09FC18B34910511F40C94CD5208F063
:1094A000A7C08831910509F481C608F06CC08231EB
:1094B000910511F40C94375400F58230910508F4AD
:1094C000F2C5419709F06BCB83E092E00E94991AB4
:1094D000882309F43DC688E50E94BD1A81115E9873
:1094E00089E50E94BD1A81115E988AE50E94BD1A25
:1094F000882309F4D5CC1598D3CC8531910509F48E
:109500003AC658F5449709F04ACB8091C51683FFB7
:109510002AC68EE995E00E94CF388091C51683FF58
:1095200017C08DEE94E10E94D76D8BE1EDEEF4E172
:10953000DE01119601900D928A95E1F770E060E0EE
:10954000CE0101960E94F4D2CE0101960E94AA6F2C
:109550008FE895E00E94CF38A3CC8631910509F4BD
:109560000EC6479709F01BCB8091390390913A03BF
:10957000FC012191222309F412C62032D1F7DF0128
:1095800011971C92F6CF8D31910509F4B1C6A0F464
:109590008A31910509F43AC608F418C68B31910551
:1095A00009F453C64C9709F0FACA80913903909197
:1095B0003A030E9482D174CC8F31910509F443C7DC
:1095C00008F49DC68032910509F4FAC689349105E4
:1095D00009F0E5CA80E50E94BD1A882309F460CC31
:1095E0000E94812F853608F084E68093D10358CC01
:1095F0008836910509F4EEC708F0C2C0823591059E
:1096000011F40C942754F0F48D34910509F4DEC75D
:1096100008F4C7C78135910509F0C1CA0E94E473F7
:109620000E94B4790E94B59210922F0668EE73E002
:1096300080E090E00E94F53260E087EA96E00E94C8
:10964000831E2ECC8435910511F40C94375410F4FC
:109650000C942F548535910511F40C948B548C3552
:10966000910509F09CCA0E94983987FD19CC83E0C6
:1096700092E00E94991A882311F40C94BB54E0E6FE
:10968000CE2EE1E0DE2EF4EFEF2EFAE0FF2E10E01A
:10969000F60181916F010E94A52F882309F466C00D
:1096A000133011F00C94B0540E94121B4B015C015A
:1096B00020E030E040EA51E40E9487E287FF4EC09C
:1096C000A50194016091140B7091150B8091160BFC
:1096D0009091170B0E9401EA2B013C01AC019B0108
:1096E00060911306709114068091150690911606EC
:1096F0000E94EDE2609313067093140680931506A2
:1097000090931606A30192016091240B7091250B92
:109710008091260B9091270B0E94EDE26093240B21
:109720007093250B8093260B9093270B6091230653
:109730007091240680912506909126060E948CE265
:10974000A30192010E94EDE20E947AEA609323064F
:109750007093240680932506909326068092140B1E
:109760009092150BA092160BB092170B1F5FB4E0EE
:10977000EB0EF11C143009F08BCF0E94807990CB56
:109780008D36910509F44FC778F48A36910509F4AE
:1097900077C708F44CC78B36910509F4A5C78C36FA
:1097A000910509F47DCBFBC98F36910509F4B9C742
:1097B00008F4A4C78037910509F472CB823791056C
:1097C00009F0EDC90E947DBC8FE195E10E94BE7554
:1097D00067CB8232E1E09E0711F40C94425708F007
:1097E00063C3883C910511F40C94945508F0ADC105
:1097F0008837910511F40C940955E8F486379105E2
:1098000011F40C94CA5410F00C9405558537910549
:1098100009F0C5C98091390390913A03009711F47A
:109820000C94C654FC012081222311F40C94C654DC
:109830000E94BFBA35CB8C38910509F4B3C758F4F0
:109840008937910509F0ABC91092990510929805D6
:109850000E94179125CB8139910511F40C94125572
:109860008E3B910509F09BC98091F30A83FD18CBCB
:1098700089E40E94A52F882311F40C948C5B0E942C
:10988000812F90E01816190614F481E090E026E08C
:10989000289FF001299FF00D1124EB54FA4F82818B
:1098A00093811CAA8C38910514F08CE890E0909379
:1098B000B3058093B2050E94EF612091B20530910B
:1098C000B3058091B0059091B105821793070CF014
:1098D00094C788E996E060E00E94831E81E080934F
:1098E00054011DAA1EAA1FAA18AE1BAE1CAE1DAEA7
:1098F0001EAE21961FAE21979CE322969FAF229722
:10990000ACE12496AFAF2497B6E42896BFAF289772
:10991000312C212CE0E8ECA7FFEBF8AB18A621E0F6
:109920002FAF812C912C54010091B2051091B305F9
:10993000B801012E000C880B990B0E948EE26B017E
:109940007C01232D322D4CA558A90E9487E2882343
:1099500089F08091B0059091B1053CA9311150C7B3
:1099600041E048A7081719070CF018A63C2C2D2C2D
:10997000ECA6F8AA0E945AC36B017C01DC01CB0162
:109980002BAD3CAD4DAD5EAD821B930BA40BB50B67
:10999000B7FD2FC0D701C60188519C4FAF4FBF4FB5
:1099A0008BAF9CAFADAFBEAF80E00E94377385E850
:1099B00096E00E94CF3881149104A104B10409F407
:1099C00034C7C501B40168577C4E8F4F9F4F6C1947
:1099D0007D098E099F0928EE33E040E050E00E94A7
:1099E000CFE8CA01B9014AE00E94273B8AE00E9401
:1099F000B7380E94603F0E945AC36093E00570939D
:109A0000E1058093E2059093E3056091B0057091C4
:109A1000B105072E000C880B990B0E948EE269AFEE
:109A20007AAF8C019B01AC01632D722D8CA598A996
:109A30000E947DE92B013C0120E030E0A9010E9459
:109A400001EB87FF04C077FA709477F87094811463
:109A50009104A104B10409F0ECC620E030E040E834
:109A60005FE3C301B2010E9487E287FF10C09FAD90
:109A7000A2E88A2EA6E09A2EA12CB12C911103C047
:109A8000812C912C54018C0C9D1CAE1CBF1CA8A5D4
:109A9000AA2309F442C02DA93EA94FA958AD21150A
:109AA00031054105510541F0D701C601821B930BD9
:109AB000A40BB50BB7FD31C029AD3AADA801219675
:109AC0006FAD219722967FAD229724968FAD249774
:109AD00028969FAD28970E947DE920E030E040E87D
:109AE0005FE30E9487E287FD8EC6D701C601805AD8
:109AF0009541AF4FBF4F8DAB9EABAFABB8AF99ADFC
:109B000021969FAF2197AAAD2296AFAF22972496B8
:109B10000FAF249728961FAF289780915401882370
:109B200009F471C681149104A104B10461F0B8E88C
:109B3000CB1AB3E1DB0AE108F108C818D908EA0832
:109B4000FB08F7FE60C61FAEEFCE8E3C910511F408
:109B50000C945F5608F0B9C08B3C910511F40C943D
:109B6000C55558F5893C910509F019C80E949839E6
:109B700087FD96C900E611E064EFE62E6AE0F62E56
:109B800074E6C72E71E0D72ED8018D918D010E9409
:109B9000BD1A882359F00E94121B0E947AEAF7012D
:109BA00060837183828393830E943279F4E0EF0EA5
:109BB000F11CC016D10641F773C98C3C910511F414
:109BC0000C94E8558D3C910511F00C94CF4580E044
:109BD00092E00E94991A882309F462C982E40E94E3
:109BE000BD1A882351F00E94EE1A6093040B709303
:109BF000050B8093060B9093070B83E50E94BD1A1B
:109C0000882351F00E94121B6093340B7093350B24
:109C10008093360B9093370B84E50E94BD1A8823FE
:109C200051F00E94121B6093380B7093390B809394
:109C30003A0B90933B0B88E50E94BD1A882351F0A4
:109C40000E94121B60930706709308068093090612
:109C500090930A0689E50E94BD1A882351F00E945C
:109C6000121B60930B0670930C0680930D06909365
:109C70000E068AE50E94BD1A8823B1F00E94121BCD
:109C800060930F067093100680931106909312064E
:109C90002DEC3CEC4CEC5DE30E9487E2181624F0BE
:109CA00082EF97E00E94CF3885E40E94BD1A882396
:109CB00009F4F6C80E94121B6093130670931406F1
:109CC0008093150690931606EBC88C3D910511F410
:109CD0000C94AD5608F0C9C0833D910511F00C9469
:109CE000CF454090F9055090FA056090FB057090C3
:109CF000FC052091290130912A0140912B015091BE
:109D00002C01C301B2010E947EE968A779A78AA746
:109D10009BA78090FD059090FE05A090FF05B09058
:109D2000000620912D0130912E0140912F0150917C
:109D30003001C501B4010E947EE96CA77DA78EA702
:109D40009FA7C0900106D0900206E0900306F09015
:109D5000040620913101309132014091330150913C
:109D60003401C701B6010E947EE968AB79AB8AABCA
:109D70009BAB2091350130913601409137015091D4
:109D80003801C301B2010E947EE92B013C01209100
:109D9000390130913A0140913B0150913C01C5019C
:109DA000B4010E947EE94B015C0120913D0130919C
:109DB0003E0140913F0150914001C701B6010E9410
:109DC0007EE96B017C010E9494398DE398E00E944A
:109DD000CF3883E50E94BD1A882321F00E94952F79
:109DE0008093270180912701882309F4B3C786EC6B
:109DF00098E00E94CF3885E398E00E94CF3848A5CC
:109E000059A56AA57BA58BEF97E10E9475394CA5F2
:109E10005DA56EA57FA58CE897E20E94753948A9DB
:109E200059A96AA97BA989E897E20E94753983E359
:109E300098E00E94CF388BE298E00E94CF38B301BF
:109E4000A2018BEF97E10E947539B501A4018CE85E
:109E500097E20E947539B701A60189E897E20E944E
:109E600075398AE00E94B7381BC88D3D910509F409
:109E7000B2C78A3F910511F00C94CF4583E40E944C
:109E8000BD1A882321F00E940E1B0E948F20609132
:109E900041017091420184E898E00E9486398AE08D
:109EA0000E94B7380C9450478C3A21E0920711F485
:109EB0000C945E5A08F089C08F3241E0940711F487
:109EC0000C94635820F58D32A1E09A0711F40C949C
:109ED0009C5710F00C941D588C32914011F00C944A
:109EE000CF4564E071E083E50E94B22F8C0168EEFB
:109EF00073E080E50E94B22F8938F3E19F0710F0EC
:109F000088E893E1B8010E94A6960C9450478A39DC
:109F1000F1E09F0711F40C94504748F480399140C8
:109F200011F00C94CF450E94A4790C945047843AC8
:109F300041E0940711F40C946758853A914011F070
:109F40000C94CF4588E50E94BD1AC82E89E40E9472
:109F5000BD1AA82E882311F40C94C5590E940E1B1B
:109F6000082F89E50E94BD1AF82E8AE40E94BD1AC6
:109F7000E82E882311F40C94F0590E940E1B182F20
:109F80008AE50E94BD1AD82EB12C811104C081E54A
:109F90000E94BD1AB82EA11001C0E12C8E2D90E0B8
:109FA000C11001C0F12C8F0D911D019731F4D1101A
:109FB0000C941B5AB1100C941B5A0E94903984E3E4
:109FC00099E00E94CF380C945047883FA1E09A074F
:109FD00011F40C94185B28F5853FE1E09E0711F41D
:109FE0000C94105B48F4843F914011F00C94CF45E1
:109FF0000E946D760C945047863F31E0930711F430
:10A000000C94145B873F914011F00C94CF4561E0B4
:10A0100083E50E94C02F91E089270E94CEA20C9474
:10A020005047803A53E0950709F4FFC180F48C3023
:10A03000924011F00C94CF458091C51682FD02C06C
:10A040000C942B5B80648093C5160C945047873E1C
:10A05000E3E09E0711F40C94335B893E934011F0CA
:10A060000C94CF458091BB1681110C94435B0E94E8
:10A0700044926D3371058105910520F087EB99E0DD
:10A080000E94BA5B83EB99E00E94BA5B84EE8093F6
:10A09000D1038FE999E00E94CF388BE999E00E94C3
:10A0A000BA5B0C94504780E50E94A52FC12CD12C9F
:10A0B0007601882321F00E94EE1A6B017C0183E572
:10A0C0000E94A52F882361F00E94121B20E030E03F
:10A0D0004AE754E40E94EDE20E947AEA6B017C01B7
:10A0E0000E94A4798091390390913A030097E1F09E
:10A0F0000E94BFBA81E080938903C114D104E104B6
:10A10000F10431F00E945AC3C60ED71EE81EF91E94
:10A11000809189038823B1F0C114D104E104F104D2
:10A1200049F40E94603FF4CF60E083E795E00E942D
:10A13000831EE0CF0E945AC36C197D098E099F09C6
:10A1400097FDEFCF109289030E941DBD0C945047DC
:10A1500060E086E895E00E94831E5E985E98159800
:10A160005E980C9450470E9494398FEA95E00E94C3
:10A17000CF380C9450470E942BD40C9450478091B8
:10A18000C51682FF02C00C9450470E94FAC9809104
:10A19000C516877F80628093C5160C94504760E097
:10A1A0000E94CAD11092D1030C9450470E942D33C3
:10A1B000882321F00E9409CA0E9491928EEE9CE0B1
:10A1C0000E94E6B70E941DBD0C9450478091C516B1
:10A1D00082FF03C08B7F8093C5168091F805813084
:10A1E00069F482E08093F8050E945AC36093E40307
:10A1F0007093E5038093E6039093E7030E941DBDEF
:10A2000089EB95E00E94E6B70C9450478091C51603
:10A2100083FD02C00C94504783E50E94A52F88233C
:10A2200011F40C9450470E94FE1AAB01BC014093FC
:10A23000C1165093C2166093C3167093C41687EB71
:10A2400094E10E946BCE0C94504783E40E94BD1AA7
:10A250008823E9F089EC95E00E94CF388091BA1408
:10A26000882381F0BE016F5F7F4F87EB94E10E94EE
:10A27000A26CCE0101960E9410CE8AE00E94B738EF
:10A280000C9450478FEB95E00E94CF38F6CF809129
:10A29000C51682FF27C0C090C116D090C216E090AC
:10A2A000C316F090C41688ED95E00E94CF384AE0BE
:10A2B000C701B6010E9486C98FE20E94B73860913B
:10A2C000BD167091BE168091BF169091C0164AE0DF
:10A2D0000E9486C98DE00E94B7388AE00E94B73894
:10A2E0000C9450478AEE95E00E94CF380C9450476A
:10A2F0008091C5168E7F8093C5160C94504780912F
:10A30000C51683FD02C00C9450470E9451CE809127
:10A31000C51683FD02C00C945047409139035091FB
:10A320003A03BE01645E7F4F80E00E949DB98C01BC
:10A33000009711F40C9450476C8D7D8D19821C820E
:10A3400022E0AC01CE0101960E94B06F811119C0CC
:10A35000F12CCE0101960E94AA6FB801FF2031F1C5
:10A3600086E196E00E94563F8AE00E94B73810923C
:10A37000C1161092C2161092C3161092C4160C94F5
:10A380005047CE0101960E94FFCE882309F361E079
:10A39000CE0101960E94886C0097D1F225EEDC0177
:10A3A0002C931C820E94A0CAF82ED3CF8EEF95E08A
:10A3B0000E94563F8BEF95E00E94CF380C94504797
:10A3C0008091C51682FD0E94A4798091C51683FDF7
:10A3D00002C00C94504760E080E50E94C02F182F07
:10A3E000682F8091390390913A030E94CAD183E586
:10A3F0000E94A52F882381F00E94FE1AAB01BC01A8
:10A400004093C1165093C2166093C3167093C4163E
:10A4100087EB94E10E946BCE0E9409CA11110C9443
:10A4200050470E9491920C945047209139033091EB
:10A430003A039091C51692609093C516C9010E9487
:10A4400082D10C9450470E9444927B018C0120E8F9
:10A4500031E541E050E00E94CFE8C9016DE671E0CE
:10A460000E9425E94B015C01C801B70120E13EE0F3
:10A4700040E050E00E94CFE8CA01B90128E130E095
:10A4800040E050E00E94CFE8762E672EC62ED72EF1
:10A490008CE3282E312C412C512CC801B701A2018C
:10A4A00091010E94CFE8F62EE72ECA01B901A20160
:10A4B00091010E94CFE8CB018E010F5F1F4F8114E5
:10A4C000910431F1EF92FF927F936F936F927F929D
:10A4D000BF92AF929F928F928CE496E09F938F935E
:10A4E0001F930F930E941EE20FB6F894DEBF0FBEBB
:10A4F000CDBFC8010E94BFBA0E949439B80180E65E
:10A5000096E00E94563F8AE00E94B7380C9450476C
:10A51000A114B10489F0EF92FF927F936F936F9231
:10A520007F92BF92AF928CE396E09F938F931F939D
:10A530000F930E941EE2D8CFCD2879F0EF92FF92C0
:10A540007F936F936F927F9280E396E09F938F93B8
:10A550001F930F930E941EE2C7CF892B69F0EF92E1
:10A56000FF927F936F9388E296E09F938F931F9360
:10A570000F930E941EE2B8CFEF92FF9284E296E022
:10A580009F938F931F930F930E941EE20F900F9043
:10A590000F900F900F900F90ACCF0E9491920C945F
:10A5A00050478091F805813011F00C94504782E0BB
:10A5B0008093F8050E945AC36093E4037093E50307
:10A5C0008093E6039093E7030C9450470E94B59262
:10A5D0000C9450478091F30A83FF02C00C945047BB
:10A5E0000E94983987FF02C00C94504789E40E946A
:10A5F000A52F882311F40C946B5B0E94812F90E0AF
:10A600001816190614F481E090E026E0289FF00166
:10A61000299FF00D1124EB54FA4F808191810E9403
:10A6200094A20C9450470E94AD430C9450470E9452
:10A630009839182F87FD0AC08DE696E00E94CF3822
:10A64000812F0E9437738AE00E94B738C55BDF4FC5
:10A650000FB6F894DEBF0FBECDBFDF91CF911F9133
:10A660000F91FF90EF90DF90CF90BF90AF909F90B1
:10A670008F907F906F905F904F903F902F900895B4
:10A6800080E50E94A6BD81110C94504781E40E9490
:10A69000BD1A60912F06062F10E0811102C00FEF46
:10A6A00010E089E40E94A52F882311F40C94765BB6
:10A6B0000E94812F90E01816190614F481E090E0B2
:10A6C00026E0289FF001299FF00D1124EB54FA4F4A
:10A6D000048115810F3F110519F010F00FEF10E004
:10A6E00000932F060C94504780E50E94A6BD81116F
:10A6F0000C94504710922F060C9450478EE40E9401
:10A70000A52F882311F40C9450470E94FE1A6093E1
:10A71000CE0B7093CF0B8093D00B9093D10B0C94F6
:10A72000504783E50E94BD1A882329F083E50E94E3
:10A73000A6BD8093F30A0E9494398EE796E00E94AA
:10A74000CF388091F30A882351F110E000E020E037
:10A750008091F30A90E0B0E0A0E0002E04C0B6952E
:10A76000A795979587950A94D2F780FF12C0FF248A
:10A77000F394F20E222319F08CE20E94B738F8010C
:10A78000EE0FFF1FEC58F94F859194910E94CF383E
:10A790002F2D0F5F1F4F05301105D1F66ECD80E7CD
:10A7A00096E072CD8091F30A83FF02C00C9450476B
:10A7B00089E40E94A52F882309F4A4C70E94812F51
:10A7C00090E01816190614F481E090E026E0289F26
:10A7D000F001299FF00D1124EB54FA4F82819381EF
:10A7E0008C38910514F08CE890E09093B305809339
:10A7F000B2050E94EF610C94504789E896E06BC85F
:10A800000817190764F480915401882311F40C94FB
:10A810005047109254010E941DBD0C9450473C2C8F
:10A820002D2CECA6F8AA18A6A5C88FE30E94B7386D
:10A83000DDC820E030E040E450E4C301B2010E94F2
:10A8400001EB18160CF023C94601570120C980916D
:10A8500038038F7D8061809338030C94504780913A
:10A8600038038F7E8062809338030C94504783E5D1
:10A870000E94A52F8823F1F00E945AC36093E0053F
:10A880007093E1058093E2059093E3050E94121B0B
:10A8900020E030E04AE754E40E94EDE20E947AEAC8
:10A8A00060930B0170930C0180930D0190930E0146
:10A8B0000C94504783E092E00E94991A882339F162
:10A8C0000E94A47988E50E94BD1A882331F05E9A1F
:10A8D00080919B058E7F80939B0589E50E94BD1A20
:10A8E000882331F05E9A80919B058D7F80939B0534
:10A8F0008AE50E94BD1A882311F40C945047159ADA
:10A9000080919B058B7F80939B050C9450470E9400
:10A91000B4790C94504783E50E94BD1A882311F442
:10A920000C9450470E945AC36093E0057093E10570
:10A930008093E2059093E3050E94121B20E030E033
:10A940004AE754E40E94EDE20E947AEA60933403FD
:10A950007093350380933603909337030C945047DC
:10A960000E94121BD70154966D937D938D939C93F7
:10A9700057970C94B64B81E00E94E2BC0C94504770
:10A9800088EB96E00E94CF380C9450470E941DBD82
:10A990000C9450470091390310913A0394E0F12C44
:10A9A00040E0915009F1D8018C91282F2B7F213460
:10A9B000A1F411962C912133B9F4813419F1853425
:10A9C00009F441E098012E5F3F4F89012F5F3F4F0F
:10A9D000D8018C918032C9F3E4CF803529F4F80195
:10A9E000818180538A3070F341110E949439FF2095
:10A9F00021F08AEB97E00E94CF38C8010E94BE3850
:10AA00000C945047FF24F394DDCF0E94FC900C94EB
:10AA1000504781E080939905809398050E94179193
:10AA20000C94504783E50E94A52F882309F45FC04A
:10AA30000E940E1B823008F05DC08C01112788E453
:10AA40000E94A52F8823C1F00E940E1B8A3A91050F
:10AA50000CF458C00E940E1B843B91400CF055C072
:10AA60000E940E1B26E0209FF001219FF00D112473
:10AA7000EB54FA4F9183808382E40E94A52F8823B0
:10AA8000B9F00E940E1B05970CF442C00E940E1BE9
:10AA90008D3891050CF03FC00E940E1B26E0209FD0
:10AAA000F001219FF00D1124EB54FA4F9383828320
:10AAB00086E40E94A52F882311F40C9450470E942D
:10AAC0000E1B97FD2BC00E940E1B8F3F910509F0B6
:10AAD00044F50E940E1B26E0209FF001219FF00DFF
:10AAE0001124EB54FA4F958384830C94504790E0E3
:10AAF00080E0A3CF0E9490398DEB97E00E94CF3881
:10AB00000C9450478AEA90E0ADCF83EB91E0AACF56
:10AB100085E090E0C3CF8CE890E0C0CF90E080E08B
:10AB2000DACF8FEF90E0D7CF0E949839182F87FFA8
:10AB300002C00C94504700910D0484E40E94A52F9C
:10AB4000F82E8823B1F00E94121B4B015C0120E01B
:10AB500030E0A9010E9487E28823A9F024E01202D4
:10AB6000F0011124E75FFB4F80829182A282B382C1
:10AB70000F2D602F83E50E94C02F80930D040E944B
:10AB8000B65E0C94504780E0F8CF0E94983987FF5A
:10AB900002C00C94504750E6E52E51E0F52E10E02F
:10ABA00000E0D7018D917D010E94BD1A882349F0F4
:10ABB0000E94121BF801EC50F54F64A375A386A305
:10ABC00097A30C5F1F4F0031110559F70C945047A4
:10ABD0008BEF91E00E94991A811129C04091280BB6
:10ABE0005091290B60912A0B70912B0B82EE97E00C
:10ABF0000E94753940912C0B50912D0B60912E0BBA
:10AC000070912F0B8FED97E00E9475394091300BBA
:10AC10005091310B6091320B7091330B8AE898E1BF
:10AC20000E9475398AE00E94B7380C94504783E53A
:10AC30000E94A52F882391F00E94121B6093280B7D
:10AC40007093290B80932A0B90932B0B6093300BFE
:10AC50007093310B8093320B9093330B80E50E94FD
:10AC6000A52F882351F00E94121B6093280B70932C
:10AC7000290B80932A0B90932B0B82E50E94A52F22
:10AC8000882351F00E94121B60932C0B70932D0BA4
:10AC900080932E0B90932F0B84E50E94A52F882381
:10ACA00011F40C9450470E94121B6093300B709368
:10ACB000310B8093320B9093330B0C9450474CE93B
:10ACC000E42E45E0F42E10E088E5810F0E94BD1AC5
:10ACD000882351F00E94121BF701608371838283E5
:10ACE0009383812F0E9431871F5FF4E0EF0EF11CE8
:10ACF000133051F788E092E00E94991A81110C9468
:10AD0000CA4640919C0550919D0560919E057091A9
:10AD10009F0584E298E00E9475394091A00550910A
:10AD2000A1056091A2057091A3058CE897E20E94AD
:10AD300075394091A4055091A5056091A6057091C3
:10AD4000A70589E897E20E9475398AE00E94B73822
:10AD50000C94504782EC98E04CC882E40E94BD1AE3
:10AD6000882341F080911F01909120019093100160
:10AD700080930F0182E50E94BD1A882341F08091E3
:10AD80000F01909110019093200180931F0183E5A2
:10AD90000E94A52F882331F00E940E1B9093200162
:10ADA00080931F01E0913B03F0913C038081882355
:10ADB00011F40C94504760911F01709120018DE4B3
:10ADC00098E00E94863985E20E94B7388AE00E94A6
:10ADD000B7380C9450470E949839082F87FF02C05B
:10ADE0000C94504783E50E94A52F002E000C110BF8
:10ADF0007801EE0CFF1C882359F10E940E1BF7010D
:10AE0000EB5DFE4F91838083000F111F000F111F18
:10AE10009801265A3E4F7901BC01990F880B990B76
:10AE20000E948EE22AE037ED43E25CE30E94EDE20D
:10AE30000C5F1B4FD8012D913D914D915C910E946B
:10AE4000EDE2F70160837183828393830C94504712
:10AE50000E94943985E40E94B73880E3800F0E94F5
:10AE6000B738F701EB5DFE4F6081718181E598E0B5
:10AE70000E94863985E20E94B7388AE00E94B7387E
:10AE80000C9450478AE50E94A52F882331F10E9437
:10AE9000121B20E030E040E050EC0E9487E287FD8A
:10AEA0003AC00E94121B20E030E040E050E40E94D3
:10AEB00001EB1816ACF10E94121B2091100B30917F
:10AEC000110B4091120B5091130B0E94EDE20E9466
:10AED00073EACB010E9493C305C083E50E94A52FAE
:10AEE0008111D5CF88E092E00E94991A81111DC08E
:10AEF0000E949439409172045091730460917404DB
:10AF00007091750489E598E00E9475398AE00E9485
:10AF1000B7380C94504760E070E080E090ECCDCF03
:10AF200060E070E080E090E4C8CF82E50E94BD1A46
:10AF30008111DECF0C94504785E40E94A6BD81119B
:10AF400074C080E50E94BD1A882351F00E94121B34
:10AF50006093A9147093AA148093AB149093AC14CB
:10AF600089E40E94BD1A882381F00E94121B2CEAFA
:10AF700035EC47E25EE30E94EDE26093AD1470931E
:10AF8000AE148093AF149093B01484E40E94BD1A61
:10AF9000882381F00E94121B2CEA35EC47E25EE325
:10AFA0000E9401EA6093B1147093B2148093B314B9
:10AFB0009093B4140E9494394091A9145091AA140A
:10AFC0006091AB147091AC148EE698E00E947539D4
:10AFD0002CEA35EC47E25EE36091AD147091AE145B
:10AFE0008091AF149091B0140E9401EAAB01BC01B2
:10AFF0008AE698E00E9475392CEA35EC47E25EE378
:10B000006091B1147091B2148091B3149091B41402
:10B010000E94EDE2AB01BC0186E698E00E94753922
:10B020008AE00E94B7380C9450470E94903982E71A
:10B0300098E00E94CF380C94504783E50E94BD1AD7
:10B04000182F882369F00E940E1B9C0190935F01CA
:10B0500080935E0191E0232B09F090E090934006ED
:10B0600080E50E94BD1A882361F020915E01309135
:10B070005F01232B11F00E94952F809340060C94C2
:10B08000504711110C9450470E9494398FEA98E070
:10B090000E94CF3880914006882391F087E998E09C
:10B0A0000E94CF3860915E0170915F018EE998E057
:10B0B0000E9486398AE998E00E94CF380C94504764
:10B0C00083E998E0EDCF0E94593B0C94504783E50B
:10B0D0000E94BD1A182F30900804882319F00E948E
:10B0E000952F382E20913C0B30913D0B40913E0B1B
:10B0F00050913F0B27962CAF3DAF4EAF5FAF2797D8
:10B100004090400B5090410B6090420B7090430B6D
:10B110008091440B9091450BA091460BB091470B49
:10B120002B968CAF9DAFAEAFBFAF2B97112329F0FD
:10B13000311003C080E00E94E52F86E50E94BD1A11
:10B1400021968FAF21970E940630882309F4B8C05A
:10B1500083E40E94BD1A882309F49FC00E94121B39
:10B160006B017C01AEE0B4E0B9ABA8ABB9A7A8A76E
:10B17000F5E0FCA71AAE1BAE28EC2FAF02EC1CAA20
:10B18000212C38EC3DAB42E449AF88A599A5239624
:10B190009FAF8EAF239715E02396AEADBFAD23973B
:10B1A0008D909D90AD90BD902396BFAFAEAF23978D
:10B1B0002CA9322D4DA959ADC501B4010E9487E2D9
:10B1C00087FF04C08CAA292CADAAB9AE2AAD3BAD2D
:10B1D0004FAD502FC501B4010E9401EB181624F4A5
:10B1E0008AAE9BAEAFAE0B2D1150B1F6BCA5B150DF
:10B1F000BCA7E8A5F9A57496F9A7E8A7B111C5CF32
:10B200002AAD3BAD4FAD502F6CA9722D8DA999ADD4
:10B210000E947EE920E030E040E05FE30E94EDE242
:10B22000A70196010E947EE96B017C012DEB37E3BB
:10B2300046E855EB0E9401EB87FD0AC02DEB37E392
:10B2400046E855E3C701B6010E9487E218162CF5BF
:10B2500080E00E94E52F15E0A8A8B9A805E0D50177
:10B260006D917D918D919D915D014D01B4E08B1AA1
:10B270009108A70196010E947DE9F4016083718322
:10B2800082839383015059F7115028A939A92C5E64
:10B290003F4F39AB28AB1111DFCF21964FAD21972E
:10B2A000442351F00E940630882331F086EF98E065
:10B2B0000E94CF380E94F638832D0E94E52F0DC0E2
:10B2C000311005C021963FAD21973323A9F30E9489
:10B2D00094398CE099E00E94CF38332051F080916E
:10B2E0000804811106C00E94903987ED98E00E9401
:10B2F000CF380E94943989EC98E00E94CF38809131
:10B300000804882309F43EC086EC98E00E94CF38F8
:10B310008AE00E94B73820913C0B30913D0B409160
:10B320003E0B50913F0B27966CAD7DAD8EAD9FAD22
:10B3300027970E9487E281110C94CA462091400B06
:10B340003091410B4091420B5091430BC301B2012C
:10B350000E9487E281110C94CA462091440B3091DF
:10B36000450B4091460B5091470B2B966CAD7DAD34
:10B370008EAD9FAD2B970E9487E281110C94CA4637
:10B380000C94504782EC98E0C1CFC11003C00FEF7E
:10B390000C94B14F0E94121B2091F9053091FA05CF
:10B3A0004091FB055091FC050E947DE920E030E0D2
:10B3B00040EA51E40E947DE920E030E04CE551E4B0
:10B3C0000E947EE929E032EF44E15DE30E94EDE274
:10B3D0000E9473EA062F653010F40C94B14FD7CF5A
:10B3E000F11003C01FEF0C94C04F0E94121B20915C
:10B3F000FD053091FE054091FF05509100060E9429
:10B400007DE920E030E040EA51E40E947DE920E05F
:10B4100030E04CE551E40E947EE929E032EF44E15E
:10B420005DE30E94EDE20E9473EA162F653010F48E
:10B430000C94C04FD7CF07FD02C017FF08C00E9471
:10B4400090398BE199E00E94CF380C9450470E94CC
:10B45000121BE02E000FFF08A12F110FBB0B20E0E5
:10B4600030E0A901BB2091F025E02E9DF0012F9D39
:10B47000F00D1124EA0FFB1FEE0FFF1FEE0FFF1F51
:10B48000E25FFB4F2081318142815381E5E0EE9DF7
:10B490008001EF9D100D11240A0F1B1F000F111FBB
:10B4A000000F111F025F1B4F0E947EE9D8016D93B0
:10B4B0007D938D939C9313970C9450470E9451BD9C
:10B4C00081110C94504796ECC92E96E1D92EECE3ED
:10B4D000FBE0F9A7E8A79E012F5F3F4F1901790113
:10B4E00010E000E0F6016591759185919491A8A511
:10B4F000B9A58D909D90AD90BD90B9A7A8A7A501C5
:10B5000094010E947DE92B013C01F70140825182A8
:10B510006282738220E030E040EA51EC0E9401EB4D
:10B5200087FD0AC020E030E040EA51E4C301B201E7
:10B530000E9487E2181684F4F801E15DF84DE49169
:10B540001E1654F4B7FAB094B7F8B094D7018D92A0
:10B550009D92AD92BC921397F70181909190A1902A
:10B56000B1907F0120E030E040EA51ECC501B40128
:10B570000E9401EB87FD3FC020E030E040EA51E44B
:10B58000C501B4010E9487E21816ACF10F5F1F4F8E
:10B59000F4E0CF0ED11C0330110509F0A3CF8CE9E4
:10B5A000E82E85E0F82E10E0F10181919191A191B2
:10B5B000B1911F01F70181939193A193B1937F0101
:10B5C000812F0E9431871F5F133071F70E941A90FC
:10B5D00060E084E599E00E94831E63E972E084E6FE
:10B5E00090E00E94A6966AEB72E084E690E00E94EA
:10B5F000A6960C9450470E94903982E799E00E94E9
:10B60000CF3861E084E699E00E94831E0E94791C95
:10B6100068E270E088EC90E00E94A6960C94504797
:10B620000E94C0A80C9450470E9422910C9450474D
:10B6300081E0809376040E94B4A810927604882357
:10B6400011F40C9450470E94943980E999E00E94CB
:10B65000CF380C94504783FD02C00C9450470E9491
:10B6600051CE0C94504781E08093AB0510928E121E
:10B6700060E083E50E94C02F81110C9450470E9426
:10B68000F9BA0C9450470E9486D481110C9450470B
:10B690000C94375010913D030E945AC36093E0050B
:10B6A0007093E1058093E2059093E305112311F473
:10B6B0000C9450470E94943984E50E94B738812F3A
:10B6C0000E94EDC980E20E94B7388BEB99E00E949E
:10B6D000CF380C94504783E50E94A52F882311F49E
:10B6E0000C9450470E940E1B0C940F5383E50E944C
:10B6F000A52F882311F40C946A530E94FE1A8B0123
:10B700000C946A5383E50E94A52F882311F40C94AE
:10B7100050470E940E1B64C883E50E94A52F8CAB86
:10B72000811107C082E50E94A52F882311F40C9493
:10B7300050470E940E1B0C94524CF1100C948149FE
:10B7400090E1ECE3FBE0A4EFB3E001900D929A9559
:10B75000E1F70C948F4980E001110C94604680E180
:10B76000ECE3FBE0A4EFB3E001900D928A95E1F7E2
:10B770000C94B5494F925F926F927F928F929F92F5
:10B78000AF92BF92CF92DF92EF92FF920F931F93EF
:10B79000CF93DF93CDB7DEB77C014DB65EB6609038
:10B7A000E9057090EA058DB69EB66AE070E0C701C3
:10B7B0000E94C9E16C018C010E191F09892B21F42B
:10B7C000C7010E94D4E18C01C80101962DB73EB794
:10B7D000281B390B0FB6F8943EBF0FBE2DBF8DB797
:10B7E0009EB701965C01A801B7010E94F5E1F50141
:10B7F000E00FF11F1082C5010E947B2E81E00E94A4
:10B800009445C114D10451F076019FEFE91AF90A69
:10B810000FB6F8949EBE0FBE8DBEC5CF0FB6F8947E
:10B820009EBE0FBE8DBEC3010E947B2E0FB6F89444
:10B830005EBE0FBE4DBEDF91CF911F910F91FF9065
:10B84000EF90DF90CF90BF90AF909F908F907F90C0
:10B850006F905F904F9008954F925F926F927F929A
:10B860008F929F92AF92BF92CF92DF92EF92FF9210
:10B870000F931F93CF93DF93CDB7DEB728970FB603
:10B88000F894DEBF0FBECDBF83E50E94A6BD863013
:10B8900028F087E295E00E94CF3849C0833009F450
:10B8A0006EC1E8F4813071F1823009F45AC084E14C
:10B8B00095E00E94CF380E9406308823F1F08091F5
:10B8C0000804811117C082EC98E00E94CF388AE00A
:10B8D0000E94B7380E94F6380E941A9028C084301F
:10B8E00009F493C1853019F780E00E94E52F0E948A
:10B8F000D52FF2CF86EC98E0E8CF86E095E00E9465
:10B90000CF38EACF0E94D52F10920A011092090178
:10B910008091D903811125C08EE40E94BD1A811146
:10B920001DC084EF94E09093A9058093A805289604
:10B930000FB6F894DEBF0FBECDBFDF91CF911F9140
:10B940000F91FF90EF90DF90CF90BF90AF909F90BE
:10B950008F907F906F905F904F9008958AEF94E062
:10B96000E2CF8091090190910A0197FF03C08BEC0F
:10B9700094E091CF009709F0A8C01D821E821F821B
:10B9800018868DEC9CECACE4BEE389839A83AB8390
:10B99000BC83BE016B5F7F4FCE0101960E943A8847
:10B9A0008091090190910A01893191050CF0B3C091
:10B9B00021E0209328019C012F5F3F4F30930A0123
:10B9C0002093090165E00E9417E980FF03C024E08D
:10B9D000291B922F24E09202F0011124E856FA4E1E
:10B9E00080809180A280B38094E08902F0011124CC
:10B9F000EC57FA4E40805180628073808DEC9CEC55
:10BA0000ACE4BEE38D839E83AF83B88719821A822C
:10BA10001B821C82CE0101966C01E12CF12C00EA04
:10BA200010E4A3019201C501B4010E94828719822A
:10BA30001A821B821C82B601CE0105960E943A88AA
:10BA400080923C0B90923D0BA0923E0BB0923F0B2C
:10BA50004092400B5092410B6092420B7092430B0C
:10BA60001092D9030091090110910A0189E1E82E91
:10BA7000F12C093111050CF47801B70184E694E04A
:10BA80000E94863969E170E08FE594E00E94863972
:10BA90008AE00E94B738101611060CF01DCF1F92D5
:10BAA00089E18F93FF92EF9288E494E09F938F93C4
:10BAB00086E594E09F938F931F920E946A1E0FB6B3
:10BAC000F894DEBF0FBECDBF07CF815065E00E9466
:10BAD00017E980FF03C024E0291B922F25E0920282
:10BAE000F0011124E80FF11D87FDFA95EE0FFF1FFD
:10BAF000EE0FFF1FE25FFB4F8091440B9091450BCF
:10BB0000A091460BB091470B80839183A283B383AE
:10BB10001092280145CF80E090E0A0EAB0E4809345
:10BB2000440B9093450BA093460BB093470B81E2D7
:10BB300091E00E9467870E94A4798FEF9FEF909316
:10BB40000A018093090187EB94E00E94CF3885EACF
:10BB500094E00E94BFBA63E972E084E690E00E943C
:10BB6000A6966AEB72E084E690E00E94A6968FE9C2
:10BB700094E00E94BA5B81E00E94E52F71CF89E4D6
:10BB80000E94A52F882371F00E940E1B182F85306C
:10BB900068F064E070E08CE894E00E94863989E8FF
:10BBA00094E079CE8AE40E94F038C1CE8AE40E9403
:10BBB000A52F8823B9F30E940E1B082F853048F06B
:10BBC00064E070E086E794E00E94863983E794E0C1
:10BBD00062CE8AE50E94A52F8823A9F00E94121B3D
:10BBE00025E01202F0011124E00FF11D07FDFA9586
:10BBF000EE0FFF1FEE0FFF1FE25FFB4F60837183AD
:10BC00008283938369CE8AE5CECF8AE50E94A52FF1
:10BC10008823C9F30E94121B60937204709373040B
:10BC2000809374049093750457CECF93DF93C091A3
:10BC3000360C81E6C89FE0011124C85CD34F809187
:10BC4000F30A80FF05C00E949439CE010E94BE38DD
:10BC5000CE010E947B2E80E0DF91CF910C94944521
:10BC60000F931F93CF93DF93CDB7DEB760970FB6D7
:10BC7000F894DEBF0FBECDBF8C01DC01ED91FC91CD
:10BC80000280F381E02DBE016F5F7F4F099588230D
:10BC900009F464C08981807CC9F56F81637070E0AC
:10BCA000762F6627770F770F8885B4E08B9FC001CA
:10BCB0001124682B792B89858295869586958370CA
:10BCC000682B6F5F7F4F90E080E02A852370220F02
:10BCD0003B8537FB332730F9232B3E813F70230F01
:10BCE0003327331F2750310904C0660F771F881F81
:10BCF000991F2A95D2F760960FB6F894DEBF0FBE53
:10BD0000CDBFDF91CF911F910F910895803419F528
:10BD100068856695669570E090E080E0CB017727B6
:10BD200066272A85622B098510E0102F0027012E37
:10BD3000000C220B330B602B712B822B932B6F5F2C
:10BD40007F4F8F4F9F4F4AE0660F771F881F991FC5
:10BD50004A95D1F7D0CF8BE0F801848360E070E0A2
:10BD6000CB01C9CF0895FC0182810895CF92DF9263
:10BD7000EF92FF9280910D04882309F457C0C09080
:10BD80000904D0900A04E0900B04F0900C0420E029
:10BD900030E0A901C701B6010E9487E2882309F4B7
:10BDA00045C020E030E040E05FE3C701B6010E94FB
:10BDB000EDE29B01AC010E94EDE22BED3FE049E496
:10BDC00050E40E94EDE29B01AC0160E070E080E88D
:10BDD0009FE30E9401EA6B017C01C0920404D092AF
:10BDE0000504E0920604F092070460912501709129
:10BDF0002601072E000C880B990B0E948EE22AE088
:10BE000037ED43E25CE30E94EDE2A70196010E9458
:10BE1000EDE260935A0170935B0180935C01909313
:10BE20005D01FF90EF90DF90CF900895C12CD12C51
:10BE300080E8E82E8FE3F82ED0CF2F923F924F92DA
:10BE40005F926F927F928F929F92AF92BF92CF92AA
:10BE5000DF92EF92FF920F931F93CF93DF93CDB7B3
:10BE6000DEB766970FB6F894DEBF0FBECDBFDC011C
:10BE7000CD90DD90ED90FC90139714962D913D910F
:10BE80004D915C9117972B873C874D875E8720E00B
:10BE900030E040EA51E4C701B6010E947DE929E0A3
:10BEA00032EF44E15DE30E94EDE20E9473EA643008
:10BEB0000CF428C163E0662E660F7708F301EE0FDD
:10BEC000FF1FEE0FFF1FE856FA4E80809180A28080
:10BED000B380F3013196FA83E98320E030E040EA51
:10BEE00051E46B857C858D859E850E947DE929E0E6
:10BEF00032EF44E15DE30E94EDE20E9473EA6430B8
:10BF00000CF404C163E0062F660F110BF801EE0F6D
:10BF1000FF1FEE0FFF1FE856FA4E2081318142814C
:10BF200053812B833C834D835E83A8014F5F5F4F1A
:10BF30005E8B4D8BA5E0A69DC001A79D900D1124A1
:10BF4000988B8F87FC01E00FF11FEE0FFF1FEE0FA4
:10BF5000FF1FE25FFB4F20813181428153812F839C
:10BF6000388749875A87E981FA81EE0FFF1FEE0F64
:10BF7000FF1FE856FA4EA50194016081718182810C
:10BF800093810E947DE9698B7A8B8B8B9C8BA501B9
:10BF90009401C701B6010E947DE92B013C0185E0B7
:10BFA00049815A81849F1001859F300C1124F10131
:10BFB000E00FF11FEE0FFF1FEE0FFF1FE25FFB4FC1
:10BFC0002F81388549855A8560817181828193816D
:10BFD0000E947DE929893A894B895C890E9401EA9E
:10BFE000A30192010E94EDE22F81388549855A858F
:10BFF0000E947EE96B017C01EF85F889AD89BE89DD
:10C00000EA0FFB1FEE0FFF1FEE0FFF1FE25FFB4F5C
:10C0100080809180A280B380FD01E20DF31DEE0FC0
:10C02000FF1FEE0FFF1FE25FFB4FA5019401608130
:10C030007181828193810E947DE929893A894B89A6
:10C040005C890E9401EAA30192010E94EDE2A50130
:10C0500094010E947EE9A70196010E947DE94B01AF
:10C060005C01ED89FE89EE0FFF1FEE0FFF1FE85602
:10C07000FA4E2B813C814D815E816081718182818C
:10C0800093810E947DE99B01AC01C501B4010E942E
:10C0900001EA4B015C012B813C814D815E816B8506
:10C0A0007C858D859E850E947DE99B01AC01C50143
:10C0B000B4010E94EDE2A70196010E947EE9209161
:10C0C00072043091730440917404509175040E947D
:10C0D0007EE966960FB6F894DEBF0FBECDBFDF9146
:10C0E000CF911F910F91FF90EF90DF90CF90BF9075
:10C0F000AF909F908F907F906F905F904F903F9008
:10C100002F90089567FFD7CE60E0D5CE67FFFBCEB6
:10C1100060E0F9CE8F929F92AF92BF92CF92DF9262
:10C12000EF92FF92FC01C080D180E280F38020E09A
:10C1300030E040E251E4C701B6010E94EDE220E0A8
:10C1400030E040E251E40E94EDE24B015C0120E06E
:10C1500030E0A901C701B6010E9487E220E030E08B
:10C1600040EA50E487FF04C020E030E040EA50ECB1
:10C17000C501B4010E947EE920E030E040E251E4D4
:10C180000E9401EA0E9473EA9B018BE237FF05C01F
:10C1900022273327261B370B8DE28093DD03C9014D
:10C1A00068EE73E00E9439E9CB01EAE0F0E0BF01FC
:10C1B0000E9439E9805D8093DE03C90164E670E086
:10C1C0000E9439E9CB01BF010E9439E9805D80936B
:10C1D000DF03C901BF010E9439E9282FCB01BF014C
:10C1E0000E9439E9805D8093E0038EE28093E10351
:10C1F000205D2093E2038DED93E0FF90EF90DF90C0
:10C20000CF90BF90AF909F908F90089524E6829F2B
:10C21000C001112481589F4F6FEF70E00E9439E9EF
:10C22000262F81E3643609F080E28093DF0390E2F9
:10C230002A3040F03AE0822F632F0E940BE90E94DF
:10C240000BE9905D9093E003822F6AE00E940BE976
:10C25000905D9093E10385E28093E2038FED93E09C
:10C2600008956091250170912601072E000C880B1E
:10C27000990B0E948EE22AE037ED43E25CE30E94D4
:10C28000EDE22091040430910504409106045091A0
:10C2900007040E94EDE260935A0170935B01809362
:10C2A0005C0190935D0108958091DD05811104C0CA
:10C2B0008091C70580932F0608958091BA16882330
:10C2C000C1F081508093BA16EDEEF4E1882351F06D
:10C2D0008150990B2BE1289FF001299FF00D11242B
:10C2E000E455FA4E8BE1A2EDB4E101900D928A95EE
:10C2F000E1F72091BA16211105C08091C516806220
:10C300008093C51681E090E0A0E0B0E0211103C069
:10C3100080E090E0DC018093D3059093D405A09356
:10C32000D505B093D6051092CE0581E08093D00557
:10C3300083E0809355010895CF93DF93EC01CB0107
:10C34000BA010E948EE220E030E0A9010E947EE95D
:10C350000E9473EA79836883DF91CF910895CF9328
:10C36000DF93EC01CB01BA010E948EE229EC38EC9C
:10C3700048EC5EE30E9401EA20E030E040E05FE349
:10C380000E947EE90E947AEA6883DF91CF91089546
:10C390000E948EE229EC38EC48EC5EE30E9401EA50
:10C3A00020E030E040E05FE30E947EE90E947AEA0C
:10C3B000862F0C94066180914101909142010C946A
:10C3C0008F20E091DD0586E0E802F0011124EB54B6
:10C3D000FA4F8091C70590E095838483089520915A
:10C3E000B2053091B30521153105E9F08091B00512
:10C3F0009091B105029624503109821793079CF45D
:10C4000090931705809316050E945AC3605E70448E
:10C410008D4F9F4F609318057093190580931A05EF
:10C4200090931B050895109218051092190510920B
:10C430001A0510921B050895CF93DF93EC018D81AF
:10C440000E94163B60E08B81DF91CF910C94D9C1A3
:10C45000DF92EF92FF920F931F93CF93DF938C01A4
:10C46000C62FD22FF32EE42ED52E0E941C620E94DE
:10C47000D9C38C2F80640E940A3B8D2D0E940A3BF9
:10C480008E2D0E940A3B8F2D0E940A3B8D2F0E9409
:10C490000A3B87E8C11101C085E90E940A3BCC3004
:10C4A00011F40E940F3BC0E00E940F3BF80186830D
:10C4B00087FF04C0CF3F11F0CF5FF6CFDF91CF9160
:10C4C0001F910F91FF90EF90DF90089561E0FC01C4
:10C4D00083810E94D9C18FEF0C940A3B0F931F9365
:10C4E000CF938C010E941C620E94D9C3C82F88235D
:10C4F00071F08DEF0E940A3B0E94D9C3C82FC8017A
:10C500000E9466628C2FCF911F910F91089582E156
:10C51000F8018483F4CF8F929F92AF92BF92CF9213
:10C52000DF92EF92FF920F931F93CF93DF93EC0173
:10C530006A017B01590120E030E0A90167E30E9414
:10C540002862A501980167E1CE010E94286281114D
:10C5500027C08F81833039F089E0CC0CDD1CEE1CC4
:10C56000FF1C8A95D1F7A701960169E1CE010E94CF
:10C57000286211E0882319F010E087E08C83CE0157
:10C580000E946662812FDF91CF911F910F91FF90E2
:10C59000EF90DF90CF90BF90AF909F908F900895D5
:10C5A00089E08C8310E0EBCFCF93DF93EC016EBD7D
:10C5B000FA01CA019E5F0DB407FEFDCF20812EBD9A
:10C5C0000DB407FEFDCF21812EBD3296E817F90785
:10C5D00091F70DB407FEFDCF8FEF0E940A3B8FEF5E
:10C5E0000E940A3B0E940F3B8E838F71853049F079
:10C5F00083E18C83CE010E94666280E0DF91CF915F
:10C60000089581E0FBCF0F931F93CF93DF93EC014D
:10C610008B010E941C620E94D9C381110CC085E16C
:10C620008C8310E0CE010E946662812FDF91CF9152
:10C630001F910F910895A8016CEFCE010E94D46262
:10C64000182F882361F3EECF0F931F93CF93DF93BF
:10C65000EC0189018F81833039F089E0440F551F47
:10C66000661F771F8A95D1F79A01AB0168E1CE0169
:10C670000E94286281112AC0A8016EEFCE010E949B
:10C68000D462182F8823B1F00E94D9C3182F8823B1
:10C69000D1F020E030E0A9016DE0CE010E942862D7
:10C6A000882321F086E18C8310E004C00E940F3BB8
:10C6B0008111F8CFCE010E946662812FDF91CF9168
:10C6C0001F910F91089587E18C83F4CF86E0EBCF23
:10C6D0001F93CF93DF93EC010E941C6220E030E0B7
:10C6E000A9016CE0CE010E94286211E0882319F0B4
:10C6F00010E083E08C83CE010E946662812FDF917F
:10C70000CF911F9108951F93CF93DF93EC018F81F9
:10C71000833039F089E0440F551F661F771F8A95D3
:10C72000D1F79A01AB0162E1CE010E94286211E0CB
:10C73000882319F010E085E08C83CE010E946662A8
:10C74000812FDF91CF911F9108958F929F92AF9289
:10C75000BF92EF92FF920F931F93CF93DF938C01C1
:10C76000EB017A010E945AC34B015C012CE2820E5C
:10C7700021E0921EA11CB11C0E940F3BF801868390
:10C780008F3F69F40E945AC3681979098A099B0985
:10C7900097FDF2CF81E1F8018483C0E021C08E3F94
:10C7A00071F5F1E0EF1AF1088FEF8EBDFE012FEF6A
:10C7B0000DB407FEFDCF8EB581932EBDCF018C1B2E
:10C7C0009D0B8E159F05A0F30DB407FEFDCF8EB512
:10C7D000CE0DDF1D88830E940F3B0E940F3BC1E0FE
:10C7E000C8010E9466628C2FDF91CF911F910F913B
:10C7F000FF90EF90BF90AF909F908F9008958FE043
:10C80000CACF0F931F93CF93DF93EC018B010E944C
:10C810001C6240E052E0B801CE01DF91CF911F9140
:10C820000F910C94A5630F931F93CF93DF93EC01AB
:10C8300089018F81833039F089E0440F551F661FCD
:10C84000771F8A95D1F79A01AB0161E1CE010E9471
:10C85000286281110AC040E052E0B801CE01DF91A8
:10C86000CF911F910F910C94A56384E08C83CE012E
:10C870000E94666280E0DF91CF911F910F91089531
:10C880008F929F92AF92BF92CF92DF92EF92FF92E0
:10C890000F931F93CF93DF93EC01162F1F821C82FF
:10C8A0004B830E945AC36B017C0120EDC20E27E02E
:10C8B000D21EE11CF11CA89561E08B810E94D9C1B8
:10C8C0008B810E94A0BA249A2C9A279A2698259A9E
:10C8D00081E00E94163B85E08D830E94163B0AE0B2
:10C8E0008FEF0E940A3B0150D9F7A89520E030E075
:10C8F000A90160E0CE010E9428628E83813081F020
:10C900000E945AC36C197D098E099F0997FDEECFCD
:10C9100081E08C83CE010E9466621A8280E06AC048
:10C92000A8952AEA31E040E050E068E0CE010E949C
:10C930002862853041F581E08F83A8958F81812C15
:10C94000912C5401823029F4812C912CA12C80E46B
:10C95000B82E20E030E0A90167E3CE010E942862F2
:10C96000A501940169E2CE010E9428628E8388238A
:10C97000F1F00E945AC36C197D098E099F0997FD39
:10C98000E8CF8AE0C6CF04E00E940F3B8E830150BF
:10C99000D9F78A3A11F482E0CFCF0E945AC36C19BA
:10C9A0007D098E099F0997FDBCCF82E0B2CF8F81B0
:10C9B0008230C1F420E030E0A9016AE3CE010E9498
:10C9C0002862882311F088E0A4CF0E940F3B807C6E
:10C9D000803C11F483E08F830E940F3B0E940F3B49
:10C9E0000E940F3BCE010E94666281E08A8317306D
:10C9F00070F41D83DF91CF911F910F91FF90EF9005
:10CA0000DF90CF90BF90AF909F908F90089588E176
:10CA10008C8384CF0F931F93CF93DF93EC018B0113
:10CA200020E030E0A90169E00E94286281110AC07B
:10CA300040E150E0B801CE01DF91CF911F910F91FD
:10CA40000C94A56380E18C83CE010E94666280E035
:10CA5000DF91CF911F910F910895CF93C82FCB01F4
:10CA60000E94CF388DE596E10E94CF388EE496E1A2
:10CA7000CC2311F083E596E10E94CF388AE0CF9174
:10CA80000C94B7380C9466C30C9466C3409176043A
:10CA900021E042276CE070E00C9447BC40917604A2
:10CAA00021E0422764E070E00C9447BC409176049A
:10CAB00021E0422761E070E00C9447BC409176048D
:10CAC00021E0422762E070E00C9447BC409176047C
:10CAD00021E0422761E070E00C9447BC409176046D
:10CAE00021E0422768E070E00C9447BC4091760456
:10CAF00021E042276CE070E00C9447BC41E061E02B
:10CB000070E00C9447BC4091760421E042270C94DD
:10CB100047BC62E070E00C94F2C26CE070E00C94F0
:10CB2000F2C264E070E00C94F2C261E070E00C9438
:10CB3000F2C261E070E00C94F2C26CE070E00C9420
:10CB4000F2C20F931F93CF93811113C0C42F8B0197
:10CB50000E9494398BE497E10E94CF38C8010E946B
:10CB6000CF38CC2331F08AE0CF911F910F910C94F4
:10CB7000B738CF911F910F910895CF93DF93809194
:10CB80001D1590911E15891B80958F7019F40E94B8
:10CB9000603FF5CF80911D158F5F8F70A0911D159F
:10CBA0009BE4A99FD0011124FD01ED5BF94FEF013A
:10CBB00019929A95E9F798E09083A85AB94F90E1B5
:10CBC000EFE1F5E101900D929A95E1F720911D15A5
:10CBD00090911E15291303C094E690931A15809323
:10CBE0001D15DF91CF910C942E3020E040E070E0D5
:10CBF00060E08EE697E60E944A1B81E08093CD05B7
:10CC00001092E7051092E605089520E040E070E0FC
:10CC100060E084E899E60C944A1B809140068111FB
:10CC200014C080915E0190915F0101972091A4143E
:10CC30003091A5142817390744F420E040E070E053
:10CC400060E089E899E60C944A1B0C94056621E0A3
:10CC50002093CD05FC0180819181A281B3818093D5
:10CC60001B0190931C01A0931D01B0931E0120E0B5
:10CC700040E070E060E08091C5059091C6050C949D
:10CC80004A1BCF93DF9300D000D0CDB7DEB78DEC39
:10CC90009CECACECBCE389839A83AB83BC83CE0170
:10CCA00001960E9427660F900F900F900F90DF91D2
:10CCB000CF910895CF93DF9300D000D0CDB7DEB7EA
:10CCC0008DEC9CECACECBDE389839A83AB83BC8395
:10CCD000CE0101960E9427660F900F900F900F9043
:10CCE000DF91CF910895CF93DF9300D000D0CDB7DF
:10CCF000DEB780E090E0A0E8BFE389839A83AB834E
:10CD0000BC83CE0101960E9427660F900F900F9072
:10CD10000F90DF91CF910895CF93DF9300D000D093
:10CD2000CDB7DEB780E090E0A0E2B1E489839A83DA
:10CD3000AB83BC83CE0101960E9427660F900F90B3
:10CD40000F900F90DF91CF91089581E08093CD05F2
:10CD500010929B051092850420E040E070E060E0B6
:10CD60008FE19CE60E944A1B88EA95E19093A90511
:10CD70008093A80508950C94921C2F923F924F9295
:10CD80005F926F927F928F929F92AF92BF92CF925B
:10CD9000DF92EF92FF920F931F93CF93DF93CDB764
:10CDA000DEB729970FB6F894DEBF0FBECDBF1C01CA
:10CDB0007987688769011A830983EB82BA01550F65
:10CDC000880B990B0E948EE220E030E0A9010E94BE
:10CDD0007EE94B015C0120E030E040E05FEC0E9426
:10CDE00001EB18162CF0812C912CA12C2FECB22EDB
:10CDF000C501B4010E9473EA2B013C01B601DD0CB0
:10CE0000880B990B0E948EE220E030E0A9010E947D
:10CE10007EE94B015C0120E030E040E05FE40E94ED
:10CE200087E287FD05C0812C912CA12C9FE4B92EAF
:10CE3000E885F98560817181072E000C880B990BBC
:10CE40000E948EE220E030E0A9010E947EE96B01A1
:10CE50007C01C301B2010E948EE29B01AC01C701BB
:10CE6000B6010E947DE90E947AEA6C837D838E83FD
:10CE70009F83C501B4010E9473EA7B018C01E41811
:10CE8000F50806091709FB81FF9389809A8083E1E1
:10CE9000A82E8CE6B82ECC80DD80A3019201688597
:10CEA0007985C1010E94051C0F9029960FB6F89450
:10CEB000DEBF0FBECDBFDF91CF911F910F91FF90CD
:10CEC000EF90DF90CF90BF90AF909F908F907F902A
:10CED0006F905F904F903F902F9008958F929F9208
:10CEE000AF92BF92CF92DF92EF92FF92CF93809159
:10CEF000CB051092CB05882369F01092CD05CF9118
:10CF0000FF90EF90DF90CF90BF90AF909F908F9069
:10CF10000C94921C4091D3055091D4056091D50595
:10CF20007091D605411551056105710599F0109272
:10CF3000D3051092D4051092D5051092D60581E044
:10CF4000809355012AE0249FC001259F900D112454
:10CF50000E9493C380915501882309F4AEC060916B
:10CF6000E6057091E705072E000C880B990B0E94CF
:10CF70008EE2209138063091390640913A06509160
:10CF80003B060E94EDE26B017C0120E030E040E2D4
:10CF900051E40E94EDE220E030E04AE754E40E94D0
:10CFA000EDE24B015C0120E030E0A901C701B601D0
:10CFB0000E9487E220E030E040EA50E487FF04C0AE
:10CFC00020E030E040EA50ECC501B4010E947EE967
:10CFD00020E030E040E251E40E9401EA0E9473EA5E
:10CFE0006B017C018BE2F7FE09C0F094E094D094D1
:10CFF000C094C11CD11CE11CF11C8DE28093DC03A8
:10D00000C701B60120E137E240E050E00E944DE95F
:10D010008AE0882E912CA12CB12CCA01B901A5015E
:10D0200094010E944DE9605D6093DD03C701B60184
:10D0300028EE33E040E050E00E944DE9CA01B9011A
:10D04000A50194010E944DE9605D6093DE038EE2CC
:10D050008093DF03C701B60124E630E040E050E0F2
:10D060000E944DE9CA01B901A50194010E944DE950
:10D07000605D6093E003C701B601A50194010E94C1
:10D080004DE9C62FCA01B901A50194010E944DE9DD
:10D09000605D6093E103C05DC093E2036CED73E0FB
:10D0A0008AE096E1CF91FF90EF90DF90CF90BF9014
:10D0B000AF909F908F900C94C922CF91FF90EF90EA
:10D0C000DF90CF90BF90AF909F908F9008956FEFBB
:10D0D0008091C7050C948FC14F925F926F927F929F
:10D0E0008F929F92AF92BF92CF92DF92EF92FF9278
:10D0F0000F931F93CF93DF930091C7050E9488BFC2
:10D10000C091CE0510E0000F111F07521A4E95E096
:10D11000592E5C0E2FEBE22E25E1F22ED3E0DC1B24
:10D1200037E6C32E38E6D32E41EBA42E45E1B42ECC
:10D1300082E0782E7C1A56EE852E55E1952E81E000
:10D14000682E6C1A4C2E4194C11137C08091D105C4
:10D150008823B1F080915501882359F081E09091A6
:10D16000D105911180E024E04DEC55E1642D0E9441
:10D17000CFBECF5F5C12E8CF84E08093CF050CC0B8
:10D180008091CB051092CB05882321F30E94921C3D
:10D190008091D0058823F1F2DF91CF911F910F91FB
:10D1A000FF90EF90DF90CF90BF90AF909F908F90C7
:10D1B0007F906F905F904F900895C13059F5F801BE
:10D1C000859194919093DF058093DE058091D10540
:10D1D000813081F080915501882359F21F929F92EE
:10D1E0008F926F9281E09091D105913009F474C0D3
:10D1F00080E072C08091CB051092CB05882351F35B
:10D200008091C705682F0E948FC18091D005882327
:10D2100009F3C2CFC23009F042C0F8018591949160
:10D220009093DF058093DE058091D1058230D1F0A7
:10D2300080915501882309F49CCFDF92CF92BF9251
:10D24000AF927F9281E09091D105923009F080E019
:10D250008F930E943C1B0F900F900F900F900F9098
:10D260000F9087CF8091CB051092CB05882301F3D7
:10D270000E9467688091D0058823D1F28DCF80917C
:10D28000CB051092CB058823C1F06091C7058FEFC5
:10D290000E948FC18091D005882379F07DCFC33063
:10D2A00009F067CFF801859194919093DF05809301
:10D2B000DE058091D105833011F3809155018823DB
:10D2C00009F457CF1F92FF92EF92DF9381E0909184
:10D2D000D105933009F08CCF8F930E943C1B0F90A7
:10D2E0000F900F900F900F9044CF64E07CE682E0A7
:10D2F0000C94F9D469E07CE681E00C94F9D46EE0FA
:10D300007CE680E00C94F9D46BEB79E683E00C9436
:10D31000F9D4EF92FF920F931F9386E5E82E85E1F3
:10D32000F82E08E515E12BEB36E645E056E668E613
:10D3300075E18DE695E10E9478C61F910F91FF90EF
:10D34000EF900895EF92FF920F931F9388E9E82ED4
:10D3500084E1F82E0BE015E12BEB36E64AEE5EE1B8
:10D360006AE974E18FE994E10E9478C61F910F91F8
:10D37000FF90EF900895CF93DF9300D000D0CDB70A
:10D38000DEB78091CB051092CB05882359F010921F
:10D39000CD050E94921C0F900F900F900F90DF917F
:10D3A000CF9108956091D3057091D4058091D505F2
:10D3B0009091D605611571058105910561F10E9475
:10D3C0008EE220911B0130911C0140911D01509172
:10D3D0001E010E94EDE22091480B3091490B4091D3
:10D3E0004A0B50914B0B0E947EE96093480B70935F
:10D3F000490B80934A0B90934B0B83E00E944F1F85
:10D4000081E0809355011092D3051092D4051092BB
:10D41000D5051092D60580915501882309F4BBCF1C
:10D420002091C1053091C2054091C3055091C405BA
:10D430006091480B7091490B80914A0B90914B0B76
:10D440000E947DE969837A838B839C83CE01019658
:10D450000E948A60BC0180E097E20E94C9229BCFB3
:10D460002F923F924F925F926F927F928F929F92F4
:10D47000AF92BF92CF92DF92EF92FF921F93CF9322
:10D48000DF93CDB7DEB72C970FB6F894DEBF0FBE93
:10D49000CDBF1C01162F8091CB051092CB058823A0
:10D4A000E1F01092CD050E94921C2C960FB6F894D4
:10D4B000DEBF0FBECDBFDF91CF911F91FF90EF90E8
:10D4C000DF90CF90BF90AF909F908F907F906F90A4
:10D4D0005F904F903F902F9008958091D305909149
:10D4E000D405A091D505B091D6058D839E83AF83D9
:10D4F000B887892B8A2B8B2B09F460C08091270178
:10D50000882309F4BDC0809128018111B9C0613020
:10D5100009F494C0623009F4A2C08090290190906F
:10D520002A01A0902B01B0902C01C0903501D09021
:10D530003601E0903701F0903801612E712C6D8139
:10D540007E818F8198850E948EE220911B0130910F
:10D550001C0140911D0150911E010E94EDE2D3017A
:10D56000AA0FBB1FAA0FBB1FBC87AB87A45CB44F1D
:10D57000BA87A9872D913D914D915C910E947EE9DA
:10D580002B013C018D819E81AF81B885B7FF8FC093
:10D59000A5019401C301B2010E9487E287FD7FC00B
:10D5A000EB85FC85E45CF44F408251826282738299
:10D5B000812F0E944F1F81E0809355011092D30567
:10D5C0001092D4051092D5051092D6058091550180
:10D5D000882309F46ACFF4E01F9FC0011124FC01E5
:10D5E000E45CF44F87509A4FDC012D913D914D91B1
:10D5F0005C9160817181828193810E947EE96B01DF
:10D600007C01C982DA82EB82FC822DEC3CEC4CEC92
:10D610005DE360911B0170911C0180911D0190914F
:10D620001E010E9401EB87FD52C0CE0101960E94AF
:10D630008A60BC01C1010E94C92237CF80902D01B0
:10D6400090902E01A0902F01B0903001C090390130
:10D65000D0903A01E0903B01F0903C016ECF809079
:10D66000310190903201A0903301B0903401C0900C
:10D670003D01D0903E01E0903F01F09040015DCF30
:10D68000812C30E5932E33ECA32E37ECB32EC12C36
:10D6900040E5D42E43ECE42E47E4F42E4ECFA9858A
:10D6A000BA858D929D92AD92BC92139781CFA701BE
:10D6B0009601C301B2010E9401EB18160CF070CF65
:10D6C000E985FA85C082D182E282F38271CF20E0BF
:10D6D00030E040E251E4C701B6010E94EDE220E0F3
:10D6E00030E04AE754E40E94EDE24B015C0120E0A7
:10D6F00030E0A901C701B6010E9487E220E030E0D6
:10D7000040EA50E487FF04C020E030E040EA50ECFB
:10D71000C501B4010E947EE920E030E040E251E41E
:10D720000E9401EA0E9473EA6B017C01F7FC62C06F
:10D7300020EA36E841E050E00E944DE9CA01B90113
:10D740002AE030E040E050E00E944DE9605D6093E7
:10D75000DC03C701B60120E137E240E050E00E945F
:10D760004DE98AE0882E912CA12CB12CCA01B90177
:10D77000A50194010E944DE9605D6093DD03C7013E
:10D78000B60128EE33E040E050E00E944DE9CA01C6
:10D79000B901A50194010E944DE9605D6093DE032B
:10D7A0008EE28093DF03C701B60124E630E040E05B
:10D7B00050E00E944DE9CA01B901A50194010E94FF
:10D7C0004DE9605D6093E003C701B601A5019401D6
:10D7D0000E944DE9162FCA01B901A50194010E94CA
:10D7E0004DE9605D6093E103105D1093E2038CED01
:10D7F00093E01FCFF094E094D094C094C11CD11C4E
:10D80000E11CF11C6DE2A3CF62E089E097E20C9489
:10D81000306A61E080E197E20C94306A60E087E171
:10D8200097E20C94306A6CE971E68DE994E90C9406
:10D8300009246FEA71E688EC91E60C940924809142
:10D840005501882331F041E061EC73E182E00E94F0
:10D8500072BE809185048770873041F420E040E0FB
:10D8600070E060E089EB92EA0C944A1B08950F93F4
:10D870001F93CF93DF93CDB7DEB72A970FB6F894F7
:10D88000DEBF0FBECDBF809155018823F1F01F92FE
:10D8900089E18F938091DA0390E001969F938F93B3
:10D8A0008EE993E19F938F938E010F5F1F4F1F931C
:10D8B0000F930E941EE2B80183E993E10E94C922FE
:10D8C0000FB6F894DEBF0FBECDBF84E08093550144
:10D8D0008091D903811108C020E040E070E060E051
:10D8E00088E493E20E944A1B2A960FB6F894DEBFA2
:10D8F0000FBECDBFDF91CF911F910F910895CF93B0
:10D90000DF93EC010E941CCE1B82DF91CF91089522
:10D91000CF93DF93EC01462F41706C857D858E851A
:10D920009F850E94E9CA882351F0888920E2829F5E
:10D93000C001112481579D4EDF91CF91089590E051
:10D9400080E0FACFCF93DF93EB01FC01238121111B
:10D9500004C080E0DF91CF9108952250223028F456
:10D960008FE28883198281E0F5CF60E00E94886CA5
:10D97000009779F3DC0160E080E09EE22D91203297
:10D9800099F0883031F49E01260F311DF901908302
:10D990006F5F9E01260F311DAD0141505109FA0103
:10D9A0004081F90140836F5F8F5F8B3039F7FE0153
:10D9B000E60FF11D1082D7CF3F924F925F926F9288
:10D9C0007F928F929F92AF92BF92CF92DF92EF920F
:10D9D000FF920F931F93CF93DF93CDB7DEB72C97B2
:10D9E0000FB6F894DEBF0FBECDBF5C01DC015996C7
:10D9F0008D909C90F40181859285A385B4859C01CE
:10DA0000AD012F5F3F4F4F4F5F4F29873A874B87BD
:10DA10005C87D50114964D905D906D907C90179722
:10DA2000411451046104710409F459C0BFEF4B1A49
:10DA30005B0A6B0A7B0A312C730162011D821E8214
:10DA40001F821886F40181859285A385B4852D8176
:10DA50003E814F815885281739074A075B0708F030
:10DA600056C089859A85AB85BC858C159D05AE050C
:10DA7000BF0550F482E0C82ED12CE12CF12C92E0AD
:10DA8000492E512C612C712C9E012F5F3F4FB70105
:10DA9000A601C4010E9423CD8823C9F189819A81FE
:10DAA000AB81BC81892B8A2B8B2B01F1260137019D
:10DAB0009FEF491A590A690A790A2D813E814F81DF
:10DAC00058852F5F3F4F4F4F5F4F2D833E834F83CE
:10DAD00058873FEFC31AD30AE30AF30AB3CF408053
:10DAE00051806280738033243394A6CFC414D5044C
:10DAF000E604F70411F70FEF1FEF2FEF3FE0B70138
:10DB0000A601C4010E9491CC782E81111AC0712CFB
:10DB1000872D2C960FB6F894DEBF0FBECDBFDF91D8
:10DB2000CF911F910F91FF90EF90DF90CF90BF901A
:10DB3000AF909F908F907F906F905F904F903F90AD
:10DB40000895F5014481558166817781411551051C
:10DB50006105710539F097018601C4010E9491CCDD
:10DB60008823A9F2D5011496CD92DD92ED92FC9214
:10DB70001797332051F0D701C6010196A11DB11DA1
:10DB8000F40180839183A283B383F501858996890B
:10DB9000A789B08D892B8A2B8B2B09F0B9CFC58A29
:10DBA000D68AE78AF08E818180688183B1CF40E098
:10DBB00050E0BA010C946BCE4F925F926F927F92BD
:10DBC000AF92BF92CF92DF92EF92FF920F931F938B
:10DBD000CF93DF931F92CDB7DEB78C017B015A0143
:10DBE000C22EDB0159968D919C91F801928F818F05
:10DBF000CB010E94D76D712CF70180859185A2859C
:10DC0000B385418952896389748984179507A6076A
:10DC1000B70708F052C055E0B695A7959795879538
:10DC20005A95D1F7F82FFF70DF2ED70113968C91FC
:10DC3000823010F480E0DBC041E050E0BE016F5F55
:10DC40007F4FC7010E9493CF0197A1F7F70180850D
:10DC50009185A285B3854F96A11DB11D80879187BF
:10DC6000A287B387F0E2DF9EB001112461577D4E99
:10DC700061157105F9F2DB018C91882341F0853E35
:10DC800009F04CC0772029F077247394B5CF711038
:10DC90000EC080918F1490919014A0919114B09126
:10DCA0009214F80184879587A687B787D08ADB010D
:10DCB0008C918111E9CF772473948C2D82748234F6
:10DCC00009F0B8CF772009F4A2C0F801D08861E04C
:10DCD000C8010E94886C009709F4ACCF20E2DC01F7
:10DCE0001D922A95E9F72BE0F501DC0101900D92D8
:10DCF0002A95E1F721E238E2FC01318B208B40E0EC
:10DD000058E057874687338B228B318F208F578B74
:10DD1000468B0E94A0CA811109C08CCF4BE050E015
:10DD2000C5010E9493EB892B09F066CFF0E2DF9EDC
:10DD3000D00111249D0121573D4EF9018385817148
:10DD400021F08C2D827109F001C1F801818D928D35
:10DD500040918F145091901460919114709192148D
:10DD60004487558766877787D08AFD01E157FD4E46
:10DD700044885588712C612C320155244424D801E3
:10DD800055964D925D926D927C925897428D538D2F
:10DD900070E060E0442955296629772955964D930E
:10DDA0005D936D937C935897D9011B962C912871A4
:10DDB00009F0BEC0848D958DA68DB78DF801818B3D
:10DDC000928BA38BB48B81E083838C2D8F70F801B1
:10DDD000818314821582168217821086118612861C
:10DDE000138681E0C4FE03C0C8010E94FFCE0F90DD
:10DDF000DF91CF911F910F91FF90EF90DF90CF9027
:10DE0000BF90AF907F906F905F904F900895D70133
:10DE100013968C911397823009F40CCF51968D9103
:10DE20009D910D90BC91A02D803E9F4FAF41B105BB
:10DE300008F000CFC7010E94DC6C882309F4FACEF9
:10DE40000E94A0CA882309F4F5CED7015996ED9116
:10DE5000FC915A9714964D905D906D907C90179719
:10DE6000B2E04B1A510861087108858504C0440C62
:10DE7000551C661C771C8A95D2F786859785A089E4
:10DE8000B189480E591E6A1E7B1E81E0809393144F
:10DE900040928F1450929014609291147092921448
:10DEA000EFE8F2E180E092E0DF019C011D92215059
:10DEB0003040E1F7DD24D394D7015996ED91FC91E0
:10DEC0008481D816C0F48091941490919514DC014B
:10DED000ED91FC910288F389E02D2FE832E1B30146
:10DEE000A2014D0D511D611D711D0995882309F475
:10DEF000A1CED394E1CF258580E092E0A0E0B0E010
:10DF000004C0880F991FAA1FBB1F2A95D2F7F701DB
:10DF10004189528963897489840F951FA61FB71F91
:10DF2000818B928BA38BB48B8FE892E1D12CD6CED0
:10DF3000203161F498012F5E3F4F0E94A6CD8823C7
:10DF400029F084E0D80113968C933FCFD801139623
:10DF50001C9270CEFC01238121110C947F6C0895DA
:10DF60002F923F924F925F926F927F928F929F92E9
:10DF7000AF92BF92CF92DF92EF92FF920F931F93D7
:10DF8000CF93DF93CDB7DEB7C354D1090FB6F89462
:10DF9000DEBF0FBECDBF4C015B016A01222E19828C
:10DFA0001C821C8E1F8E6115710521F510E0CE01BB
:10DFB0004C960E94AA6FCE0101960E94AA6F812FF3
:10DFC000CD5BDF4F0FB6F894DEBF0FBECDBFDF9144
:10DFD000CF911F910F91FF90EF90DF90CF90BF9066
:10DFE000AF909F908F907F906F905F904F903F90F9
:10DFF0002F900895FC0183818111D8CFFA0180818F
:10E000008F32A1F18B01CE0101967C013C0180E2AF
:10E01000382E2E019CE1490E511C2396EFAE23971A
:10E020002496FFAE249722963FAE229721963FAECC
:10E0300021973FAE3EAE3DAE3CAE3BAE3AAE39AEC2
:10E0400038AE3FAA960190E047E0D9018D91882330
:10E0500009F447C08F3209F444C08E3209F54A30C2
:10E0600009F4A4CF98E04AE09D01EFCFFB01838142
:10E0700082508B01823060F0618D728DCE014C96A2
:10E080000E94DBD38E01045E1F4F882309F48ECFDC
:10E09000C6016C010196F60120812F32D1F3B3CF76
:10E0A000EFE3F3E22491222321F031968213FACF99
:10E0B0007DCF491708F47ACF813208F477CF8F37B4
:10E0C00009F474CF3FE9380F3A3108F420EEE7E362
:10E0D000F0E0EC0FFD1FE90FF11D820F80839F5FC1
:10E0E000C3CF8FA9803209F461CF6901F901808122
:10E0F0002F5F3F4F8F32C9F3882301F121E0AE013A
:10E10000495C5F4FB801C7010E94DC6D882309F4A8
:10E110004DCF0A151B0519F0C8010E947F6C942D84
:10E12000852D6E147F0431F023969FAD239724969E
:10E130008FAD24978701E92EF82E75CF222DAE01E1
:10E14000495C5F4FB801C4010E94DC6D182F2FCFCE
:10E150002F923F924F925F926F927F928F929F92F7
:10E16000AF92BF92CF92DF92EF92FF920F931F93E5
:10E17000CF93DF93CDB7DEB7ED970FB6F894DEBF40
:10E180000FBECDBF8091D205882369F18091C5165D
:10E1900000E010E083FF23C082ED94E10E94D76D80
:10E1A0008BE1E2EDF4E1DE01919601900D928A950A
:10E1B000E1F710E000E0BE016F5F7F4FCE01819676
:10E1C0000E948CD018163CF4CE0101960E946FCAB2
:10E1D000080F111DF0CFCE0181960E94AA6F009307
:10E1E0007A0410937B040E9488BF1091CE051CAF67
:10E1F00085E0810F8DAF312E31948DE5C82E81E6FB
:10E20000D82E94E4A92E95E1B92E81E0782E711ACA
:10E2100028E4822E25E1922E111113C08091D105A0
:10E22000882391F180915501882359F081E09091E4
:10E23000D105911180E024E041E555E1632D0E9474
:10E24000CFBE8091C51685FF55C01130D9F480919D
:10E25000D1058130F1F180915501882309F45BC12A
:10E260001F929F928F927F9281E09091D105913081
:10E2700009F080E08F930E943C1B0F900F900F904D
:10E280000F900F9082E066C08091CB051092CB0575
:10E29000882341F20E94921C8091D005882311F2BC
:10E2A000ED960FB6F894DEBF0FBECDBFDF91CF91D4
:10E2B0001F910F91FF90EF90DF90CF90BF90AF90A4
:10E2C0009F908F907F906F905F904F903F902F9096
:10E2D00008958091CB051092CB05882309F4BBCF1C
:10E2E0001092CE050E942BD48091D005882309F48A
:10E2F000B2CFD6CF83FF2DC0113021F68091D1054A
:10E300008130D1F080915501882309F404C1DF9256
:10E31000CF92BF92AF927F9281E09091D1059130E0
:10E3200009F080E08F930E943C1B0F900F900F909C
:10E330000F900F900F90A6CF8091CB051092CB0538
:10E34000882301F30E945D618091D0058823D1F27A
:10E35000A7CF81E090915501992309F4DDC0582E93
:10E36000082FF12CE12C412E9CAD491A802F2091D1
:10E370007A0430917B04E216F30608F0CDC0011355
:10E38000A5C082ED94E10E94D76D202E25188BE167
:10E39000E2EDF4E1DE01919601900D928A95E1F7AC
:10E3A000612CBE016F5F7F4FCE0181960E948CD0A1
:10E3B00018167CF4CE0101960E946FCA882389F357
:10E3C00026106BC0BE016F5F7F4F8BEE95E00E9401
:10E3D0008ACACE0181960E94AA6F8091C51690913B
:10E3E000D10584FF78C0911366C08091CB0510924F
:10E3F000CB05882309F45FC019821C828091D51453
:10E400006DEE74E1882311F062ED74E121E04BEED2
:10E4100055E0CE0101960E94B06F882309F43FC0F9
:10E420008BE1FE013196A2EDB4E101900D928A9547
:10E43000E1F78091C5168F7D8093C516A091BA161D
:10E44000AA3080F481E08A0F8093BA168BE18A9F0C
:10E45000D0011124A455BA4EE2EDF4E101900D92E1
:10E460008A95E1F7CE0101960E94AA6F1092CE051F
:10E4700082E090E0A0E0B0E08093D3059093D405D3
:10E48000A093D505B093D60581E08093D005109276
:10E49000DB0383E08093550103CF639482CF0E9416
:10E4A00094396BEE75E08EE295E10E94563F8AE06A
:10E4B0000E94B738D7CF80915501882339F081E089
:10E4C000911380E041E0642D0E9410BF8FEFE81AA5
:10E4D000F80A0F5F4BCF911759F0809155018823AF
:10E4E000A9F381E09091D105911380E040E0EBCF5A
:10E4F0008091CB051092CB05882379F38BEE95E0C4
:10E500000E9411CA0E94791C0E941DBD8091D005F5
:10E51000882319F3C5CE82E01F5F9DAD91137CCE99
:10E520008093CF05BDCE8F929F92AF92BF92CF9234
:10E53000DF92EF92FF92CF936B017C01B42E20E02B
:10E5400030E0A9010E9487E287FF07C08DE20E94A8
:10E55000B738F7FAF094F7F8F094C0E060E070E0B4
:10E5600080E09FE3CB1541F02DEC3CEC4CEC5DE3FF
:10E570000E94EDE2CF5FF6CFA70196010E947EE9EF
:10E580006B017C010E947AEA4B015C014AE00E9427
:10E5900086C9CC2379F1C501B4010E948CE29B01AC
:10E5A000AC01C701B6010E947DE96B017C018EE2DE
:10E5B0000E94B738C150F0F020E030E040E251E472
:10E5C000C701B6010E94EDE26B017C010E947AEA6C
:10E5D0004B015C014AE00E9486C9C501B4010E945A
:10E5E0008CE29B01AC01C701B6010E947DE96B0181
:10E5F0007C01E0CFCF91FF90EF90DF90CF90BF9064
:10E60000AF909F908F900895EF92FF920F931F937A
:10E61000CF937C018B01C2E44F3F09F0C4E580E257
:10E620000E94B7388C2F0E94B7388AE30E94B7380F
:10E63000F701608171818281938142E00E9493722F
:10E6400083E393E20E94CF38F80160817181828177
:10E65000938142E00E94937262E070E080E090E07B
:10E66000CF911F910F91FF90EF900C94BFC21F9319
:10E67000CF93DF93CDB7DEB728970FB6F894DEBF00
:10E680000FBECDBF182F6091A6147091A714072E4E
:10E69000000C880B990B0E948EE26D837E838F8322
:10E6A00098876091A4147091A514072E000C880B14
:10E6B000990B0E948EE269837A838B839C834AEF55
:10E6C000BE016B5F7F4FCE0101960E940473609183
:10E6D000B2057091B305072E000C880B990B0E94B0
:10E6E0008EE26D837E838F8398876091B0057091F1
:10E6F000B105072E000C880B990B0E948EE26983EE
:10E700007A838B839C834FEFBE016B5F7F4FCE017B
:10E7100001960E9404736091B4051F3F39F085E1B2
:10E720001802F0011124E056FB4E608570E08BE387
:10E7300093E20E9486396091B40570E086E393E22B
:10E740000E94863928960FB6F894DEBF0FBECDBF63
:10E75000DF91CF911F9108950F930FB70F93009101
:10E760006E000B7F00936E0078940F930BB70F939E
:10E770000CB70F921F922F933F934F935F936F931A
:10E780007F938F939F93AF93BF93EF93FF93112446
:10E790000E946B7CFF91EF91BF91AF919F918F9100
:10E7A0007F916F915F914F913F912F911F900F90AB
:10E7B0000CBF0F910BBF0F910460F89400936E0093
:10E7C0000F910FBF0F911895CF93DF93C0EAD4E15B
:10E7D0001F821E820E9466C318865D98CCEAD5E02F
:10E7E0001F821E820E94EF6118865C98DF91CF9194
:10E7F000089510922F060E94E4730C94791C4F9296
:10E800005F926F927F928F929F92AF92BF92EF92A0
:10E81000FF920F931F93CF93DF93B0E2A0E06A2F94
:10E8200070E0AB014B0F511D55954795411117C035
:10E83000E7E5F2E285919491282F822FDF91CF9125
:10E840001F910F91FF90EF90BF90AF909F908F908E
:10E850007F906F905F904F900895B42FE2CFA417F0
:10E8600011F0B41303C0E3EDF2E2E4CF9A012150BA
:10E870003109220F331F220F331FF901EB5AFD4DCF
:10E88000E590F490F901E75AFD4D059114918E152C
:10E890009F051CF3A42F081719070CF4C0CFBC0167
:10E8A000F901E95AFD4DC591D491F901E55AFD4DA3
:10E8B000A590B4906E197F09072E000C880B990B58
:10E8C0000E948EE22B013C01B5016C1B7D0B072ED3
:10E8D000000C880B990B0E948EE29B01AC01C301D6
:10E8E000B2010E94EDE24B015C01B8016E197F0993
:10E8F000072E000C880B990B0E948EE29B01AC0145
:10E90000C501B4010E9401EA4B015C01BE01DD0FAB
:10E91000880B990B0E948EE29B01AC01C501B401EA
:10E920000E947EE90E9473EA262F972F86CFCF930D
:10E93000DF93C0EAD4E18A819B810E94FEB89D8367
:10E940008C83CCEAD5E08A819B810E94FF739D83F2
:10E950008C83A89510927904DF91CF910895EF925E
:10E96000FF920F931F93CF93DF93C82F7B018A01F0
:10E970008091AB058130A1F40E949039C7010E94BB
:10E98000CF388BE092E20E94CF38C7FD33C08C2F86
:10E990000C2E000C990B0E9496B98AE00E94B738A1
:10E9A0000E94E473A8958091FC04811132C081E03B
:10E9B0008093FC0480E88093AB050E94E473D5E16A
:10E9C000D150149AE1F069E170E080E090E00E949B
:10E9D000BFC2A895149868E270E080E090E00E94C1
:10E9E000BFC2A89568E270E080E090E00E94BFC2DC
:10E9F000A895E6CF87E092E20E94CF38CECF60E0C4
:10EA000072E2CF3F11F064E072E240E0C8010E9480
:10EA1000BD39DF91CF911F910F91FF90EF90089535
:10EA20004F925F926F927F928F929F92AF92BF921E
:10EA3000CF92DF92EF92FF920F931F93CF93DF93CA
:10EA4000EC016B014A01B22EFA01408051806280D4
:10EA50007380A30192016D817E818F8198850E94D0
:10EA600087E28823A1F04D825E826F827886AA2495
:10EA7000A39420E030E0A901F401608171818281DA
:10EA800093810E9401EB18160CF0A12CAC828C81B2
:10EA90008230A1F0833009F45AC08130C9F52D814C
:10EAA0003E814F815885F601608171818281938119
:10EAB0000E9487E287FD2CC082E08C83B701FF0CA7
:10EAC000880B990B0E948EE29B01AC016D817E81C7
:10EAD0008F8198850E947DE99B01AC01F6016081E0
:10EAE0007181828193810E9401EB87FD22C00E9487
:10EAF0005AC36B017C019801A8EEB3E00E94FCE8C8
:10EB0000C60ED71EE81EF91EC882D982EA82FB8291
:10EB1000DF91CF911F910F91FF90EF90DF90CF90F9
:10EB2000BF90AF909F908F907F906F905F904F902D
:10EB300008950E945AC3088119812A813B81601B74
:10EB4000710B820B930B97FDE3CF83E08C8345ED34
:10EB500052E265EE72E28B2DDF91CF911F910F9102
:10EB6000FF90EF90DF90CF90BF90AF909F908F90ED
:10EB70007F906F905F904F900C94AF74CF93DF9322
:10EB8000EC01488159816A817B8186EF91E20E9484
:10EB9000483B4C815D816E817F818EE997E20E94C6
:10EBA000483B488559856A857B858AE997E20E94BA
:10EBB000483B8AE0DF91CF910C94B738BC0120919B
:10EBC000DD043091DE044091DD045091DE04241711
:10EBD000350731F481E02617370709F080E0089502
:10EBE0009A01F1CF0F930FB70F9300916E000F931F
:10EBF0000B7F00936E0000916F000D7F00936F00FC
:10EC00000F930BB70F930CB70F921F922F933F9355
:10EC10004F935F936F937F938F939F93AF93BF9324
:10EC2000EF93FF9311240E94007EFF91EF91BF911B
:10EC3000AF919F918F917F916F915F914F913F9194
:10EC40002F911F900F900CBF0F910BBF0F9102607F
:10EC5000F89400936F000F9100936E000F910FBF17
:10EC60000F911895000000000000000080919A05A7
:10EC700080FF27C0459A8FEF8093930480919A0577
:10EC8000869580FF21C0479A8FEF809394048091EE
:10EC90009A058695869580FF1AC02A988FEF8093F3
:10ECA000950480919A0586958695869580FF12C079
:10ECB000289A8FEF80939604000000000000000067
:10ECC0000895459881E0D8CF479881E0DECF2A9A11
:10ECD00081E0E5CF289881E0EDCFCF92DF92EF92EF
:10ECE000FF920F931F93CF93DF93CDB7DEB7C65834
:10ECF000D1090FB6F894DEBF0FBECDBFC358DF4FAA
:10ED0000188219821A821B82CD57D04080910C0242
:10ED100090910D02A0910E02B0910F02CF57DF4FDC
:10ED200088839983AA83BB83C158D04084E690E04E
:10ED300090930606809305061092B6141092B514AF
:10ED40001092920464E070E0CE018F579F4F0E94B2
:10ED5000F2C28091050690910606029690930606EF
:10ED6000809305061092B6141092B51481E0CA572C
:10ED7000DF4F8883C658D040CE018A579F4F0E94EC
:10ED8000996568E470E084EF9AE00E94F2C260E165
:10ED900070E087E096E00E94F2C28AE097EDA3EA75
:10EDA000BCE3C358DF4F88839983AA83BB83CD57C5
:10EDB000D040CE0183589F4F0E9491658CE995E029
:10EDC0000E949D657E018DE6E80EF11C8FEFD70154
:10EDD0008C93C7010E94996519821A821B821C823A
:10EDE0008E010F5F1F4FC8010E94916519821A8220
:10EDF0001B821C82C8010E94916585E08983F7010E
:10EE0000808382E794E00E949165C8010E94996521
:10EE1000C7010E94996564E670E08EE094E00E946C
:10EE2000F2C28CE0D8011D928A95E9F7C8010E94D0
:10EE30009D65C358DF4F188219821A821B82CD57F5
:10EE4000D0403AE0D32EDA94DD2031F0CE01835861
:10EE50009F4F0E949165F7CF88E0F701982F11929C
:10EE60009A95E9F7D8011D928A95E9F783E0CB5787
:10EE7000DF4F8883C558D040EA968FAFEA97CE011E
:10EE80008B579F4F0E949965CE0187589F4F0E94D4
:10EE9000996568E070E0C8010E94F2C268E070E025
:10EEA000C7010E94F2C2C358DF4F188219821A822A
:10EEB0001B82CD57D0402AE0C22ED12CB1E0CB1A14
:10EEC000D10831F0CE0183589F4F0E949165F6CF53
:10EED00019828FEFF7018083C8010E949565C701F1
:10EEE0000E94996580E1D82ED801ED2D1D92EA95FA
:10EEF000E9F760E170E0C8010E94F2C21982C8011E
:10EF00000E9495656CE070E085EB95E00E94F2C28E
:10EF1000198A1A8A1B8A1C8A80E090E0A0E8BFE365
:10EF20008D879E87AF87B88B8091A9149091AA1482
:10EF3000A091AB14B091AC1489839A83AB83BC834A
:10EF40002CEA35EC47E25EE36091AD147091AE14AB
:10EF50008091AF149091B0140E9401EA6D837E837A
:10EF60008F8398872CEA35EC47E25EE36091B11419
:10EF70007091B2148091B3149091B4140E94EDE298
:10EF800069877A878B879C8764E170E0C8010E945B
:10EF9000F2C284E190E09A838983C8010E94896566
:10EFA0008CE0ECE8F1E0D80101900D928A95E1F750
:10EFB000C8010E948D658CE0ECE8F1E0D801019079
:10EFC0000D928A95E1F7C8010E948D651982C801EA
:10EFD0000E94996580914101909142019A838983B1
:10EFE000C8010E94896585E0E8E9F1E0D801019057
:10EFF0000D928A95E1F765E070E0C8010E94F2C2C7
:10F000001982C8010E94956580E2EDE9F1E0D8011E
:10F0100001900D928A95E1F760E270E0C8010E94CC
:10F02000F2C2D7011C92C7010E9495658DE094E061
:10F030000E94956589E094E00E949165C358DF4F76
:10F04000188219821A821B82CD57D040CE01835874
:10F050009F4F0E94916580E2F80111928A95E9F72D
:10F0600060E270E0C8010E94F2C2FE01F99688E0F9
:10F07000DF011D928A95E9F744E650E060E070E018
:10F0800049835A836B837C834D835E836F83788748
:10F0900083E090E0A0E0B0E089879A87AB87BC87E7
:10F0A0004D875E876F87788B498B5A8B6B8B7C8BF8
:10F0B0008D8B9E8BAF8BB88F898F9A8FAB8FBC8FC8
:10F0C0008D8F9E8FAF8FB8A38EE190E0A0E0B0E06F
:10F0D00089A39AA3ABA3BCA38DA39EA3AFA3B8A7F8
:10F0E00089A79AA7ABA7BCA78DA79EA7AFA7B8ABC8
:10F0F00089AB9AABABABBCAB8DAB9EABAFABB8AF98
:10F1000060E470E0C8010E94F2C2F8018D2D1192F6
:10F110008A95E9F760E170E0C8010E94F2C2D80167
:10F120001D92DA94E9F760E170E0C8010E94F2C232
:10F13000C358DF4F188219821A821B82CD57D040E4
:10F14000CE0183589F4F0E9491659CE0D92EF80113
:10F150008D2D11928A95E9F76CE070E0C8010E944C
:10F16000F2C28CE6D8011D928A95E9F76CE670E050
:10F17000C8010E94F2C286E894E00E948D65F70102
:10F1800010821182128213821482158216821782D3
:10F1900068E070E0C7010E94F2C2F7011192DA94B0
:10F1A000E9F7CB57DF4F1882C558D04080E090E098
:10F1B000A0E4B0E4ED968CAF9DAFAEAFBFAFED97DE
:10F1C000C7010E949D65CE018B579F4F0E94996594
:10F1D000CE0187589F4F0E949165809192048111C2
:10F1E00024C000910506109106068091B5149091F7
:10F1F000B614D7018D939C9384E690E09093060615
:10F200008093050664E070E089EC91E00E94F2C210
:10F21000C7010E94896591E00D34134009F490E024
:10F2200080919204892B80939204809192048111A1
:10F2300005C060E087E297E10E94831E90919204EE
:10F2400081E08927CA57DF4F0FB6F894DEBF0FBEA3
:10F25000CDBFDF91CF911F910F91FF90EF90DF9085
:10F26000CF900895AF92BF92CF92DF92EF92FF922C
:10F270000F931F93CF93DF93C4EFDAE007E116E01B
:10F2800084E0A82E8BE0B82EC12CD12C7601C3943B
:10F2900069917991899199910E948CE228893989A3
:10F2A0004A895B890E94EDE20E947AEAF801619343
:10F2B0007193819391938F01C616D706E806F906DC
:10F2C00010F46B017C01AC16BD0611F76FEF7FEFF8
:10F2D000CB01A70196010E94CFE820932706309327
:10F2E00028064093290650932A06DF91CF911F915B
:10F2F0000F91FF90EF90DF90CF90BF90AF90089567
:10F300000F931F93CF93DF9308E01BE0C0E3D6E099
:10F31000F80121913191419151918F0160E070E0AC
:10F3200080E89FE30E9401EA699379938993999316
:10F33000F6E0C034DF0761F70E9401BCDF91CF9196
:10F340001F910F910C94327990911D1580911E158B
:10F35000981306C08091410690914206892B19F0BE
:10F360000E94603FF1CF089590911D1580911E1568
:10F37000981308C08091410690914206892B11F4A0
:10F380000C9419330E94603FEFCFCF93DF9320910D
:10F390000804222379F0EC010E941D5F9B01AC015F
:10F3A000688579858A859B850E947DE9688779874C
:10F3B0008A879B87DF91CF910895CF93DF93209128
:10F3C0000804222379F0EC010E941D5F9B01AC012F
:10F3D000688579858A859B850E947EE9688779871B
:10F3E0008A879B87DF91CF9108954F925F926F92AA
:10F3F0007F928F929F92AF92BF92CF92DF92EF92C5
:10F40000FF920F931F93CF93DF93CDB7DEB76A9729
:10F410000FB6F894DEBF0FBECDBF9A8F898F5B0108
:10F420008A01DC01D6966D917D918D919C91D99741
:10F430000E948CE26B017C01F501208131814281C7
:10F4400053810E94EDE20E94EAE92B013C01D801C0
:10F450002D913D914D915C91C701B6010E94EDE265
:10F460000E94EAE94B015C01C301B2010E947AEA01
:10F47000698B7A8B8B8B9C8B683771058105910525
:10F4800040F428E730E040E050E0298B3A8B4B8B8A
:10F490005C8BC501B4010E947AEA6D877E878F87F5
:10F4A000988B683771058105910540F488E790E0F5
:10F4B000A0E0B0E08D879E87AF87B88BE98DFA8D8D
:10F4C000EE5BFF4F208131814281538129833A8352
:10F4D0004B835C83CA01B9010E948EE22B013C017F
:10F4E00069897A898B899C890E948CE269877A87ED
:10F4F0008B879C8720E030E0A901C301B2010E9404
:10F5000087E2882309F43BC1A7019601C701B60130
:10F510000E94EDE24B015C0129853A854B855C85B3
:10F52000CA01B9010E94EDE29B01AC01C501B40121
:10F530000E947DE94B015C01A3019201C301B2016C
:10F540000E947EE99B01AC01C501B4010E9401EA61
:10F550000E94EAE90E947AEA6D837E838F8398870E
:10F5600069817A818B819C81909580957095619558
:10F570007F4F8F4F9F4F0E948EE24B015C016D8544
:10F580007E858F8598890E948CE269837A838B833C
:10F590009C8320E030E0A901C501B4010E9487E20C
:10F5A000882309F4F0C029813A814B815C81CA012A
:10F5B000B9010E94EDE26D8B7E8B8F8B988FA70136
:10F5C0009601C701B6010E94EDE29B01AC016D8975
:10F5D0007E898F89988D0E947DE96B017C01A50150
:10F5E0009401C501B4010E947EE99B01AC01C701F1
:10F5F000B6010E9401EA0E94A9EAA98DBA8D9596EA
:10F600008D909D90AD90BC909897750164012D816F
:10F610003E814F815885C21AD30AE40AF50A0E9436
:10F620007AEAC61AD70AE80AF90AF7FE6EC020E09D
:10F6300030E0A901C301B2010E9487E2882309F4E6
:10F64000A6C0C501B4010E948CE26B017C01A3013C
:10F650009201C301B2010E947EE99B01AC01C70186
:10F66000B6010E94EDE26B017C0129853A854B854C
:10F670005C85CA01B9010E94EDE29B01AC01C701A2
:10F68000B6010E947DE96B017C0129813A814B81A1
:10F690005C81CA01B9010E94EDE29B01AC01C70186
:10F6A000B6010E947EE96B017C0120E030E040E879
:10F6B00050E4C301B2010E94EDE29B01AC01C7011D
:10F6C000B6010E9401EA0E94EAE96B017C0120E098
:10F6D00030E0A9010E9401EB18161CF0C12CD12CBE
:10F6E0007601C701B6010E947AEA6D837E838F831B
:10F6F000988786169706A806B90620F48D829E8202
:10F70000AF82B886C12CD12C76018D819E81AF81CC
:10F71000B885E98DFA8D81A792A7A3A7B4A7C80ED3
:10F72000D91EEA1EFB1EC5A6D6A6E7A6F0AA298901
:10F730003A894B895C8922AF33AF44AF55AFFE960F
:10F740002D853E854F85588920833183428353839D
:10F750006A960FB6F894DEBF0FBECDBFDF91CF9192
:10F760001F910F91FF90EF90DF90CF90BF90AF90DF
:10F770009F908F907F906F905F904F90089560E082
:10F7800070E0CB01E5CE60E070E0CB0134CF60E00B
:10F7900070E0CB0198CF90916F0081E091FD02C0A5
:10F7A00080E0089590916F009D7F90936F00089581
:10F7B000CF93C82F0E94CB7B94E0C99F9001112466
:10F7C000F901E052FB4F24513B4FD9014D915D911E
:10F7D0006D917C91408351836283738391E0909318
:10F7E000DF04882319F0CF910C942E30CF91089527
:10F7F000CF92DF92EF92FF9280918404329B60C09F
:10F8000081608093840480918404339B5BC0826018
:10F810008093840480918404349B56C084608093D8
:10F820008404C090D004C0FE10C080919A0580FF6F
:10F830000CC08091840480FF08C08091AA0581607B
:10F840008093AA0580E00E94D87BD12CF12CE12C7A
:10F85000D701C601B695A7959795879580FF11C0EA
:10F8600080919A05869580FF0CC08091840481FF69
:10F8700008C08091AA0582608093AA0581E00E9459
:10F88000D87B82E0F694E794D794C7948A95D1F711
:10F89000C0FE1CC080919A058695869580FF16C093
:10F8A0008091840482FF12C08091AA0584608093B5
:10F8B000AA0582E0FF90EF90DF90CF900C94D87B68
:10F8C0008E7F9FCF8D7FA4CF8B7FA9CFFF90EF90AE
:10F8D000DF90CF9008950F931F93CF93DF93809184
:10F8E00049018F3708F447C08F579091A81490931F
:10F8F0001F05992309F43DC05D9A9091B40590933A
:10F900001E05992309F441C05C9A8F5F80934901D9
:10F9100080911D0591E0892780931D0581110E942A
:10F92000FE1E80914801C1E0C80F85300CF0C0E098
:10F93000823009F4D3C05CF5882309F43EC08130DD
:10F9400009F4C1C0C09348018091990581110E94BA
:10F95000F87B8091410690914206009729F001972B
:10F960009093420680934106DF91CF911F910F91B2
:10F9700008955D98C2CF90911F05891708F05D9892
:10F9800090911E05891708F4C0CF5C98BECF8430D3
:10F9900009F4BBC00CF4B5C08530A1F690911C05EC
:10F9A000911102C080931C0580911C0581508093A9
:10F9B0001C05882339F2C5E0C5CF809147018F5FD0
:10F9C00080311CF480934701BDCF10924701809194
:10F9D0007904811113C08091A0149091A114909387
:10F9E000A3148093A2148091AC059091AD059093DF
:10F9F000AF058093AE0581E0809379041092A11445
:10FA00001092A0141092AD051092AC050091A214B2
:10FA10001091A3148091A6149091A714D1E0181608
:10FA200019062CF08091A814811101C0D0E08091BA
:10FA30004E0190914F01081719073CF445EF52E22F
:10FA400062E073E280E00E94AF74DD2371F0809188
:10FA50004C0190914D01801791073CF444E153E231
:10FA600061E273E280E00E94AF740091B2051091F0
:10FA7000B3052091AE053091AF0580919605909128
:10FA80009705281739073CF445EF52E262E073E22C
:10FA90008FEF0E94AF74101611060CF053CF209117
:10FAA000AE053091AF0580914A0190914B018217CC
:10FAB00093070CF047CF44E153E261E273E28FEF2A
:10FAC0000E94AF743FCF10927B0087E480937C004C
:10FAD00080917A00806480937A0034CF80917A009C
:10FAE00086FD26C020917800309179008091A01485
:10FAF0009091A114820F931F9093A1148093A0144E
:10FB000021CF10927B0086E4E1CF80917A0086FDC0
:10FB100011C020917800309179008091AC059091CE
:10FB2000AD05820F931F9093AD058093AC050ACF6E
:10FB3000C2E008CFC4E006CF0E94CB7B10922B0618
:10FB400010922C0610922D0610922E0681110C9404
:10FB50002E3008950F931F9380911D1590911E15BF
:10FB6000891B8F7009F449C090911A15992361F08F
:10FB7000833040F48FEF890F29F080931A1590E0BD
:10FB800080E038C010921A1580911E152BE4829FD8
:10FB9000C00111248D5B994FFC01208120FDEFCF26
:10FBA00040912B0650912C0660912D0670912E06E7
:10FBB000E95BFF4F0081118122813381401B510B92
:10FBC000620B730B40932B0650932C0660932D060B
:10FBD00070932E0620911E152F5F2F7020931B15FA
:10FBE00030911E1520911C15321304C020911B1555
:10FBF00020931C151F910F9108950E949C7DBFCFEB
:10FC00002F923F924F925F926F927F928F929F922C
:10FC1000AF92BF92CF92DF92EF92FF920F931F931A
:10FC2000CF93DF9300D000D0CDB7DEB78FEF9FEF3B
:10FC300090938900809388000AE00983312C212C5D
:10FC400078948091D9049091DA04A091DB04B0916A
:10FC5000DC04892B8A2B8B2B09F0C4C18091DF0433
:10FC60008823E1F08091DD049091DE041092DF049E
:10FC7000892B09F4B7C11092DE041092DD041092B2
:10FC8000D00490911D1580911E15981709F4AAC1F2
:10FC900080911E158F5F8F7080931E158091DD04FB
:10FCA0009091DE04892B09F49DC14091D5045091B7
:10FCB000D6046091D7047091D8048091D1049091BA
:10FCC000D204A091D304B091D4040091C30410E0F5
:10FCD00030E020E0841B950BA60BB70B0817190723
:10FCE0002A073B0710F4D901C8018A83840F951FA6
:10FCF000A61FB71F8093D5049093D604A093D70472
:10FD0000B093D804E1E0C0909B04D0909C04E090B4
:10FD10009D04F0909E048091AB049091AC04A0915E
:10FD2000AD04B091AE04C80ED91EEA1EFB1EC092EF
:10FD3000AB04D092AC04E092AD04F092AE04F7FCB8
:10FD400033C040919304042E000C550B660B770BC7
:10FD50008091EC049091ED04A091EE04B091EF0439
:10FD6000840F951FA61FB71F8093EC049093ED049A
:10FD7000A093EE04B093EF048091970490919804BF
:10FD8000A0919904B0919A04A7019601281B390B00
:10FD90004A0B5B0BDA01C9018093AB049093AC046E
:10FDA000A093AD04B093AE0400919F041091A00401
:10FDB0002091A1043091A2048091AF049091B004ED
:10FDC000A091B104B091B204080F191F2A1F3B1F64
:10FDD0000093AF041093B0042093B1043093B204A5
:10FDE00037FD33C080919404082E000C990BAA0BA8
:10FDF000BB0B4091F0045091F1046091F2047091BA
:10FE0000F304840F951FA61FB71F8093F0049093EF
:10FE1000F104A093F204B093F304809197049091BD
:10FE20009804A0919904B0919A04B901A801481BC3
:10FE3000590B6A0B7B0BDB01CA018093AF049093D3
:10FE4000B004A093B104B093B2044091A3045091C4
:10FE5000A4046091A5047091A6048091B3049091CC
:10FE6000B404A091B504B091B604480F591F6A1F9D
:10FE70007B1F4093B3045093B4046093B504709314
:10FE8000B60477FD33C080919504082E000C990BC1
:10FE9000AA0BBB0B8090F4049090F504A090F6049C
:10FEA000B090F704880D991DAA1DBB1D8093F40422
:10FEB0009093F504A093F604B093F704809197040F
:10FEC00090919804A0919904B0919A042A013B0161
:10FED000481A590A6A0A7B0AD301C2018093B30403
:10FEE0009093B404A093B504B093B6048090A70493
:10FEF0009090A804A090A904B090AA048091B7049F
:10FF00009091B804A091B904B091BA04880D991DDC
:10FF1000AA1DBB1D8093B7049093B804A093B904A5
:10FF2000B093BA04B7FD33C040909604042C000C83
:10FF30005508660877088090F8049090F904A0901E
:10FF4000FA04B090FB04840C951CA61CB71C80928C
:10FF5000F8049092F904A092FA04B092FB04809005
:10FF6000970490909804A0909904B0909A042C0162
:10FF70003D01481859086A087B08530142018092E4
:10FF8000B7049092B804A092B904B092BA04E111F7
:10FF900004C0E0918400F0918500F7FE5F9A37FF7E
:10FFA000469A77FF2B9AB7FF299AE0918400F09147
:10FFB0008500E0918400F0918500F7FE5F9837FF9F
:10FFC000469877FF2B98B7FF29985A80552021F043
:10FFD00080918400909185000A8101500A83E0E0BD
:10FFE000011191CE8090560190905701A090580138
:10FFF000B090590181149104A104B10409F047C0E3
:020000021000EC
:100000008091E4059091E505009709F42FC023B194
:100010002470159800000000000000001816190652
:100020000CF0D7C02A9A00000000000000002B9AB4
:1000300034E03A950000E9F72B980000000000003A
:100040000000222309F4C7C02A9A00000000000023
:100050000000181619060CF0C0C08091E4059091BC
:10006000E50501979093E5058093E4050E94DE3253
:10007000882309F4B8C080ED97E0A0E0B0E0809359
:10008000560190935701A0935801B0935901809164
:10009000D9049091DA04A091DB04B091DC04892B9F
:1000A0008A2B8B2B09F053C4E091DD04F091DE0420
:1000B000309709F427C58091D5049091D604A0917A
:1000C000D704B091D8044091D1045091D2046091EA
:1000D000D3047091D40484179507A607B70708F4D2
:1000E00086C01092DE041092DD041092D00490912C
:1000F0001D1580911E15981709F404C580911E15D1
:100100008F5F8F7080931E1580EDC82E87E0D82EEC
:10011000E12CF12C8091DD049091DE04892B09F013
:100120000EC40E94AA7D9093DE048093DD04892B87
:1001300009F405C44090DD045090DE045C824B82DB
:10014000D2018C9183FFB3C2F201858D968DA78D6C
:10015000B0A1418D528D638D748D058916892789D3
:10016000308D0093EC041093ED042093EE04309353
:10017000EF044093F0045093F1046093F204709301
:10018000F3048093F4049093F504A093F604B093E1
:10019000F70481A192A1A3A1B4A18093F804909344
:1001A000F904A093FA04B093FB041092DE041092B9
:1001B000DD041092D00490911D1580911E159817A2
:1001C00009F4AFCF80911E158F5F8F7080931E153D
:1001D000A8CF2A9828CF2A9838CF8091E40590910B
:1001E000E50501963FCF8FEF9FEFDC0148CF4091AF
:1001F000CC045091CD046091CE047091CF04481787
:1002000059076A077B0708F4DEC08091C804909103
:10021000C904A091CA04B091CB0441A952A963A911
:1002200074A91127859F412C969F9001A69F300DA0
:10023000A59F200D311D869F400C211D311F959FCC
:10024000400C211D311FA49F400C211D311F949F84
:10025000410C211F311F4694211F311F789F200D13
:10026000311D799F300D112442AD53AD64AD75AD94
:10027000420F531F611D711D4093C4045093C50468
:100280006093C6047093C70406A917A920AD31ADC9
:10029000041715072607370740F40093C40410938A
:1002A000C5042093C6043093C7044090C404509002
:1002B000C5046090C6047090C70426ED31E201E0E9
:1002C0000A83F9014591559165917491441555053D
:1002D0006605770570F476946794579447941A816D
:1002E000110F1A832C5F3F4F42EF51E24217530721
:1002F00041F75A815093C30460E2461651046104E9
:10030000710428F410E2412E512C612C712C70E202
:10031000471A5108610871084114E8E05E0661045B
:10032000710408F42EC0F4E05F9E900111242A525B
:10033000324EF901329645915491042DEE27059FD6
:10034000B001049F610D7E1F06946E1F7E1F112455
:10035000AB0170E060E0F901C590D490F12CE12C84
:10036000C41AD50AE60AF70A8C0D9D1DAE1DBF1DE5
:100370008093C8049093C904A093CA04B093CB049B
:10038000C9CEB301A20176956795579547959A0115
:100390002C7F2A52364EF901C590D490F90132963D
:1003A00045915491142D1770149F9001159F300D95
:1003B0001124F3E036952795FA95E1F7C21AD30A8E
:1003C000F12CE12CD1CF4091BF045091C004609139
:1003D000C1047091C204481759076A077B0708F0E7
:1003E000D4C08091BB049091BC04A091BD04B09195
:1003F000BE0441A952A963A974A92227859F312D62
:10040000969F8001A69F100DA59F000D111D869F30
:10041000300D011D121F959F300D011D121FA49F4D
:10042000300D011D121F949F310D021F121F3695B2
:10043000021F121F789F000D111D799F100D1124AE
:1004400030E020E04091C4045091C5046091C6049E
:100450007091C704FE9640805180628073800417BB
:1004600015072607370758F4401B510B620B730B17
:10047000441655066606770610F42A013B0126ED60
:1004800031E241E04A83F9014591559165917491BA
:10049000441555056605770570F47694679457946E
:1004A00047945A81550F5A832C5F3F4F62EF71E298
:1004B0006217730741F77A817093C304E0E24E1626
:1004C00051046104710428F400E2402E512C612C87
:1004D000712CF0E24F1A510861087108411408E0CC
:1004E00050066104710408F42EC014E0519E90017E
:1004F00011242A52324EF901329645915491F42D2D
:10050000EE27F59FB001F49F610D7E1F06946E1FCC
:100510007E1F1124AB0170E060E0F901C590D4901A
:10052000F12CE12CC41AD50AE60AF70A8C0D9D1DA0
:10053000AE1DBF1D8093BB049093BC04A093BD046B
:10054000B093BE04E7CDB301A201769567955795A8
:1005500047959A012C7F2A52364EF901C590D490C6
:10056000F901329645915491042D0770049F900132
:10057000059F300D112413E0369527951A95E1F764
:10058000C21AD30AF12CE12CD1CF80914301909172
:100590004401A0914501B0914601B7FF5DC0C6A8D6
:1005A000D7A8E0ACF1AC86ED91E221E0FC014591E9
:1005B0005591659174914C155D056E057F0558F454
:1005C000F694E794D794C794220F049642EF51E231
:1005D0004817590759F72093C30450E2C516D104B0
:1005E000E104F10428F470E2C72ED12CE12CF12CA7
:1005F00060E2C61AD108E108F108C11478E0D70614
:10060000E104F10408F431C0A4E0DA9EC001112431
:100610008A52924EFC01329625913491BC2D662768
:10062000B39FA001B29F410D561F0694461F561F4F
:10063000112470E060E0FC0185919491B0E0A0E0AD
:10064000841B950BA60BB70B809343019093440139
:10065000A0934501B0934601C0904301D09044015E
:10066000E0904501F090460155CDD701C601B69501
:10067000A795979587958C7F8A52964EFC01259178
:100680003491FC01329645915491EC2DE770E49F32
:10069000C001E59F900D112463E0969587956A95BA
:1006A000E1F7281B390BC901B0E0A0E0CDCFAB8149
:1006B000BC8155960D911D912D913C91589781E0EB
:1006C000011511052105310509F480E0EB81FC815C
:1006D000C18CD28CE38CF48CC114D104E104F104FC
:1006E00009F08260AB81BC815D964D915D916D9109
:1006F0007C919097411551056105710509F0846061
:100700008093D0041092BB041092BC041092BD04DC
:100710001092BE041092C8041092C9041092CA0428
:100720001092CB04EB81FC8185A196A1A7A1B0A575
:100730008093D1049093D204A093D304B093D404B3
:10074000442455243201481A590A6A0A7B0A409205
:10075000AB045092AC046092AD047092AE0440922F
:10076000AF045092B0046092B1047092B20440920F
:10077000B3045092B4046092B5047092B6044092EF
:10078000B7045092B8046092B9047092BA0441A0C0
:1007900052A063A074A0440C551C661C771C000F6B
:1007A000111F221F331F00939B0410939C0420935E
:1007B0009D0430939E04CC0CDD1CEE1CFF1CC092EB
:1007C0009F04D092A004E092A104F092A204440FEE
:1007D000551F661F771F4093A3045093A404609392
:1007E000A5047093A6044092A7045092A8046092B6
:1007F000A9047092AA04880F991FAA1FBB1F809397
:10080000970490939804A0939904B0939A0410923B
:10081000D5041092D6041092D7041092D80481A562
:1008200092A5A3A5B4A58093CC049093CD04A093E6
:10083000CE04B093CF0485A596A5A7A5B0A98093B3
:10084000BF049093C004A093C104B093C20485A9CF
:1008500090919A05891721F080939A050E9432762B
:100860008091990581110E94F87B44244A94542C6C
:1008700032014092430150924401609245017092CE
:100880004601AB81BC81DA964D915D916D917C9171
:10089000DD974093C4045093C5046093C6047093DD
:1008A000C70486ED91E2A1E0FC0105911591259127
:1008B0003491041715072607370758F4769567957E
:1008C00057954795AA0F0496E2EFF1E2E817F9076A
:1008D00059F7A093C304403251056105710520F416
:1008E00040E250E060E070E0405251096109710956
:1008F0004115F8E05F076105710508F4DAC004E00E
:10090000509FC00111248A52924EFC0132962591CB
:100910003491AA27439FF001429FE10DFA1F0694EC
:10092000EA1FFA1F1124AF0170E060E0FC01C590DE
:10093000D490F12CE12CC41AD50AE60AF70AC09229
:10094000D904D092DA04E092DB04F092DC04892826
:100950008A288B28C9F48091D9049091DA04A09157
:10096000DB04B091DC048A3F9105A105B10560F478
:100970002AEF30E040E050E02093D9043093DA04CD
:100980004093DB045093DC04409156015091570191
:1009900060915801709159010091D9041091DA04C5
:1009A0002091DB043091DC044F3F8FEF580768073C
:1009B000780799F0D901C801B695A79597958795BD
:1009C000481759076A077B0740F4809356019093B4
:1009D0005701A0935801B09359014091560150918D
:1009E000570160915801709159014F3F9FEF59078E
:1009F0006105710508F07DC04B835A83F62FE72F00
:100A00008B819A81AF2FBE2F081719072A073B0742
:100A100010F4D901C801081B190B2A0B3B0B0093DA
:100A2000D9041093DA042093DB043093DC044F3FA5
:100A3000EFEF5E076E077E0761F0481B590B6A0BEC
:100A40007B0B40935601509357016093580170936C
:100A50005901F8942091840030918500205F3F4F28
:100A6000098101500983002309F44AC0280E391E68
:100A70002216330610F40C94207E309289002092C6
:100A8000880078940F900F900F900F90DF91CF9186
:100A90001F910F91FF90EF90DF90CF90BF90AF909C
:100AA0009F908F907F906F905F904F903F902F908E
:100AB0000895DB01CA01B695A795979587958C7F18
:100AC0008A52964EFC01C590D490FC013296259135
:100AD00034914770429FC001439F900D1124A3E0C1
:100AE00096958795AA95E1F7C81AD90AF12CE12CB9
:100AF00026CFAFEFAB83BFEFBA83F0E0E0E080CF6B
:100B00001901BBCF80EDC82E87E0D82EE12CF12C47
:100B100008CBFC0120813181428153816091140B0B
:100B20007091150B8091160B9091170B0E94EDE2BE
:100B30000E9406EB60932B1570932C1580932D1556
:100B400090932E1590911D1580911E1598130C945D
:100B5000BD650E94A4790E94CB7B40912B155091DA
:100B60002C1560912D1570912E154093F80450931B
:100B7000F9046093FA047093FB0481110C942E30F5
:100B800008954F925F926F927F928F929F92AF9251
:100B9000BF92CF92DF92EF92FF920F931F93CF936A
:100BA000DF93EC018B015A01F9012091140B309174
:100BB000150B4091160B5091170B6081718182814A
:100BC00093810E94EDE20E9406EB6B017C01209173
:100BD000100B3091110B4091120B5091130BF5013A
:100BE00060817181828193810E94EDE20E9406EB17
:100BF0004B015C0120910C0B30910D0B40910E0BC1
:100C000050910F0BF80160817181828193810E9464
:100C1000EDE20E9406EB2B013C012091080B309184
:100C2000090B40910A0B50910B0B688179818A81E5
:100C30009B810E94EDE20E9406EB60931F1570936A
:100C400020158093211590932215409223155092E0
:100C50002415609225157092261580922715909282
:100C60002815A0922915B0922A15C0922B15D09262
:100C70002C15E0922D15F0922E1590911D15809156
:100C80001E15981791F0DF91CF911F910F91FF9052
:100C9000EF90DF90CF90BF90AF909F908F907F901C
:100CA0006F905F904F900C94BD650E94A4790E9454
:100CB000CB7B409127155091281560912915709193
:100CC0002A15009123151091241520912515309196
:100CD0002615C0901F15D0902015E0902115F0909A
:100CE0002215C092EC04D092ED04E092EE04F09252
:100CF000EF040093F0041093F1042093F204309376
:100D0000F3044093F4045093F5046093F604709355
:100D1000F70440912B1550912C1560912D15709171
:100D20002E154093F8045093F9046093FA047093DD
:100D3000FB04882391F0DF91CF911F910F91FF90D9
:100D4000EF90DF90CF90BF90AF909F908F907F906B
:100D50006F905F904F900C942E30DF91CF911F9148
:100D60000F91FF90EF90DF90CF90BF90AF909F904A
:100D70008F907F906F905F904F900895CF92DF9209
:100D8000EF92FF92CF93DF93C82F0E94CB7B94E02A
:100D9000C99FE0011124FE01E451FB4FC080D180C6
:100DA000E280F38081110E942E30C05DD94FC701CF
:100DB000B6010E948EE2288139814A815B810E94BE
:100DC000EDE2DF91CF91FF90EF90DF90CF9008950B
:100DD000CF92DF92EF92FF92CF93DF93C82F0E94C2
:100DE000CB7B94E0C99FE0011124FE01E052FB4F50
:100DF000C080D180E280F38081110E942E30C05DDE
:100E0000D94FC701B6010E948EE2288139814A81FB
:100E10005B810E94EDE2DF91CF91FF90EF90DF9038
:100E2000CF900895CF930E94CB7BC82F80911E1541
:100E300080931D1580931C1580931B1584E6809369
:100E40001A150E949C7D80ED93E09093420680935A
:100E50004106C1110E942E3081E08093DF04CF91C2
:100E60000895CF93DF9324E0829FC0011124EC0109
:100E7000C750DA4FFC01E456FA4F88519C4FDC0111
:100E80002D913D914D915C91608171818281938121
:100E90000E947EE9688379838A839B83DF91CF9167
:100EA000089580FF04C09091850490FD8E7F81FF9E
:100EB00005C090918504969590FD8D7F82FF06C0B8
:100EC000909185049695969590FD8B7F0895CF928D
:100ED000DF92EF92FF920F931F93C12CD12C7601DA
:100EE0008C0128E43BE044E45BE060E47BE08CE3DD
:100EF0009BE00E949FBB1F910F91FF90EF90DF90AE
:100F0000CF9008954F925F926F927F928F929F92AF
:100F1000AF92BF92CF92DF92EF92FF920F931F9307
:100F2000CF93DF93CDB7DEB72C970FB6F894DEBF23
:100F30000FBECDBF2B013C0129873A874B875C87C9
:100F400047015801F601E080F1800281138120E021
:100F500030E0A901B701C8010E9487E2882309F4A3
:100F600084C05E2D4F2D302F212F852F942FA32F3E
:100F7000B22F89839A83AB83BC8320E030E0A90140
:100F8000B701C8010E9487E2811104C0E12CF12C55
:100F900008E413E4C701D8018D839E83AF83B8872B
:100FA000A50194016091440B7091450B8091460B13
:100FB0009091470B0E9487E287FF0CC08092440B00
:100FC0009092450BA092460BB092470BCE01019632
:100FD0000E94678740923C0B50923D0B60923E0B03
:100FE00070923F0B89859A85AB85BC858093400BB9
:100FF0009093410BA093420BB093430BCE01059607
:101000000E946787A50194016091440B7091450B84
:101010008091460B9091470B0E9401EB181664F4E7
:101020008092440B9092450BA092460BB092470BD6
:10103000CE0101960E9467870E94A4792C960FB674
:10104000F894DEBF0FBECDBFDF91CF911F910F91FE
:10105000FF90EF90DF90CF90BF90AF909F908F90D8
:101060007F906F905F904F90089550E040E030E89F
:1010700020E47BCFCF92DF92EF92FF920F931F93EA
:101080006B01FC01E080F18002811381ECE3FBE065
:10109000248135814681578160817181828193816C
:1010A0000E9482871F910F91FF90EF90DF90CF9069
:1010B00008950C9401BC2F923F924F925F926F92D1
:1010C0007F928F929F92AF92BF92CF92DF92EF92D8
:1010D000FF920F931F93CF93DF93CDB7DEB76C973B
:1010E0000FB6F894DEBF0FBECDBF8091780481119A
:1010F00050C18091770481113CC1809179048111A4
:1011000019C06C960FB6F894DEBF0FBECDBFDF914D
:10111000CF911F910F91FF90EF90DF90CF90BF90F4
:10112000AF909F908F907F906F905F904F903F9087
:101130002F9008950E9497740E945AC34B015C013E
:101140000091A4141091A514809152019091530123
:10115000801791070CF448C26091A6147091A714EF
:10116000072E000C880B990B0E948EE26D837E8304
:101170008F839887B801110F880B990B0E948EE21C
:1011800069837A838B839C832AE0E22EF12C0CE323
:1011900010E020E0AE014B5F5F4FBE016F5F7F4FFD
:1011A00088E095E10E9410750091A4141091A51497
:1011B0008091500190915101801791070CF4F0C07B
:1011C00060E06093A81480919C1490919D14A0916C
:1011D0009E14B0919F140097A105B10539F1A501A6
:1011E0009401281B390B4A0B5B0BDA01C901B7FDCF
:1011F0001DC080919A1490919B14081719070CF444
:1012000013C28091A6149091A714009739F00E5F35
:101210001F4F0497081719070CF41CC210929C1456
:1012200010929D1410929E1410929F148091B005FC
:101230009091B105873991050CF0E2C180911805B4
:1012400090911905A0911A05B0911B050097A10571
:10125000B10561F1A5019401281B390B4A0B5B0B09
:10126000DA01C901B7FD22C08091B0059091B105A6
:101270002091160530911705821793070CF4CCC105
:101280002091B2053091B3052115310539F0029650
:1012900024503109821793070CF4EFC110921805FE
:1012A0001092190510921A0510921B0580911205D3
:1012B00090911305A0911405B0911505A501940115
:1012C000281B390B4A0B5B0BDA01C901B7FD19CF9B
:1012D00038E8830E33E1931EA11CB11C80921205E5
:1012E00090921305A0921405B09215056091B20575
:1012F0007091B305072E000C880B990B0E948EE2AB
:101300006D837E838F8398876091B0057091B1055E
:10131000072E000C880B990B0E948EE269837A835A
:101320008B839C8382E0E82EF12C02E310E02FEF08
:10133000AE014B5F5F4FBE016F5F7F4F81E195E173
:101340000E9410758091B0059091B1059C012550C7
:1013500031092239310508F05BC12091B205309185
:10136000B305821793070CF467C180E08093B4053E
:10137000C8CE109277040E9412870E94A4790E941E
:101380003ABB0E94598880917904882309F4B9CE28
:10139000D1CE41E070E060E087E492E20E94BD3986
:1013A0008091520190915301081719070CF008CF52
:1013B000E090A614F090A714B801012E000C880B41
:1013C000990B0E948EE21B012C01E114F10409F437
:1013D0003CC1B701601B710B072E000C880B990BE9
:1013E0000E948EE26B017C0120E030E040E251EC93
:1013F0000E9487E287FD29C120E030E040E251E40D
:10140000C701B6010E9401EB18160CF449C1809186
:101410001105811149C12091090530910A054091BA
:101420000B0550910C0529873A874B875C87809183
:101430000D0590910E05A0910F05B09110058D87B7
:101440009E87AF87B88BA20191016091FD047091D6
:10145000FE048091FF04909100050E947DE9209197
:10146000B1143091B2144091B3145091B4140E944D
:10147000EDE229853A854B855C850E947DE920ED6A
:101480003CEC4CE45DE30E94EDE229853A854B8516
:101490005C850E947EE9698B7A8B8B8B9C8B609339
:1014A000090570930A0580930B0590930C05209114
:1014B000AD143091AE144091AF145091B0142D8BF7
:1014C0003E8B4F8B588F2D853E854F855889C701A0
:1014D000B6010E947EE9762E672E89879D8720E0DF
:1014E00030E0A9010E9487E287FDE9C02D893E898D
:1014F0004F89588D60E070E08FE793E40E9401EA25
:10150000698F7A8F8B8F9C8F272D362D49855D852E
:101510000E9487E287FF06C0798C6A8C3B8D3987F1
:101520004C8D4D87872D962DA985BD8580930D0502
:1015300090930E05A0930F05B09310052091A91468
:101540003091AA144091AB145091AC14C701B6016C
:101550000E94EDE26B017C01C0920105D092020570
:10156000E0920305F0920405272D362D49855D850F
:101570006D897E898F89988D0E94EDE29B01AC0177
:101580002093050530930605409307055093080501
:10159000C701B6010E947EE929893A894B895C8995
:1015A0000E947EE920E030E0A9010E947EE96B0103
:1015B0007C0120E030E0A9010E9487E287FD48C05D
:1015C00020E030E04FE753E4C701B6010E9401EB91
:1015D0001816A4F56FE72092FD043092FE044092A5
:1015E000FF0450920005EDCD45EF52E262E073E258
:1015F00080E00E94AF740091A4141091A514ACCDAA
:1016000045EF52E262E073E28FEF0E94AF7416CEB4
:101610001092B4055C9875CD49E252E268E372E23B
:101620008FEF0E94AF7442CE49E252E268E372E269
:1016300080E00E94AF74FACD8FE798CEC701B60163
:101640000E9473EA75956795C6CF81E08093110576
:1016500060E0C1CF10939B1400939A140E945AC368
:10166000605B7C438F4F9F4F60939C1470939D14DD
:1016700080939E1490939F14D9CD909317058093D7
:1016800016050E945AC3605E70448D4F9F4F609351
:1016900018057093190580931A0590931B0506CEC3
:1016A00081E08093110596CF109211051D861E864C
:1016B0001F86188A19861A861B861C86C4CE712C32
:1016C000612C19861D862ECF2F923F924F925F92EA
:1016D0006F927F928F929F92AF92BF92CF92DF9242
:1016E000EF92FF920F931F93CF93DF93CDB7DEB7A7
:1016F000A6970FB6F894DEBF0FBECDBF809127012D
:10170000882309F4CDC080918504C82ED12CF12CFA
:10171000E12C80FF3CC08090290190902A01A0908C
:101720002B01B0902C012091F4033091F5034091EE
:10173000F6035091F703C501B4010E9401EB18169E
:1017400044F48092F4039092F503A092F603B092D1
:10175000F7038090350190903601A0903701B0904A
:1017600038012091F4033091F5034091F603509134
:10177000F703C501B4010E9487E287FF08C0809289
:10178000F4039092F503A092F603B092F703D70109
:10179000C601B695A7959795879580FF3CC0809028
:1017A0002D0190902E01A0902F01B090300120913A
:1017B000F8033091F9034091FA035091FB03C501FE
:1017C000B4010E9401EB181644F48092F803909241
:1017D000F903A092FA03B092FB0380903901909034
:1017E0003A01A0903B01B0903C012091F803309168
:1017F000F9034091FA035091FB03C501B4010E9423
:1018000087E287FF08C08092F8039092F903A092C4
:10181000FA03B092FB0392E0F694E794D794C7944E
:101820009A95D1F7C0FE3CC0C0903101D0903201F2
:10183000E0903301F09034012091FC033091FD03DE
:101840004091FE035091FF03C701B6010E9401EBD6
:10185000181644F4C092FC03D092FD03E092FE03FC
:10186000F092FF03C0903D01D0903E01E0903F0117
:10187000F09040012091FC033091FD034091FE0364
:101880005091FF03C701B6010E9487E287FF08C09D
:10189000C092FC03D092FD03E092FE03F092FF039E
:1018A0008091F30A83FD7EC02091480B3091490B53
:1018B00040914A0B50914B0B6091000470910104D0
:1018C00080910204909103040E9487E2882309F426
:1018D00069C010914006111161C080915E01909124
:1018E0005F0101972091A4143091A514281739079E
:1018F0003CF40E9494398BEA96E10E94CF3811E0C3
:101900002091480B3091490B40914A0B50914B0B61
:10191000609100047091010480910204909103048D
:101920000E947DE96B017C0120E030E0A9010E946A
:1019300001EB87FF04C0F7FAF094F7F8F0942091D8
:101940005A0130915B0140915C0150915D01C701EA
:10195000B6010E94EDE220E030E84BE354E40E943F
:1019600001EB1816ECF40E9494398CE896E10E9481
:10197000CF388091000490910104A0910204B091AD
:1019800003048093480B9093490BA0934A0BB093A8
:101990004B0B80E094E00E94898504C010E0B0CF3A
:1019A0001111E7CF2AE037ED43E25CE360912101BA
:1019B0007091220180912301909124010E94EDE217
:1019C0006B017C0160911F0170912001072E000CBA
:1019D000880B990B0E948EE29B01AC01C701B601F6
:1019E0000E94EDE2698B7A8B8B8B9C8B8091080433
:1019F000882309F46CC020913C0B30913D0B409141
:101A00003E0B50913F0B6091F4037091F503809170
:101A1000F6039091F7030E947DE96D8B7E8B8F8B8F
:101A2000988F2091400B3091410B4091420B509187
:101A3000430B6091F8037091F9038091FA03909140
:101A4000FB030E947DE9698F7A8F8B8F9C8F209199
:101A5000440B3091450B4091460B5091470B6091E0
:101A6000FC037091FD038091FE039091FF030E949F
:101A70007DE96D8F7E8F8F8F98A32091480B3091D9
:101A8000490B40914A0B50914B0B609100047091AF
:101A9000010480910204909103040E947DE96B018E
:101AA0007C0120E030E0A9016D897E898F89988DC5
:101AB0000E9487E281110FC020E030E0A901698D0A
:101AC0007A8D8B8D9C8D0E9487E2811104C0C12C80
:101AD000D12C76012CC12D893E894F89588DCA01A0
:101AE000B9010E94EDE24B015C01298D3A8D4B8DCD
:101AF0005C8DCA01B9010E94EDE29B01AC01C501F8
:101B0000B4010E947EE94B015C012D8D3E8D4F8D0D
:101B100058A1CA01B9010E94EDE29B01AC01C501C7
:101B2000B4010E947EE94B015C01A7019601C70147
:101B3000B6010E94EDE29B01AC01C501B4010E9417
:101B40007EE90E943FEB4B015C012DEB37E346E859
:101B500055E30E9487E287FF0FC020E030E0A90133
:101B6000C701B6010E9401EB4601570187FF04C07F
:101B7000B7FAB094B7F8B0942DEB37E346E855E3E5
:101B8000C501B4010E9487E287FDDEC020E030E09D
:101B900040EA51E4C501B4010E9401EA0E947AEAD8
:101BA0001B01672B19F422242394312CB10190E0FE
:101BB00080E00E948CE29B01AC0160E070E080E874
:101BC0009FE30E9401EA2B013C01AC019B01C5018E
:101BD000B4010E94EDE24B015C01A30192016D8909
:101BE0007E898F89988D0E94EDE26D8B7E8B8F8B25
:101BF000988FA3019201698D7A8D8B8D9C8D0E94A7
:101C0000EDE2698F7A8F8B8F9C8FA30192016D8D8E
